:020000040800F2
:10000000002000108DDB0208D1CA0108FDA4000801
:10001000CDCA0108C9CA0108C5CA0108000000000C
:10002000000000000000000000000000C1CA01083C
:10003000BDCA010800000000B9CA0108FFBB0008E2
:10004000F5DB0208F5DB0208F5DB0208F5DB020848
:10005000F5DB0208F5DB02080D230008392400084F
:10006000FD230008C12300088523000845820008FD
:1000700035820008258200081582000805820008E4
:10008000F1810008DD810008F5DB0208F5DB0208DC
:100090000DF80108F5DB0208F5DB0208492300082A
:1000A000F5DB0208F5DB0208F5DB0208F5DB0208E8
:1000B000F5AD000839AD00087DAC0008F5DB02089D
:1000C000F5DB0208F5DB0208F5DB0208F5DB0208C8
:1000D000F5DB0208F5DB0208F5DB0208FDE60008A7
:1000E000D1220008F5DB0208A9CA0108F5DB0208E5
:1000F000EDAA0008F5DB0208B5AB0008F5DB020845
:10010000000000000000000000000000F5DB020815
:10011000F5DB0208F5DB0208F5DB0208F5DB020877
:10012000C9810008B5810008A18100088D810008FF
:1001300079810008F5DB02080000000000000000E3
:10014000F5DB0208F5DB0208F5DB02080000000021
:10015000000000000000000000000000000000009F
:100160000000000000000000F5DB0208F5DB0208DB
:10017000F5DB0208000000000000000000000000A5
:0801800000000000F5DB02089D
:100188002B2303732A238370002383757047036826
:100198002DE9F0415D6A1DB12B46BDE8F0411847D5
:1001A800002A174611DD04460E460F4400E0236876
:1001B8009B68204698470028F9D0236816F8011B49
:1001C8001B6820469847BE42F1D1BDE8F08103681C
:1001D8001B69184700232322027043708370C37081
:1001E80070470B4B984211D0A3F57843984202D040
:1001F8004FF0FF3070470122064B03EB02135A8978
:10020800013292B25A81588980B270470022F3E7CE
:10021800003001406443002008B5838940F2E93387
:1002280000E09BB10289013B12F0020F9BB2F8D0AB
:10023800017340F2E93300E043B10289013B12F057
:10024800010F9BB2F8D0007BC0B208BDFFF7C9FF11
:10025800C0B208BDF8B50546806816461F4610B1FD
:10026800036882881A85686840F2E934838901E066
:10027800002C44D00389013C13F0020FA4B2F7D03C
:10028800017340F2E93101E0002938D003890139CE
:1002980013F0010F89B2F7D0037B686883894FF0A8
:1002A800000C4FF47A714FF6FF724FF0FF0E67455E
:1002B80002D11DE0914219D0038901399C0789B206
:1002C800F8D580F80CE04FF47A7102E0A1B29142BF
:1002D8000CD00389DB0701F1FF34F7D5037BDBB2D0
:1002E8000EB1337001360CF1010CE0E7FFF779FF2E
:1002F800AB6813B11A689B8893610120F8BDFFF7BA
:1003080070FFCAE7836810B5044613B11A689B8862
:100318001385606840F2E933828900E0BBB1028945
:10032800013B12F0020F9BB2F8D0017340F2E9339F
:1003380000E063B10289013B12F0010F9BB2F8D0D3
:10034800037BA36813B11A689B88936110BDFFF7FC
:1003580048FFF6E7437A5A1C0344D2B242729972B4
:10036800037A93420AD84AB110B5044604F10A0147
:10037800D0E9003098470023637210BD704720B160
:100388000078B0FA80F0400970470120704703797F
:1003980003F01803082B0AD002D82BB100207047AD
:1003A800102B16D0182BF9D1B0F80B007047124B50
:1003B800B0F80B0093F90030591C06BF0F4B1B789F
:1003C800DBB2C3EB0312C3EB820300EB430080B242
:1003D8007047094BB0F80B0093F901305A1C06BF5F
:1003E800064B5B78DBB203EB430203EB820300EBC3
:1003F800430080B2704700BF00000020245C00204A
:10040800F0B5067906F06003402B09D144794FF026
:10041800FF350023012006F00706A3420BD1F0BDEB
:10042800602B08BF45794FF001040CBF04FA05F5AD
:100438004FF0FF35EDE7042E0CD8DFE806F0030D8A
:1004480018242E0030B1C85CD75C784028420CBF15
:10045800012000200133E0E70028FBD0C856D7561A
:10046800A0EB070CDCF1000040EB0C00F2E70028E1
:10047800F0D031F8130032F81370784028420CBFDE
:1004880001200020E6E70028E4D031F9130032F912
:100498001370C71B78427841DCE70028DAD051F89E
:1004A800230052F82370784028420CBF0120002016
:1004B800D0E74FE790ED057A90ED004AD0ED066A57
:1004C800D0ED014AD0ED047A90ED035AD0ED025AEE
:1004D800A4EE007AB0EE406AB0EE470AB0EE667A53
:1004E800A4EE867A67EEC07AA5EE407AE5EE867AC3
:1004F80080ED057AC0ED067A7047D0ED057A90ED6B
:10050800013AD0ED003AD0ED064A90ED024A90ED5E
:10051800077A90ED035A90ED086AD0ED045AC0EDC1
:10052800067AF0EE406A27EE830AC0ED056AA3EE6C
:10053800A60A80ED087AA4EE240AA5EE470AA5EEDD
:10054800C60A80ED070A7047D0ED007A90ED017A6F
:1005580030EE670AE7EE007AB0EE670AC0ED007A7F
:10056800704770470378202B024600F10100F9D04C
:10057800092BF7D02D2B00F0A4802B2B03BF537829
:10058800B7EE000A0246B7EE000AA3F13001C8B27E
:1005980009289FED577A10D8F2EE046A07EE901AF0
:1005A800F8EEE77A12F8013FE7EE267AA3F1300178
:1005B800C8B20928B0EE677AF0D92E2B63D003F0C1
:1005C800DF03452B02D020EE070A704710B451789C
:1005D8002D294FD02B2979D0A1F13003092B02F115
:1005E80001027AD80024002303EB830301EB4303C1
:1005F80012F8011FA1F130000928A3F13003F3D943
:10060800B3F59A7F1A4628BF4FF49A72072B6CD914
:10061800DFED386A1346F7EE007A083B072B67EEE2
:10062800A67AFAD802F00702DAB1F2EE046A012AD1
:1006380067EEA67A15D0022A67EEA67A11D0032AA9
:1006480067EEA67A0DD0042A67EEA67A09D0052AA5
:1006580067EEA67A05D067EEA67A062A18BF67EE77
:10066800A67A002C3BD087EE277A5DF8044B20EE63
:10067800070A70479178A1F13003092B02F10202B1
:1006880030D80124AFE75378A3F13001C8B2092864
:1006980002F1010293D8F2EE046AF0EE665A07EE10
:1006A800901AF8EEE77A12F8013F87EEA66AA3F1EE
:1006B8003001C8B2092866EEA56A37EE067AEED987
:1006C8007DE75378BFEE000A02465EE79178A1F114
:1006D8003003092B02F1020284D9F7EE007A27EEE3
:1006E800277AC2E7F7EE007ABDE7F7EE007A9BE7D4
:1006F8000000000020BCBE4C0028F0B403DA2D2313
:100708000B7040420131092804464FF0010307DD10
:1007180003EB83035B00B0FBF3F2092AF8D883B13B
:100728000F48A0FB0326B4FBF3F2092A02F1570C89
:1007380002F1300709DD03FB1244F30801F801CB8D
:10074800EFD100230B70F0BC704703FB1244F30891
:1007580001F8017BE5D100230B70F0BC704700BFA6
:10076800CDCCCCCC884270B44FF0010442D301FB0D
:1007780004F4B0FBF4F58D42F9D2ECB142BB092D7B
:1007880004FB150005F1570605F130020EDDB4FB38
:10079800F1F403F8016B7CB1B0FBF4F5092D04FB0F
:1007A800150005F1570605F13002F0DCB4FBF1F451
:1007B80003F8012B002CEFD100221A7070BC70478F
:1007C80003F8016BB4FBF1F4002CF5D0B0FBF4F5A1
:1007D800092D04FB150005F1370605F13002EFDCA1
:1007E800B4FBF1F403F8012B002CEFD100221A70AE
:1007F80070BC70470546002AEAD1C0E72DE9F047EA
:1008080014461D4606464FF47A72002320462946B0
:100818002CF0ECFF4D4BDFF848814D4A4D4F034417
:1008280088FB03101844D91782FB032CC1EB601016
:1008380088FB002887FB03279C44474AC1EBEC2C24
:10084800C0EB001E82FB0C29A3EB8E0E1F44434A0B
:1008580086F806E0C1EB27474FEAEC7E08EB000A72
:10086800CEEBA90E82FB07824FEAE0780EEB4E0E24
:10087800C8EB6A18ACEBCE0CC8EB0818DFF8E4E05C
:1008880086F804C0A0EB880070718EFB0303F8178C
:10089800C0EBE21240F2B55000FB1272C1EBE35319
:1008A800B2F5896F4FEA83073CDA40F2DA239A42BD
:1008B80042DCB2F5B77FB4BF4FF0000E4FF0010E27
:1008C8004FEA4E09DFF8A08009EB0E0308EBC303DB
:1008D8001FFA8EFCD88A09EB0E0108EBC10116310C
:1008E8000B2301E031F8020D904218DD013BF9D1EC
:1008F800CE44012338F83E00B37007F5FA67013299
:10090800121ABC44F270A6F800C0204629464FF4DB
:100918007A7200232CF06AFF3281BDE8F087013338
:10092800DBB2E9E74FF0030CE64640F29650DFF8F9
:1009380038804FF00609CEE74FF0020CDFF8288028
:10094800E64640F229404FF00409C4E780BC92C74C
:10095800C5B3A29107452EC2ABAAAA2A73B06D16D9
:1009680089888888792D0311E0E0020803685A1CF9
:100978000260197070472DE9F047089C2578002B14
:10098800804689460CBF4FF0200A4FF0300A661C9B
:1009980025B3002A26DD334601E0024698B113F854
:1009A800011B501E0029F8D1971E60B13D46013D3C
:1009B80051464046C8476B1C002BF8DC257827EACF
:1009C800E770013045B1041B29464046C847301935
:1009D80016F8015B002DF7D1BDE8F087002A03DC8B
:1009E8002846F9E70020EEE7571EDFE7034600F147
:1009F8001001FF221A705A7002338B42FAD1027129
:100A0800427170470123212100224170C270037096
:100A18008370704730B41522162317252D242E21F4
:100A2800027043702F22FF23857044718171C27157
:100A380043738373C37003710372437230BC70478E
:100A480030B40B222C23022518241921027043727A
:100A58001A22002385728473C1720273437330BCF7
:100A68007047094B09498B4203D309E014338B4281
:100A780006D21A88C2F30B029042F7D11846704783
:100A880000231846704700BFEC6B03084C7003083E
:100A980070B50546B0F80900FFF7E3FF064B1E786E
:100AA80004462846FFF773FC16B1A368184470BDC6
:100AB80063681844FBE700BFF80F002038B5054607
:100AC8000C46FFF7E5FF2A7902F0070302F06002FF
:100AD800602A28D1022B0ED0042B18D03BB96A7992
:100AE80001239340DBB2027814B11343037038BD7D
:100AF80022EA0303FAE76A79012393409BB202884A
:100B080014B113430380F2E722EA0303FAE76A7990
:100B1800012303FA02F2036814B113430360E6E702
:100B280023EA0203FAE7042BE1D8DFE803F0030322
:100B3800050507000470DAE70480D8E70460D6E703
:100B480030B402230025012414213D22057084704D
:100B5800C17082714370C37130BC70470023062195
:100B68004FF47A720170C0E9012303737047C0B172
:100B7800B9B110B40B4B9B780B2B01F1010114BFD9
:100B880010241C2402380C440A7811F8013C023164
:100B980043EA02238C4220F8023FF5D15DF8044B6A
:100BA80070477047000000204FF4006303837047CC
:100BB800012380F850307047F0B5836983B006464A
:100BC80013B11A689B8813857069DFF8A0C0838900
:100BD800C3244FF47A7306276D464FF6FF710CF164
:100BE800010C03E0013B9BB28B421CD002899207A7
:100BF800F8D504734FF47A7302E0A3B28B4212D093
:100C08000289D20703F1FF34F7D5027BD2B20DB1C6
:100C18002A7001354FB1013FFF24BCF1000FE5D028
:100C28009CF80040DBE7FFF7DCFAB36913B11A68F8
:100C38009B8893619DF805009DF801509DF802106E
:100C48009DF803409DF804209DF8063041EA0521EF
:100C580043EA002342EA04220120A6F85010A6F82D
:100C68005220A6F8543003B0F0BD00BF40E102089E
:100C7800037B022B01D000207047F0B5436983B095
:100C880013B11A689B8813850146006940F2E9335D
:100C9800828901E0002B5ED00289013B12F0020F2D
:100CA8009BB2F7D0BB23037340F2E93301E0002B7A
:100CB80051D00289013B12F0010F9BB2F7D0037BA0
:100CC8000869838903899C074FF005076E464FF42E
:100CD8007A724FF0FF0C4FF6FF7506D4531E9BB285
:100CE800D2B11A4603899C07F8D580F80CC04FF496
:100CF8007A7302E0A3B2AB420ED00289D20703F1A5
:100D0800FF34F7D5027BD2B20EB1327001367A1EAB
:100D180027B117461A46E5E7FFF763FA4B6913B19F
:100D28001A689B8893619DF800609DF801009DF802
:100D380002509DF803209DF804409DF8053040EAD4
:100D4800062042EA052243EA0423488301208A83D5
:100D5800CB8303B0F0BDFFF744FAB1E770B4D0E934
:100D68000041057B02690223AB4063600B684FF6C4
:100D7800FE7003400B60EFF31183502181F312885A
:100D8800D66B3168C9071CD4706870B9D2E90941BB
:100D98008C4213D095690D44F56017D81469611A0F
:100DA80071609062002182F85810326842F00102A6
:100DB800DBB2326083F3118870BC7047012182F87E
:100DC8005810DBB283F3118870BC7047611A7160E8
:100DD8009462E7E770B40468037B2268022101FA91
:100DE80003F31A4216D0026911481249642505FB1B
:100DF80002020D785068016875B91569528928682A
:100E08004FF6FE7630402860C868D24392B202405E
:100E1800CA60636070BC7047006902684FF6FE756F
:100E28002A400260CA684FF6FF600240CA60F0E7D5
:100E3800D44B0020D04B002030B50446406D2171C2
:100E48000368A26823F00103036087B06379009206
:100E580013F0040F4FEA03324FEA032314BF4FF491
:100E68008055002503F4806302F400520195CDE912
:100E78000223002511F0010305952ED104930823C0
:100E88008D07694648BF04931CF03AFA2079636DD0
:100E9800617900F00202002A15BF4FF440324FF486
:100EA80080324FF40034002410F0010F586808BF56
:100EB8002246CC074CBF024320EA02025A609A68D5
:100EC80009074CBF42F0080222F008029A601A682B
:100ED80042F001021A6007B030BD042304930C23CA
:100EE800CEE730B50446406DA160036823F00103E6
:100EF80003606379257987B013F0040F4FEA033252
:100F08004FEA032303F4806302F40052CDE902237D
:100F1800009114BF4FF480510021EB0748BF042310
:100F280001914FF00001CDE9041154BF0823049347
:100F3800694648BF0C23AD0748BF04931CF0E0F98D
:100F48002079636D617900F00202002A15BF4FF421
:100F580040324FF480324FF40034002410F0010F77
:100F6800586808BF2246CC074CBF024320EA020259
:100F78005A609A6809074CBF42F0080222F008023A
:100F88009A601A6842F001021A6007B030BD30B4A6
:100F980001220023102511244FF6FF71457044717A
:100FA80002720270027143818381C381018281745C
:100FB80030BC704710B50368017B1A6802238B4068
:100FC800134204460FD00F4A53680133202B536055
:100FD8000AD1182200210C482DF02BF8217B226819
:100FE80002238B40536010BD222BF7D1002353609E
:100FF800064A13704268136823F001031B041B0C94
:101008001360EBE7F80F00202C2200201D2200209F
:101018002DE9F04F87B00346029040689A6803882C
:1010280023F040031B041B0C038003889BB223F0AE
:10103800380343F038030380038843F040030380F8
:1010480012B1136892881A85838940F2E93302E065
:10105800002B00F082810289013B12F0020F9BB243
:10106800F6D06B23037340F2E93302E0002B00F063
:1010780074810289013B12F0010F9BB2F6D0037B09
:10108800029B586840F2E933828902E0002B00F0A5
:1010980061810289013B12F0020F9BB2F6D08023D6
:1010A800037340F2E93302E0002B00F05381028918
:1010B800013B12F0010F9BB2F6D0037B029B9B68A9
:1010C80013B11A689B8893610623A54CDFF89C82AC
:1010D800DFF89CA2A34DA44E04939623DFF894C294
:1010E80001934FF0100EDAF80430C3F30803002B15
:1010F80040F0B480EFF31183002B40F0AF802068FC
:10110800AA6823689842FAD133689A42F7D8D8F87F
:1011180000704FF47A7101FB07F39B1AB3FBF7F3E6
:1011280001FB00304FF47A774FF00109DAF8043008
:10113800C3F30803002B72D1EFF31183002B6ED198
:101148002368A96822689342FAD132689142F7D895
:10115800D8F8002007FB02FBABEB0101B1FBF2F171
:1011680007FB03131B1AB3F57A7FDFD3019B013BFF
:101178000193B8D1029B9B6813B11A689B881385A9
:10118800029B586840F2E933828902E0002B00F0A4
:1011980087800289013B12F0020F9BB2F6D0F5233B
:1011A800037340F2E93301E0002B79D00289013B57
:1011B80012F0010F9BB2F7D0037B029B586883891A
:1011C80040F2E93301E0002B67D00289013B12F0BD
:1011D800020F9BB2F7D0FF23037340F2E93301E01B
:1011E800002B5AD00289013B12F0010F9BB2F7D0B5
:1011F800037BDBB20393029B9A6812B11368918850
:101208009961039B682B4ED0049B013B13F0FF03AD
:1012180004937FF462AF184607B0BDE8F08FEFF390
:1012280011818EF31288D5F808B02B68DB0344BF10
:10123800CCF80090D5F808B02368DCF80020C9B2D3
:1012480081F31188D8F80010134407FB01F2A2EBD0
:101258000B02B2FBF1F207FB032383E7EFF31183E1
:101268008EF31288AF682A68D20303D50122CCF81E
:101278000020AF682068DCF80090DBB283F31188A7
:10128800D8F800104FF47A72484402FB01F3DB1BD4
:10129800B3FBF1F302FB003044E7FEF7A2FFAAE735
:1012A800FEF79FFF89E712B1136892881A85029B9F
:1012B800586840F2E933828901E0002B47D002895F
:1012C800013B12F0020F9BB2F7D08C23037340F25C
:1012D800E93301E0002B3AD00289013B12F0010FFB
:1012E8009BB2F7D0037B029B5868838940F2E933AD
:1012F8000289013B12F0020F9BB215D1002BF7D1E6
:10130800FEF76FFF029B9B6813B11A689B88936175
:10131800059B142B04D3182B17D9543B062B14D92F
:10132800002007B0BDE8F08FFF23037340F2E933D4
:1013380001E0002BE4D00289013B12F0010F9BB2BF
:10134800F7D0037BDBB20593DCE7032064E7FEF705
:1013580048FFC8E7FEF745FFB0E6FEF742FF8FE615
:10136800603D002010E000E0743D0020703D00204A
:1013780000ED00E06C3D002008B520212CF070FE47
:101388000346184623B10278202A03F10103F8D056
:1013980008BD38B52C2200212CF04BFE034640F244
:1013A800DC51642040F21A4240F26C7540F202248B
:1013B80018745982132040F275319A8240F643021C
:1013C800DD821C830E2502249876D9830A201921F0
:1013D8001A84012283F82B001973197783F8225095
:1013E80083F82A409A7383F8252083F82920194620
:1013F8000248BDE8384022F0C1B800BFF82C030805
:1014080038B5074C074DAC4203D3074B00221A707E
:1014180038BD6288D4E901012CF0E7FD1434F2E705
:10142800EC6B03084C700308F80F002038B5074C24
:10143800074DAC4203D3074B01221A7038BD6288AE
:10144800D4E901102CF0D1FD1434F2E7EC6B030859
:101458004C700308F80F0020B5EEC00ADFED317AB2
:10146800F1EE10FACCBF30EE270A30EE670ADFED56
:101478002E7A20EE270A30B5FDEEC07A87B017EE37
:10148800904A054684EAE470002303A9A0EBE470BF
:10149800CDE9003302932AF035FE002CACBF20239F
:1014A8002D2303A88DF800302BF0E4FE012803A9B2
:1014B80024D002282DD0032805BF3023684668466B
:1014C8008DF801302CF0BDFD68462BF0D3FE0338B3
:1014D800C4B22246694628462CF0E9FD00232B5564
:1014E80028462BF0C7FE2E22431C2A540DEB04017C
:1014F800E8182CF0C2FD284607B030BD30236846F6
:101508008DF801308DF802308DF803302CF099FDFC
:10151800DAE7302368468DF801308DF802302CF078
:1015280090FDD1E76F12033A00007A4410B500210C
:101538000446012009F0FCFC207010BDF8B5304EBF
:10154800304D32782B789A424FD12F4B93F800C008
:10155800BCF1000F48D02D4A2D4B1078002140F2E5
:101568000D3E11E05C681F896760276847F0010736
:101578002760A2F848E0D468013144F480748C45AF
:10158800D46003F59A730FDD1A680028EAD1506217
:10159800B3F83041D76801313C438C45D46003F53A
:1015A8009A7323F8040CEFDC31782B7899421BD01E
:1015B80003EB83029200174FB858BE18A0B9327ACD
:1015C80092B9727A82B9013303F00303D8B2814227
:1015D800287009D003EB83039C003B191A720AF0A8
:1015E80089F9736803443B51F8BD14F0DDF900280C
:1015F800FAD0054B93F800C0BCF1000FABD1D3E78C
:10160800F8130020F9130020F44E0020D04B0020DE
:10161800F84E0020FC130020002A12DD70B50446A5
:101628000D468E18236820469B6898470028F9D0F5
:10163800236815F8011B1B6820469847B542F1D16D
:1016480070BD70470368DB6A03B1184770470368C9
:101658009B6A03B11847704703682DE9F0415D6A3A
:101668001DB12B46BDE8F0411847002A174611DD89
:1016780004460E460F4400E023689B6820469847BE
:101688000028F9D0236816F8011B1B6820469847E4
:10169800BE42F1D1BDE8F08103685B691847036871
:1016A800DB68184703689B68184703685B68184736
:1016B80003681B681847014B1868F9E738130020BE
:1016C800036803F138422DE9F04F920AA74DAA5C4E
:1016D80002F01F0552090124022A04FA05F400F059
:1016E8009F81032A00F09781012A00F0518101F0BF
:1016F80003077A1E012AC1F3810EC1F300188488FA
:10170800C1F3411140F24981E60700F13181A50793
:1017180000F11A81600700F10581220700F1F080CD
:10172800E60600F1DB80A50600F1C680600600F140
:10173800B180220600F19C80E60500F18780A505AE
:1017480072D460055FD422054CD4E60439D4A504CC
:1017580026D4600413D4220401D4BDE8F08F1A689B
:1017680022F040421A601A6842EA87771F60DA68F6
:1017780022F0404242EA8171D960BDE8F08F1A68D0
:1017880022F040521A601A6842EA07721A60DA6850
:1017980022F0405242EA0172DA602204DDD5DEE727
:1017A8001A6822F040621A601A6842EA87621A6070
:1017B800DA6822F0406242EA81626004DA60CAD5DF
:1017C800DDE71A6822F040721A601A6842EA076276
:1017D8001A60DA6822F0407242EA0162A504DA600F
:1017E800B7D5DDE71A6822F440021A601A6842EA9F
:1017F80087521A60DA6822F4400242EA8152E6040B
:10180800DA60A4D5DDE71A6822F440121A601A6873
:1018180042EA07521A60DA6822F4401242EA015298
:10182800DA60220591D5DDE71A6822F440221A60B1
:101838001A6842EA87421A60DA6822F4402242EAC9
:1018480081426005DA607FF57EAFDCE71A6822F432
:1018580040321A601A6842EA07421A60DA6822F4CB
:10186800403242EA0142A505DA607FF56AAFDBE75C
:101878001A6822F440421A601A6842EA87321A60EB
:10188800DA6822F4404242EA8132E605DA607FF5FE
:1018980056AFDBE71A6822F440521A601A6842EA27
:1018A80007321A60DA6822F4405242EA0132DA60FA
:1018B80022067FF541AFDBE71A6822F440621A601E
:1018C8001A6842EA87221A60DA6822F4406242EA19
:1018D80081226006DA607FF52CAFDBE71A6822F414
:1018E80040721A601A6842EA07221A60DA6822F41B
:1018F800407242EA0122A506DA607FF517AFDBE7FE
:101908001A6822F0C0021A601A6842EA87121A603E
:10191800DA6822F0C00242EA8112E606DA607FF550
:1019280002AFDBE71A6822F030021A601A6842EA4E
:1019380007121A60DA6822F0300242EA0112DA600D
:1019480022077FF5EDAEDBE71A6822F00C021A6079
:101958001A6842EA87021A60DA6822F00C0242EA40
:1019680081026007DA607FF5D8AEDBE7881E0308DE
:101978001A6822F003021A601A683A431A60DA6891
:1019880022F003020A43A507DA607FF5C3AEDBE75E
:10199800264A55692C435461A9E600224FF0010CF0
:1019A8004FF003090CFA02F636EA04002ED1500073
:1019B800D3F808A009FA00F5ED430AEA050AC3F8C6
:1019C80008A0D3F808B00EFA00FA4AEA0B0AC3F8DE
:1019D80008A0B3F804A02AEA06069E80B3F804A07B
:1019E80008FA02F646EA0A06B6B29E801E682E403B
:1019F8001E60D3F800A007FA00F646EA0A061E6041
:101A0800DE6801FA00F035402843D8600132102A18
:101A1800C8D1BDE8F08F054AD5692C43D46166E684
:101A2800024A95692C43946161E600BF00100240A8
:101A380010B50409013C052C17D80E4B33F81420B7
:101A480000F00F0042FA00F313F001030FD0012356
:101A580003FA00F0013810402BF018FF064A074B34
:101A6800125D104403EBC00010BD002010BD1846E5
:101A780010BD00BFC01F0308F81E0308783D0020F2
:101A88002DE9F04F4A484B4B4B4C4FF090414FF0EB
:101A9800010A4FF002094FF004084FF0080E4FF00A
:101AA800100C20274026802530F8022B12F0010F59
:101AB80003D01960A3F804A0083312F0020F03D072
:101AC8001960A3F80490083312F0040F03D01960CA
:101AD800A3F80480083312F0080F03D01960A3F8A4
:101AE80004E0083312F0100F03D01960A3F804C003
:101AF800083312F0200F02D019609F80083312F0CB
:101B0800400F02D019609E80083312F0800F02D077
:101B180019609D80083312F4807F05D04FF4807BD4
:101B28001960A3F804B0083312F4007F05D04FF40D
:101B3800007B1960A3F804B0083312F4806F05D055
:101B48004FF4806B1960A3F804B0083312F4006FE7
:101B580005D04FF4006B1960A3F804B0083312F4F1
:101B6800805F05D04FF4805B1960A3F804B0083398
:101B780012F4005F05D04FF4005B1960A3F804B0BD
:101B8800083312F4804F05D04FF4804B1960A3F846
:101B980004B00833D20B04D04FF4004219609A8085
:101BA800083301F58061A1427FF47EAFBDE8F08F74
:101BB800C01F0308783D00200018004800B970478E
:101BC80003682DE9F04F03F138449C4EA40A01251F
:101BD800345D04F01F066409022C05FA06F500F0CE
:101BE8007481032C00F06C81012C00F02281808824
:101BF800B0FA80F4C4F11F04A4B2E50803EB85052C
:101C080004F007042E6AA4000F27A74026EA070657
:101C18002E622E6A01F00307A2407C1E3243012C7B
:101C2800C1F3810EC1F300182A62C1F3411140F2D9
:101C38000981C6070BD51A6822F003021A601A68D0
:101C48003A431A60DA6822F003020A43DA60850729
:101C58000DD51A6822F00C021A601A6842EA870247
:101C68001A60DA6822F00C0242EA8102DA6044075C
:101C78000DD51A6822F030021A601A6842EA071273
:101C88001A60DA6822F0300242EA0112DA600207CA
:101C98000DD51A6822F0C0021A601A6842EA871243
:101CA8001A60DA6822F0C00242EA8112DA60C606D7
:101CB8000DD51A6822F440721A601A6842EA07229F
:101CC8001A60DA6822F4407242EA0122DA60850674
:101CD8000DD51A6822F440621A601A6842EA87220F
:101CE8001A60DA6822F4406242EA8122DA60440625
:101CF8000DD51A6822F440521A601A6842EA07326F
:101D08001A60DA6822F4405242EA0132DA600206C6
:101D18000DD51A6822F440421A601A6842EA8732DE
:101D28001A60DA6822F4404242EA8132DA60C60573
:101D38000DD51A6822F440321A601A6842EA07423E
:101D48001A60DA6822F4403242EA0142DA60850514
:101D58000DD51A6822F440221A601A6842EA8742AE
:101D68001A60DA6822F4402242EA8142DA604405C5
:101D78000DD51A6822F440121A601A6842EA07520E
:101D88001A60DA6822F4401242EA0152DA60020567
:101D98000DD51A6822F440021A601A6842EA87527E
:101DA8001A60DA6822F4400242EA8152DA60C60414
:101DB8000DD51A6822F040721A601A6842EA076262
:101DC8001A60DA6822F0407242EA0162DA60850439
:101DD8000DD51A6822F040621A601A6842EA8762D2
:101DE8001A60DA6822F0406242EA8162DA604404EA
:101DF8000DD51A6822F040521A601A6842EA077232
:101E08001A60DA6822F0405242EA0172DA6002048B
:101E18000DD51A6822F040421A601A6842EA87779C
:101E28001F60DA6822F0404242EA8171D960BDE859
:101E3800F08F034C666935436561D8E6881E030850
:101E48000010024000224FF0010C4FF003090CFA79
:101E580002F636EA00042ED15400D3F808A009FA95
:101E680004F5ED4305EA0A0AC3F808A0D3F808B058
:101E78000EFA04FA4AEA0B0AC3F808A0B3F804A059
:101E88002AEA06069E80B3F804A008FA02F646EA93
:101E98000A06B6B29E801E682E401E60D3F800A0C7
:101EA80007FA04F646EA0A061E60DE6801FA04F438
:101EB80035402C43DC600132102AC8D1BDE8F08FD0
:101EC800044CE6693543E56191E6024CA669354361
:101ED800A5618CE60010024000B97047036803F161
:101EE80038422DE9F04F920AB24DAA5C02F01F0564
:101EF80052090124022A04FA05F400F05F81032A3A
:101F080000F05381012A00F00D8101F003077A1EC9
:101F1800012AC1F3810EC1F300188488C1F341116D
:101F280040F20581E6070BD51A6822F003021A6011
:101F38001A683A431A60DA6822F003020A43DA6040
:101F4800A5070DD51A6822F00C021A601A6842EA31
:101F580087021A60DA6822F00C0242EA8102DA602B
:101F680060070DD51A6822F030021A601A6842EA32
:101F780007121A60DA6822F0300242EA0112DA60C7
:101F880022070DD51A6822F0C0021A601A6842EAC0
:101F980087121A60DA6822F0C00242EA8112DA6017
:101FA800E6060DD51A6822F440721A601A6842EAE9
:101FB80007221A60DA6822F4407242EA0122DA60E3
:101FC800A5060DD51A6822F440621A601A6842EA1A
:101FD80087221A60DA6822F4406242EA8122DA60D3
:101FE80060060DD51A6822F440521A601A6842EA4F
:101FF80007321A60DA6822F4405242EA0132DA60A3
:1020080022060DD51A6822F440421A601A6842EA7C
:1020180087321A60DA6822F4404242EA8132DA6092
:10202800E6050DD51A6822F440321A601A6842EAA9
:1020380007421A60DA6822F4403242EA0142DA6062
:10204800A5050DD51A6822F440221A601A6842EADA
:1020580087421A60DA6822F4402242EA8142DA6052
:1020680060050DD51A6822F440121A601A6842EA0F
:1020780007521A60DA6822F4401242EA0152DA6022
:1020880022050DD51A6822F440021A601A6842EA3D
:1020980087521A60DA6822F4400242EA8152DA6012
:1020A800E6040DD51A6822F040721A601A6842EAEE
:1020B80007621A60DA6822F0407242EA0162DA6066
:1020C800A5040DD51A6822F040621A601A6842EA1F
:1020D80087621A60DA6822F0406242EA8162DA6056
:1020E80060040DD51A6822F040521A601A6842EA54
:1020F80007721A60DA6822F0405242EA0172DA6026
:1021080022040DD51A6822F040421A601A6842EA81
:1021180087771F60DA6822F0404242EA8171D9600D
:10212800BDE8F08F244A55692C435461EDE600223E
:102138004FF0010C4FF003090CFA02F636EA0400DE
:102148002ED15000D3F808A009FA00F5ED430AEAA9
:10215800050AC3F808A0D3F808B00EFA00FA4AEA4C
:102168000B0AC3F808A0B3F804A02AEA06069E8062
:10217800B3F804A008FA02F646EA0A06B6B29E8048
:102188001E682E401E60D3F800A007FA00F646EA43
:102198000A061E60DE6801FA00F035402843D86060
:1021A8000132102AC8D1BDE8F08F034AD5692C4303
:1021B800D461AAE6881E030800100240024A956905
:1021C8002C439461A1E600BF0010024030B10268C0
:1021D8008388918A0B4218BF1B0493617047024B96
:1021E80053F82000F2E700BF203F002010B1036839
:1021F80082881A85704710B1036882889A6170478F
:1022080018B1838811B10268936170471B04FAE71B
:1022180038B5074B03EBC0052C796A794C40A242CC
:1022280005D053F830002146FFF7EAFF6C7138BD3E
:10223800B043002010B501F0010428B1C94301F0F2
:1022480001010138FFF7E4FF14B9024B024ADA60D2
:1022580010BD00BF00ED00E00400FA0510B40A4B01
:102268000A4A1C7801238340234052F8200029B9E8
:10227800B3FA83F149095DF8044BC1E7191C18BF8B
:1022880001215DF8044BBBE71F3F0020203F0020E1
:1022980030B102688388128A1A4214BF01200020D4
:1022A800704708B5064B1868FFF7F2FF00B908BD7C
:1022B80009F020FB034B012298601A7308BD00BF88
:1022C800903F0020F80F00202DE9F0410B4E3468B4
:1022D80073691C400FD0DFF828800127B4FA84F313
:1022E800C3F11F0307FA03F558F82300036898475A
:1022F800AC437561F2D1BDE8F08100BF0004014034
:10230800D83E00202DE9F0410B4E346873691C401B
:102318000FD0DFF828800127B4FA84F3C3F11F0334
:1023280007FA03F558F8230003689847AC4375612A
:10233800F2D1BDE8F08100BF00040140D83E002082
:102348002DE9F0410B4E346873691C400FD0DFF85B
:1023580028800127B4FA84F3C3F11F0307FA03F5B1
:1023680058F8230003689847AC437561F2D1BDE87B
:10237800F08100BF00040140D83E00202DE9F04163
:102388000B4E346873691C400FD0DFF82880012792
:10239800B4FA84F3C3F11F0307FA03F558F82300CE
:1023A80003689847AC437561F2D1BDE8F08100BF7E
:1023B80000040140D83E00202DE9F0410B4E34685E
:1023C80073691C400FD0DFF828800127B4FA84F322
:1023D800C3F11F0307FA03F558F823000368984769
:1023E800AC437561F2D1BDE8F08100BF0004014043
:1023F800D83E00202DE9F0410B4E346873691C402B
:102408000FD0DFF828800127B4FA84F3C3F11F0343
:1024180007FA03F558F8230003689847AC43756139
:10242800F2D1BDE8F08100BF00040140D83E002091
:102438002DE9F0410B4E346873691C400FD0DFF86A
:1024480028800127B4FA84F3C3F11F0307FA03F5C0
:1024580058F8230003689847AC437561F2D1BDE88A
:10246800F08100BF00040140D83E0020A8B1838855
:10247800B3FA83F3C3F11F035A1C08D0012202FAEE
:1024880003F329B906490A6822EA03030B60704777
:10249800034A11680B43136070470123F1E700BF3B
:1024A80000040140084A094808B5936943F001034C
:1024B8009361002140222BF0BCFD054B4FF0FF3209
:1024C8001A60C3F8032008BD00100240D83E00205F
:1024D800183F002003681B6A184770B44E1C056833
:1024E800C2728672AC69A44670BC60472DE9F0419F
:1024F800044618460D4616461F462AF0BBFE2844D9
:10250800A0722068E672294645693B463246204655
:10251800AC46BDE8F0416047036810B504461B6847
:102528009847236820469B689847E37B0133E37309
:1025380010BD10B5036804469B689847FF23012225
:10254800A373627310BD70B5054600780E46FFF799
:102558006FFA044618B1382301368371C6712046D4
:102568006978FFF7B9FCAB78204613B1BDE8704035
:1025780041E6BDE8704039E64268138823F040031D
:10258800B1F5807F4FEA0343A8BF4FF480711B0C5D
:10259800138002291388B8BF022191FAA1F00029FB
:1025A800B0FA80F09BB208BF4FF0FF30013823F03B
:1025B800380343EAC0039BB21380138843F04003F7
:1025C80013807047038823F04003B1F5807F4FEAFA
:1025D8000343A8BF4FF480711B0C038002290388B2
:1025E800B8BF022191FAA1F20029B2FA82F29BB295
:1025F80008BF4FF0FF32013A23F0380343EAC20321
:102608009BB20380038843F040030380704738B5CA
:102618008368054613B11A689B881385686840F279
:10262800E933828901E0002B35D00289013B12F0A1
:10263800020F9BB2F7D0017340F2E93300E053B3C5
:102648000289013B12F0010F9BB2F8D0037B686846
:10265800838940F2E93300E0D3B10289013B12F0EB
:10266800020F9BB2F8D0FF23037340F2E93300E076
:1026780073B10289013B12F0010F9BB2F8D0047BC1
:10268800E4B2AB6813B11A689B889361204638BDE1
:10269800FDF7A7FDF5E7FDF7A4FDD8E7F8B55D213F
:1026A8001448FFF7B4FF1449144BCD890A8ADFF8A0
:1026B80054C04C196E1C277D2075D21B104400B2E3
:1026C80083FB0034C3179CF800500882C3EBE40373
:1026D800323306F00F029BB2032DCA818B8400D0DF
:1026E800F8BDA3EB8303DB00054A03F6E803138078
:1026F800F8BD00BF843F0020F80F0020ABAAAA2A2B
:10270800A42F00207C2F0020F8B584894FF6FF768F
:102718004FF47A742BB311B30F78013101E0B4424E
:1027280017D00589013CAD07A4B2F8D507734FF45B
:102738007A7402E0BCB2B4420BD00589ED0704F10B
:10274800FF37F7D5057BEDB20AB115700132013BB1
:10275800E0E7FDF746FD003018BF0120F8BDFF2770
:10276800DFE70120F8BD2DE9F04F90F8613085B022
:102778000746002B40F05384D7E90502038823F06D
:1027880040031B041B0C038003889BB223F038030F
:1027980043F038030380038843F04003038012B1F9
:1027A800136892881A85838940F2E93302E0002B86
:1027B80000F06D850289013B12F0020F9BB2F6D042
:1027C8006B23037340F2E93302E0002B00F05F85CE
:1027D8000289013B12F0010F9BB2F6D0037B7869A6
:1027E80040F2E933828902E0002B00F03C8602893E
:1027F800013B12F0020F9BB2F6D08023037340F224
:10280800E93302E0002B00F02E860289013B12F02A
:10281800010F9BB2F6D0037BBB6913B11A689B8882
:1028280093619623AA4CAB4EDFF8B092AA4DDFF81D
:10283800B0820093019709F05DF84FF0100C4FF447
:102848007A714FF0010ED9F80430C3F30803002B56
:1028580040F0C383EFF31183002B40F0BE8323685D
:10286800AF6822689342FAD1D8F800209742F6D888
:10287800D6F800A001FB0AF2D21BB2FBFAF201FB68
:1028880003231B1AB3F57A7FDDD3009B013B00932A
:10289800D1D1019FBB6913B11A689B8813857869E8
:1028A80040F2E933828902E0002B00F0D8850289E2
:1028B800013B12F0020F9BB2F6D06823037340F27B
:1028C800E93302E0002B00F0CA850289013B12F0CF
:1028D800010F9BB2F6D0037B786940F2E933828915
:1028E80002E0002B00F0B7850289013B12F0020FCD
:1028F8009BB2F6D00323037340F2E93302E0002BC6
:1029080000F0A9850289013B12F0010F9BB2F6D0B5
:10291800037BBB6913B11A689B8893619623DFF820
:10292800BC916D4DDFF8B8810093019708F0E2FF84
:102938004FF0100C4FF47A714FF0010ED9F80430B3
:10294800C3F30803002B40F02883EFF31183002B17
:1029580040F023832368AF6822689342FAD1D8F8FD
:1029680000209742F6D8D6F800A001FB0AF2D21B45
:10297800B2FBFAF201FB03231B1AB3F57A7FDDD30E
:10298800009B013B0093D1D1019FBB6913B11A6829
:102998009B881385786940F2E933828902E0002B2D
:1029A80000F055850289013B12F0020F9BB2F6D068
:1029B8006B23037340F2E93302E0002B00F04785F4
:1029C8000289013B12F0010F9BB2F6D0037B7869B4
:1029D80040F2E933828902E0002B00F03485028955
:1029E800013B12F0020F9BB2F6D00323037340F2AF
:1029F800E93302E0002B00F026850289013B12F042
:102A0800010F9BB2F6D0037BBB6913B11A689B8890
:102A1800936108F06FFF054608F06CFF401B0E2815
:102A2800FAD9BB6913B11A689B881385786940F293
:102A3800E933828902E0002B00F001850289013B1D
:102A480012F0020F9BB2F6D06A23037340F2E93307
:102A580002E0002B00F0F3840289013B12F0010F21
:102A68009BB2F6D0037B786940F2E933828902E0B1
:102A7800002B00F0E0840289013B12F0020F9BB2A8
:102A8800F6D01023037340F2E93302E0002B00F084
:102A9800D2840289013B12F0010F9BB2F6D0037B6E
:102AA800BB6913B11A689B88936108F023FF054638
:102AB80008F020FF401B0E28FAD9BB6913B11A6829
:102AC8009B881385786940F2E93382890DE000BF5D
:102AD800603D0020703D002010E000E000ED00E0C7
:102AE800743D0020002B00F0A2840289013B12F003
:102AF800020F9BB2F6D06C23037340F2E93302E075
:102B0800002B00F094840289013B12F0010F9BB264
:102B1800F6D0037B786940F2E933828902E0002B22
:102B280000F081840289013B12F0020F9BB2F6D0BB
:102B38000023037340F2E93302E0002B00F07384B2
:102B48000289013B12F0010F9BB2F6D0037BBB69EF
:102B580013B11A689B88936108F0CCFE054608F00B
:102B6800C9FE401B0E28FAD9BB6997F8601013B14B
:102B78001A689B881385786940F2E933828902E0F4
:102B8800002B00F04C840289013B12F0020F9BB22B
:102B9800F6D01923037340F2E93302E0002B00F06A
:102BA8003E840289013B12F0010F9BB2F6D0037BF1
:102BB800786940F2E933828902E0002B00F02B8427
:102BC8000289013B12F0020F9BB2F6D0017340F26A
:102BD800E93302E0002B00F01E840289013B12F069
:102BE800010F9BB2F6D0037BBB6913B11A689B88AF
:102BF800936108F07FFE054608F07CFE401B0E2816
:102C0800FAD9BB6913B11A689B881385786940F2B1
:102C1800E933828902E0002B00F0FA830289013B44
:102C280012F0020F9BB2F6D01B23037340F2E93374
:102C380002E0002B00F0EC830289013B12F0010F47
:102C48009BB2F6D0037B786940F2E933828902E0CF
:102C5800002B00F0DA830289013B12F0020F9BB2CD
:102C6800F6D01823037340F2E93302E0002B00F09A
:102C7800CC830289013B12F0010F9BB2F6D0037B93
:102C8800BB6913B11A689B88936108F033FE054647
:102C980008F030FE401B0E28FAD9BB6913B11A6838
:102CA8009B881385786940F2E933828902E0002B1A
:102CB80000F0A8830289013B12F0020F9BB2F6D004
:102CC8001C23037340F2E93302E0002B00F09A83DF
:102CD8000289013B12F0010F9BB2F6D0037B7869A1
:102CE80040F2E933828902E0002B00F088830289F0
:102CF800013B12F0020F9BB2F6D01823037340F287
:102D0800E93302E0002B00F07A830289013B12F0DC
:102D1800010F9BB2F6D0037BBB6913B11A689B887D
:102D2800936108F0E7FD054608F0E4FD401B0E2816
:102D3800FAD9BB6913B11A689B881385786940F280
:102D4800E933828902E0002B00F056830289013BB7
:102D580012F0020F9BB2F6D03723037340F2E93327
:102D680002E0002B00F048830289013B12F0010FBA
:102D78009BB2F6D0037B786940F2E933828902E09E
:102D8800002B00F036830289013B12F0020F9BB240
:102D9800F6D01023037340F2E93302E0002B00F071
:102DA80028830289013B12F0010F9BB2F6D0037B06
:102DB800BB6913B11A689B88936108F09BFD0546AF
:102DC80008F098FD401B0E28FAD9BB6913B11A68A0
:102DD8009B881385786940F2E933828902E0002BE9
:102DE80000F004830289013B12F0020F9BB2F6D077
:102DF8003823037340F2E93302E0002B00F0F68237
:102E08000289013B12F0010F9BB2F6D0037B78696F
:102E180040F2E933828902E0002B00F0E482028963
:102E2800013B12F0020F9BB2F6D00123037340F26C
:102E3800E93302E0002B00F0D6820289013B12F050
:102E4800010F9BB2F6D0037BBB6913B11A689B884C
:102E5800936108F04FFD054608F04CFD401B0E2815
:102E6800FAD97A69138823F040031B041B0C1380DA
:102E7800138823F038031B041B0C1380138843F0BA
:102E88004003138008F036FD054608F033FD8542FF
:102E9800FBD07869038823F040031B041B0C0380D4
:102EA80003889BB223F0380343F038030380038878
:102EB80043F04003038097F85B30032B00F2AD80AA
:102EC80097F85E10A1F10101B1FA81F14909BB69D6
:102ED80013B11A689B881385838940F2E93302E0AD
:102EE800002B00F07D820289013B12F0020F9BB299
:102EF800F6D01A23037340F2E93302E0002B00F006
:102F08006F820289013B12F0010F9BB2F6D0037B5E
:102F1800786940F2E933828902E0002B00F05D8293
:102F28000289013B12F0020F9BB2F6D0017340F206
:102F3800E93302E0002B00F050820289013B12F0D5
:102F4800010F9BB2F6D0037BBB6913B11A689B884B
:102F5800936108F0CFFC054608F0CCFC8542FBD015
:102F68007869038823F040031B041B0C0380038843
:102F780023F038031B041B0C0380038843F0400331
:102F880003803B7C022B00F03F81B7F952305BB2E3
:102F980001337FD005B0BDE8F08FEFF311828CF3D9
:102FA8001288D5F808A02B68DF0304D5BB4BC3F8FB
:102FB80000E0D5F808A0B94F2368D7F800B0D2B21E
:102FC80082F3118837685B4401FB07F2A2EB0A021F
:102FD800B2FBF7F201FB0323CEE4EFF311828CF38B
:102FE8001288D5F808A02B68DB0304D5AB4BC3F8CF
:102FF80000E0D5F808A0A94F2368D7F800B0D2B2EE
:1030080082F3118837685B4401FB07F2A2EB0A02DE
:10301800B2FBF7F201FB032333E4002157E71D0954
:10302800013D052D03F00F0300F10C0600F2CC81E1
:103038009B4A32F8150040FA03F2D10740F1C481E7
:10304800012202FA03F3013B18402AF01FFC954BBA
:10305800954C5B5D184414EBC00400F0B581002268
:10306800924BE2712021A1712046FB60314625F088
:10307800E3FEA388B3FA83F3C3F11F035A1C3FF49A
:103088007BAB8B490122086802FA03F303430B6008
:10309800FFF772BB97F9503001337FF47BAF0A23F7
:1030A800DFF81CA2834D844F019326F003F94FF4F7
:1030B800FA73DFF8E8E100934FF01008DAF804300B
:1030C800C3F30803002B40F03D81EFF31183002B7D
:1030D80040F038812068AA6823689842FAD13B6892
:1030E8009A42F7D8D6F800C04FF47A7101FB0CF376
:1030F8009B1AB3FBFCF301FB00304FF47A7C4FF0D2
:103108000109DAF80430C3F30803002B40F0FC800F
:10311800EFF31183002B40F0F7802368A968226839
:103128009342FAD13A689142F7D832680CFB02FB15
:10313800ABEB0101B1FBF2F10CFB03131B1AB3F566
:103148007A7FDED3009B013B0093B7D1072025F09F
:103158001DFF4FF47A73DFF844E100934FF0100835
:10316800DAF80430C3F30803002B40F00C81EFF3C6
:103178001183002B40F007812068AA6823689842D1
:10318800FAD13B689A42F7D8D6F800C04FF47A7162
:1031980001FB0CF39B1AB3FBFCF301FB00304FF46B
:1031A8007A7C4FF00109DAF80430C3F30803002BE6
:1031B80040F08C80EFF31183002B40F08780236868
:1031C800A96822689342FAD13A689142F7D83268DE
:1031D8000CFB02FBABEB0101B1FBF2F10CFB03139F
:1031E8001B1AB3F57A7FDED3009B013B0093B7D15E
:1031F800019B013B01937FF458AF3049304B314874
:10320800314A0860DA60C5E6BB6913B11A689B8861
:103218001385838940F2E93301E0002B3BD0028912
:10322800013B12F0020F9BB2F7D0C323037340F2A5
:10323800E93300E07BB30289013B12F0010F9BB236
:10324800F8D0037B7869062302AA0021FFF75CFA0D
:10325800BB6913B11A689B8893619DF808209DF893
:1032680009109DF80A509DF80B309DF80C0041EAB2
:1032780002219DF80D20A7F8501043EA05231BB240
:1032880042EA0022A7F85230A7F854207FE6FCF75C
:10329800A8FFFFF7A4BAFCF7A4FFD3E76C3D002012
:1032A800C01F0308F81E0308783D0020B90B00086A
:1032B8000004014010E000E0743D0020FC9F002065
:1032C80000ED00E0EFBEADDE0400FA05EFF311817A
:1032D80088F31288D5F808B02B68DB0344BFCEF812
:1032E8000090D5F808B02368DEF80020C9B281F351
:1032F8001188316813440CFB01F2A2EB0B02B2FBFC
:10330800F1F20CFB03236BE7EFF3118188F31288CA
:10331800D5F808B02B68DB0344BFCEF80090D5F889
:1033280008B02368DEF80020C9B281F3118831683B
:1033380013440CFB01F2A2EB0B02B2FBF1F20CFB03
:103348000323FBE6EFF3118388F31288D5F808C04E
:103358002A68D20304D50122CEF80020D5F808C087
:103368002068DEF80090DBB283F3118831684FF4EF
:103378007A72484402FB01F3A3EB0C03B3FBF1F3AD
:1033880002FB0030B9E6EFF3118388F31288D5F811
:1033980008C02A68D20304D50122CEF80020D5F847
:1033A80008C02068DEF80090DBB283F3118831682A
:1033B8004FF47A72484402FB01F3A3EB0C03B3FB0E
:1033C800F1F302FB0030EAE6294BFB6000223146AC
:1033D800104625F031FD002353E6FCF702FFB3E564
:1033E800FCF7FFFE94E5FCF7FCFE2DE5FCF7F9FE83
:1033F8000DE5FCF7F6FEDBE4FCF7F3FEBBE4FCF7B7
:10340800F0FE89E4FCF7EDFE69E4FCF7EAFE37E438
:10341800FCF7E7FE17E4FCF7E4FEFFF7E5BBFCF773
:10342800E0FEFFF7C5BBFCF7DCFEFFF790BBFCF73F
:10343800D8FEFFF76FBBFCF7D4FEFFF731BBFCF7F4
:10344800D0FEFFF710BBFCF7CCFEFFF7DDBAFCF7A8
:10345800C8FEFFF7BCBAFCF7C4FEFFF75ABAFCF780
:10346800C0FEFFF739BAFCF7BCFEFFF7D5B900BFBD
:10347800B90B0008F8B50546806816461F4610B116
:10348800036882881A85686840F2E934838901E014
:10349800002C43D00289013C12F0020FA4B2F7D0ED
:1034A800017340F2E93101E0002937D0028901397E
:1034B80012F0010F89B2F7D0037B686807F1FF3C6F
:1034C800838907B34FF47A734FF6FF7126B33478C4
:1034D800013601E08B421CD00289013B97079BB261
:1034E800F8D504734FF47A7302E0A3B28B4210D07C
:1034F8000289D20703F1FF34F7D50CF1FF3CBCF188
:10350800FF3F027BE2D1AB6813B11A689B889361D5
:10351800F8BDFCF766FEF6E7FF24DDE7FCF761FE81
:10352800CBE738B583680446154613B11A689B88FB
:103538001385606840F2E933828901E0002B30D0BE
:103548000289013B12F0020F9BB2F7D0017340F2DF
:10355800E93300E02BB30289013B12F0010F9BB263
:10356800F8D0037B606840F2E933828900E0DBB180
:103578000189013B11F0020F9BB2F8D0057340F2AC
:10358800E93300E083B10289013B12F0010F9BB2DD
:10359800F8D0037BA36813B11A689B889361012054
:1035A80038BDFCF71EFEDDE7FCF71BFEF2E7427AAA
:1035B8004AB110B5044604F10A01D0E90030984731
:1035C8000023637210BD7047A8B10D4B012210B4DF
:1035D80002FA01F103F1750402E00333A3420BD0B0
:1035E80013F8012C8242F8D11A780A42F5D001204A
:1035F8005DF8044B7047704700205DF8044B704736
:1036080049E1020830B40A4D002305F1680401E0DD
:10361800272B0AD003EB43020133A15C8142F7D187
:103628002A4430BC92F86A007047002030BC7047CA
:10363800E0E00208024B01461868FCF78BBE00BFA9
:103648002C12002038B5064D441E14F8011F2868B6
:1036580011B9BDE83840AAE7FCF77CFEF5E700BFE2
:103668002C12002010B504460B48FFF7EBFF0B4B5C
:103678001868FFF79CFF0A4B186808F0B1FA22F0A7
:10368800F9F9084B084A24B1084909480860DA6082
:1036980010BDDA60FCE700BF902303082C1200205D
:1036A8003012002000ED00E00400FA05FC9F002025
:1036B800EFBEADDE38B5094D2868FFF778FF084B37
:1036C80000241C70074B1C60074B1C7022F060FB29
:1036D8002046FFF7C7FF2C6038BD00BF2C12002022
:1036E80038120020341200204D2700200120B9E7AD
:1036F800064B1B780A3B012B01D90548A2E7054B6D
:103708000548012283F826209CE700BFB434002036
:103718009C230308F80F0020AB230308004891E717
:103728006328030838B5064D002455F834000134E1
:10373800FFF788FFFFF7F2FF262CF6D138BD00BF50
:103748005CFE020808B5FFF77DFFBDE80840E5E725
:10375800024A136823EA000010607047904A00206C
:103768002DE9F341056906460F467DBBD0F8008078
:10377800C8F30A0323B30023D6F80080019326F088
:10378800DFF8042819D1224C236943F0010323618F
:10379800BBB2A8F8003026F0D3F804282ED108F1DF
:1037A80002030193019B3F0C1F8026F0C9F823698F
:1037B800042823F00103236125D06FF0010505E0FB
:1037C80026F0BEF8042805D04FF0FF35284602B091
:1037D800BDE8F0810E4C236943F002032361C4F86D
:1037E8001480236943F04003236126F0A9F8236974
:1037F800042823F002032361BDD0E5E7236923F001
:1038080001032361D9E7336804333360DEE700BF7F
:1038180000200240F8B504460D468E180027B54230
:1038280001D12069F8BDE368591CE160234415F80B
:10383800012B1A720429F2D1A1682046FFF790FFE4
:10384800C4E90370EBE730B402681146531C036007
:1038580011F8024B0160D31C517803609378151D51
:1038680005601B0443EA0123D078234343EA006040
:1038780030BC70470368591C1A46016012F8021BD5
:103888000260587841EA0020704703685A1C0260B9
:103898001878704738B50446006815462AF0A5FB25
:1038A80022682A44226038BD03685A1C026010B49A
:1038B800197003680A0A5C1C04601A7003680A0C11
:1038C8005C1C04601A700368090E5A1C02601970A7
:1038D8005DF8044B704703685A1C0260197003684E
:1038E800090A5A1C02601970704707EE901AF8EE20
:1038F800677A9FED847A27EE800A20EE070AFDEEAC
:10390800C07A17EE903A2033402B00F28180DFED29
:103918007E7AB4EEE70AF1EE10FA40F3E680B0EEF4
:10392800407A9FED7A6ADFED7A6A01E0B0EE677A55
:10393800B4EEE67AF1EE10FA77EE467AF6DC9FED11
:10394800757AF4EEC77AF1EE10FA40F1D1809FED66
:103958006F6ADFED716A01E0F0EE477AF4EEE67A1D
:10396800F1EE10FA37EE867AF6D4DFED6C7AB4EE23
:10397800E77AF1EE10FA40F3A780DFED637A37EECD
:10398800C77A27EE076ADFED665ADFED667ADFED64
:10399800666A9FED665AE6EE257A67EE065AE6EE07
:1039A800276AF7EE007AA5EEA67AF0EE675AE7EEF8
:1039B800055AE7EE457A87EEA55ADFED587A30EEDC
:1039C800277AFDEEC76A16EE903A2033402B24D9A9
:1039D8009FED577AF6EE006AB7EE006AF7EE004AF6
:1039E800C4EEA57A0023836143610362C36180ED5D
:1039F800045A67EEA66A27EE866A27EE877AC0ED34
:103A0800006AC0ED026A80ED016A80ED037A7047B2
:103A1800B7EE005AF0EE455ACFE7B4EEE70AF1EEFA
:103A280010FA6BDD9FED396ADFED396A01E0B0EE1F
:103A3800677AB4EEE67AF1EE10FA77EE467AF6DCBB
:103A48009FED347AF4EEC77AF1EE10FA53D59FED74
:103A58002F6ADFED316A01E0F0EE477AF4EEE67A9C
:103A6800F1EE10FA37EE867AF6D4DFED2C7AB4EE62
:103A7800E77AF1EE10FA33DCDFED2E7AB4EEE77A6E
:103A8800F1EE10FA44BFDFED237A37EEC77A27EE5E
:103A9800076ADFED234ADFED236ADFED237AE6EEDE
:103AA800246A67EE064AE6EE267AB7EE006AA4EEC6
:103AB800A77AF6EE006A36EE476AF8EE007A27EE45
:103AC800277A66EE266A89E7DFED1A7AB4EEE77A96
:103AD800F1EE10FA44BFDFED0F7A37EEC77A50E700
:103AE800DFED097A37EEC77AD1E7F0EE407A26E7BC
:103AF800B0EE677A39E7B0EE677AB6E7F0EE477A64
:103B08009EE700BF27D4D236DB0F4940DB0FC94000
:103B1800E4CB1641DB0F49C0E4CB16C1DB0FC93F2C
:103B280092E741B99730083C15A82ABEF304353FFF
:103B380000000000DB0FC9BFDFED2E7AB4EEE70A04
:103B4800F1EE10FA4ADDDFED2C6A9FED2C7A01E0E8
:103B5800B0EE670AB4EEC70AF1EE10FA70EE667AB4
:103B6800F6DC9FED277AF4EEC77AF1EE10FA3ED52F
:103B7800DFED216A9FED237A01E0F0EE407AF4EE62
:103B8800C77AF1EE10FA37EEA60AF6D4DFED1E7A00
:103B9800B4EEE70AF1EE10FA14DDDFED167A37EE2F
:103BA800C00A60EE006A9FED196A9FED197ADFED91
:103BB800197AA6EE867A20EE266AE6EE877AA6EECF
:103BC800270A7047DFED147AB4EEE70AF1EE10FA2F
:103BD80044BFDFED0B7A37EEC00AE2E79FED087AC3
:103BE800F0EE407AF4EEC77AF1EE10FAC0D4B0EEF7
:103BF800670ACBE7DB0F4940DB0FC940E4CB16412E
:103C0800DB0F49C0E4CB16C1DB0FC93F92E741B9CE
:103C18009730083C15A82ABEDB0FC9BF02B370B4A1
:103C28008E1803E0121B14D1B14215D010F8012BE5
:103C3800A2F14103192B11F8013BA3F1410598BFEB
:103C48002032192D03F12004ECD9D21A01D1002B0E
:103C5800EAD1104670BC70470022104670BC70470D
:103C68001046704770B5044608460D4629F002FB19
:103C7800064602E014F8013F43B132462946204681
:103C8800FFF7CCFF0028F5D1204670BD1C46204622
:103C980070BD4FF0FF32FFF7C1BFA0F16103192BD0
:103CA80098BF20387047A0F14103192B98BF2030E6
:103CB8007047202805D0093804288CBF002001202F
:103CC80070470120704770B5044608460E4629F033
:103CD800D1FA3146054602462046FFF79FFF68B9EC
:103CE800635D1846FFF7E5FF00B933B901352C4489
:103CF800204601340378202BFAD070BD0020FCE761
:103D0800613819288CBF00200120704741381928D4
:103D18008CBF002001207047303809288CBF002054
:103D280001207047A0F13003092B07D920F02000AB
:103D3800413819288CBF00200120704701207047A6
:103D4800012129F0EDB970B50D461446FDF714FBB5
:103D58000646A0B1FFF7F4FF40F634039842A8BF27
:103D68001846B0F5617FB8BF4FF461701923A0F50C
:103D7800617090FBF3F0287023780133237030468C
:103D8800FDF7FAFA0646A0B1FFF7DAFF40F634036A
:103D98009842A8BF1846B0F5617FB8BF4FF461706C
:103DA8001923A0F5617090FBF3F068702378013354
:103DB8002370304670BDF8B5064615460846B6FB72
:103DC800F2F434B905FB14640B4B1B5D00F8013B9E
:103DD800F8BDB4FBF2F75FB905FB1747064B05FBC7
:103DE8001464DA5D00F8012B1B5D00F8013BF8BD97
:103DF8003846FFF7E0FFEFE7042D03080F4B2DE9E6
:103E08003048D3E9004554EA05020AD1034640F296
:103E1800011200201880988098715A801881BDE896
:103E28003088074B1A6814EB020B45F1000C5A4610
:103E38006346FCF7E3FC0120BDE83088001200204F
:103E4800603D00200A44914215D010B40139541E37
:103E580011F8012F0823504010F0800F4FEA40005E
:103E680018BF80F0D500013BC0B2F5D1A142EFD117
:103E78005DF8044B704770474840082310F0800FE6
:103E88004FEA400018BF80F0D500013BC0B2F5D121
:103E980070470A44914215D030B40139551E41F299
:103EA800210211F8014F082380EA042004044CBFC2
:103EB80082EA40004000013B80B2F7D18D42F0D148
:103EC80030BC7047704770B502221349134C144E2A
:103ED8004FF6FF70FFF7DDFF22884AB1A518B542FB
:103EE80018D2052A16D92146FFF7D3FF2C46F3E747
:103EF80021460222FFF7CDFF0222A118FFF7C9FFD2
:103F0800084BE41A084B1C8541F60F53C31A584254
:103F1800584170BD0020FCE700F0030802F00308D8
:103F280000000408FAEF0308F80F00202DE9F04319
:103F3800002489B006460D461F46A04605E02529FF
:103F48000CD030460134A847039A531C03931178C8
:103F58000029F4D1204609B0BDE8F083931CCDE9CF
:103F680003385078302842D0A0F13003DBB2092B57
:103F78004FF0000945D96C282AD0642873D019D984
:103F8800732858D063D9752840F0828007F1040C53
:103F9800386805AB00220A216746FCF7E3FB05AB4E
:103FA800049A009329464B463046FCF7E4FC039AF2
:103FB8000444CAE725283CD051D958286BD0632837
:103FC800C2D139783046A84704370134039ABCE790
:103FD800039B5A1C03921B78642B52D016D8252BAE
:103FE80027D064D9582B18D0632BEAD0ADE7D31C5F
:103FF80003939078A0F13003DBB2092B4FF001094D
:10400800B9D804AA03A926F07FFAB4E7732B12D013
:1040180051D9752B2DD0782B97D1A3F15802B2FA2C
:1040280082F23868520905AB10210437FCF79AFB75
:10403800B5E7252185E73B68049A009329460023C4
:104048003046FCF798FC04370444039A7DE76E2851
:104058007FF47AAF039A3B6804371C6075E7002841
:104068003FF478AF70E7386805A9FCF745FB0437DB
:1040780095E7386805AB00220A21FCF773FB043783
:104088008DE73B1D386805A91F46FCF735FB86E719
:1040980078287FF459AFA0F15802B2FA82F2386852
:1040A800520905AB1021FCF75DFB043777E7002BBD
:1040B8003FF450AF49E76E2BCDD046E710B5064C1C
:1040C8000B46024605492068FFF730FF2068BDE827
:1040D8001040FFF76CBA00BF2C120020BB04000888
:1040E80038B504460D460848FFF7ACFA294620467D
:1040F800FFF7E4FF0548FFF7A5FA054B1B7813B156
:10410800044B01221A7038BDB6230308C1230308E3
:1041180088130020891300200FB407B504A951F8AB
:10412800040B0191FFF7DCFFFFF7F8FA03B05DF825
:1041380004EB04B0704738B50F4D2B7863B10F4CC2
:1041480023784BB10E48FFF7E7FF0E48FFF7E4FF6F
:1041580000232B70237038BD0B4B93F82A203AB1FB
:10416800D86A07F016FA0020BDE83840FFF77ABA97
:1041780007F032F9F7E700BF881300208913002001
:10418800C5230308FC230308F80F002038B50522CF
:1041980015490446FFF742FD58B9144A13781BB96C
:1041A80001211170124A13701248BDE83840FFF718
:1041B800C9BA032210492046FFF730FD80B90B4CDD
:1041C8000B4D227842B12B7833B10C48FFF7A4FF8E
:1041D800002323702B7038BD0948FFF7B3FAF7E7BF
:1041E8000848BDE8384097E75D2C0308881300208D
:1041F800891300201A240308B62C0308C5230308D2
:104208003024030844240308004885E7532403089E
:104218000FB407B504A951F8040B0191FFF760FF2B
:1042280003B05DF804EB04B070470FB407B504A9F8
:1042380051F8040B0191FFF741FFFFF76FFA03B044
:104248005DF804EB04B0704710B5104C03461846EF
:10425800FCF795F858B10E4B0E4893F901104B1C1A
:104268000ABF0D4BC9B25978BDE81040DDE71846C2
:10427800FFF766FD052804D8C0B211F0EFFD23460C
:10428800E5E705210548BDE8104045E7652803082E
:10429800000000205F240308245C00206E2403082B
:1042A80010B5104C03461846FCF769F858B10E4B88
:1042B8000E4893F900104B1C0ABF0D4BC9B2197870
:1042C800BDE81040B1E71846FFF73AFD022804D8C8
:1042D800C0B207F0FEFD2346E5E702210548BDE828
:1042E800104019E76528030800000020632403082C
:1042F800245C0020732403082DE9F3410346FCF7EE
:104308003EF8044620B1FFF77FFF02B0BDE8F08118
:1043180001AA2B49DFF8A880184629F0C1FD2746D5
:10432800054626467DB9022CEDD1A7F57A73B3F57B
:104338007A7F1FD94FF4FA634FF47A7221492248E1
:10434800FFF7EAFEE1E74CB1012C0ED001AA414685
:10435800002029F0A5FD01340546E3E7284627F0AB
:10436800DBFF431C0646F1D1CFE72846FFF7E8FC00
:104378000746EBE7B8B221F009FBFF2EBCEEC00AF6
:10438800124B0BD1124AF8EE407A1278AA4212DC8C
:1043980010EE101A0F48FFF748FFB6E7F8EE407A1C
:1043A80003EB860310EE102A31460B48C3ED007A62
:1043B800FFF73BFFA9E7E3EC017A0135E6E700BF29
:1043C80011270308F02C03088E240308F83700206F
:1043D80020590020B4240308A72403082DE9F34733
:1043E8000346FBF7CCFF044618B92B4A9278042AF7
:1043F80004D8FFF709FF02B0BDE8F08701AA2749F2
:10440800DFF8AC80DFF8AC90DFF8ACA0184629F0F4
:1044180047FD0127264640B9214B224A1B689B1AB3
:10442800214A18BF01231370E5E75EB927F074FF2E
:10443800431C0446DFD001AA18490020013629F0A0
:104448002FFDE8E7FFF77CFC2F2805461ED8D7B1DB
:1044580011F002FB062D06D1052007F01DFB504682
:10446800FFF770F909E0012007F016FB0F49012357
:10447800EAB20978E0B210F055FE29464846FFF73F
:10448800D4FE0027D7E70628F0D1E8E72F214046D9
:10449800FFF742FECFE700BFA84B00201127030813
:1044A800C44B002089F700089858002020590020A4
:1044B800D4240308C32403089C23030813B5304CF1
:1044C800237C022B55D1A36913B11A689B881385E5
:1044D800F5216069FBF7A0FE01230DF10702002119
:1044E8006069FEF711F9A36913B11A689B88936193
:1044F8009DF807102348FFF798FE237C022B3AD13A
:10450800A36913B11A689B8813859A216069FBF720
:1045180083FE01230DF1070200216069FEF7F4F81C
:10452800A36913B11A689B8893619DF80710164810
:10453800FFF77BFE237C022B1FD1A36913B11A68F6
:104548009B8813859B216069FBF766FE01230DF1AB
:10455800070200216069FEF7D7F8A36913B11A684A
:104568009B8893619DF807100848FFF75EFE02B02C
:1045780010BD0021BEE70021D9E70021F4E700BF04
:1045880008440020F4240308072503081A25030813
:104598002DE9FF41074628F06DFE08283CD100228E
:1045A80001AEB85CFFF779FBB0540132082AF8D1A4
:1045B8000024DFF870808DF80C40385DFFF76DFB44
:1045C800C5B230552946404629F04AFD28B1013484
:1045D8002946301929F044FD20B1FFF715FE04B033
:1045E800BDE8F081082CE8D10D4930461EF0C6FF21
:1045F8000B4C0C4800231A5D04A90A44195C02F804
:104608000C1C0133082BF6D1002301A906488DF8AC
:104618000C30FFF70AFEE2E70028E9D0DDE700BF2B
:10462800E4590020A01D03082D250308034B044A64
:1046380004491B68126809680348F6E5B4F7FF1FC8
:10464800B0F7FF1FACF7FF1F34250308F7B5064680
:10465800FBF795FE054658B1002401A9204627F02E
:1046680051FD0134FFF7F2FF122CF6D103B0F0BD73
:104678003046FFF765FBC4B2112C61D8701CFCF7FB
:104688007BFE334D0746D0B9324B13F814108A1EFF
:10469800514251412F4B13F81420154495F8DD2051
:1046A800002948D003EB440319205B7840F2EE213F
:1046B80000FB031321462848FFF7B7FDD6E705F1AD
:1046C800DD060178304629F0CBFC58B1032C8CBFAD
:1046D80003230023801B2B4453FA80F090F8E160F9
:1046E800032E02D1FFF790FDC0E73846FCF744FEE1
:1046F800F0B1022EF6D1FFF723FB40F6CA0280B2D2
:104708009042144BA8BF104640F2EE22904203EBB1
:104718004403B8BF1046A0F2EE20192290FBF2F035
:104728005870B31E594259410A4B03F81460B1E757
:10473800022EF6D1D6E721460848FFF776FD95E721
:1047480011232A4606490748FFF7E6FC8EE700BF13
:10475800E0E00208843A00204825030858250308A9
:10476800652503088E2403080FB407B504A951F87A
:10477800040B0191FFF7A2FC03B05DF804EB04B051
:1047880070472DE9F843044628F074FD024680B3CB
:1047980020461949FFF742FA044650BBFEF7BEFF10
:1047A8001648174D174E184FDFF86480FEF7CAFFFA
:1047B8002B7D072194FBF1F1C1EBC10206EB8303CA
:1047C800A21A013201313846D3F8E890FFF7CCFF3E
:1047D8006A7D49464AB10D48FFF727FD01340C2C84
:1047E80005F11C05E4D1BDE8F8834046FFF71DFD3F
:1047F800F4E7BDE8F84307E56D25030872250308CB
:1048080004000020E0E00208772503088925030852
:10481800CE27030838B50B4B03EBC0040D4694F8BC
:10482800DC21094803EB8203D3F8E810FFF79CFF6B
:1048380094F8E23123B1691C0448BDE8384093E795
:1048480038BD00BFE0E00208CF270308312903087C
:1048580070B5374C3748FEF7F5FE94F82530012B34
:1048680060D13548354EFEF76DFF94F82A3013B104
:1048780094F8273013B194F8263043B9B6F8985015
:104888002F48FEF7DFFE8DBB2E48FEF75BFF2E4854
:104898002E4DFEF7D7FE94F8293005EB8303D3F8A5
:1048A8008C02FFF7C2FCB6F894102948FFF75CFFAA
:1048B80094F826302BBB2748FEF744FF2648FEF71E
:1048C800C1FE94F82A3005EB8305D5F89402FFF76A
:1048D800ACFCB6F896102148FFF746FF94F82A304A
:1048E8009BB91F48BDE87040FEF72CBF4FF47A72A1
:1048F800B5FBF2F102FB115292B21A48FFF795FC90
:10490800C5E71948FEF71EFFD8E794F8273023B902
:104918001648BDE87040FEF715BF1548BDE8704061
:10492800FEF710BF1348BDE87040FEF70BBF00BF8D
:10493800E459002090250308A62503083C590020C7
:10494800AD250308C8250308DA250308E0E00208B6
:10495800F02503080D2603081D260308382603083A
:104968005B260308D2250308142603080E2603082D
:1049780015260308602603087FB50B4B04930B4BE1
:1049880003930B4B02930B4B01930B4B00930B4A76
:104998000B4B0C490C48FFF7E7FE0C48022107B007
:1049A8005DF804EB41E400BFB1260308B62603080E
:1049B800BE260308C7260308D32603086E26030865
:1049C8002B5C00207B26030886260308D9260308CB
:1049D8002DE9F04F93B00025DFF8A4B1DFF8C0A1AE
:1049E800DFF8C0910795A84608A9E8B213F0BAFD08
:1049F8009DF82830002B6DD0022D40F09A809DED57
:104A0800117AB5EE407AF1EE10FA00F08980DFED08
:104A1800586AC6EE877AFDEEE77AF8EEE77AFDEE99
:104A2800E77A17EE906A99F80040089B012C79D92B
:104A380096FBF4F41A4602214E48FFF795FE0D9AAC
:104A4800002A00F08B8041F2883002FB04004FF40A
:104A58007A73B0FBF3F00F9B002B00F0818041F2DA
:104A6800883103FB04114FF47A7CB1FBFCF1062D6D
:104A780003D0079F0F44804407979BF803C0BCF1FD
:104A8800000F6FD04FF47A7C0E9FB7FBFCFCCDF87B
:104A980010C04FF00A0C91FBFCFE0CFB1E11CDE977
:104AA80002E190FBFCF10CFB1100CDE9001021465E
:104AB8003148FFF7BAFB022D08D199F80030012BD5
:104AC80004D9324609992D48FFF7AFFB0AEB851345
:104AD80000229A630135142D86D1294BDB78E3B186
:104AE800284B29481968294B1A684FF47A73B1FB87
:104AF800F3F3274952090968FFF797FB0798079BC3
:104B08000A2293FBF2F302FB130798FBF2F10097DA
:104B180002FB11821F48FFF788FB13B0BDE8F08F36
:104B2800002680E7099A1C480221FFF71DFE34463B
:104B380085E7109C5CB107EE904ADFED0D6AF8EE50
:104B4800677A86EEA77AFDEEC77A17EE904A089A3A
:104B580008482946FFF708FE002670E710467AE75E
:104B6800194684E721460D48FFF75FFBA3E700BF1E
:104B780000247449F126030813270308372703087C
:104B8800245C00201C180020472703081418002064
:104B98002018002067270308002703084327030875
:104BA80094010020983000202DE9F047214FDFF8CC
:104BB800A480DFF88490DFF8A0A00546284628F0F6
:104BC80059FB064658B91C4B1C481A781C4B03EB7A
:104BD8008203BDE8F047D3F89C12FFF726BB0246D4
:104BE80039462846FFF71AF878B91648164C174D73
:104BF800FEF728FD54F8041F19B12846FFF7B4FD45
:104C0800F8E7BDE8F047FEF789BD002458F82410FE
:104C180021B90F48BDE8F047FFF77EBA324628466B
:104C2800FEF7FCFF01340028F0D189F80040554612
:104C3800C4E700BF9F270308043A0020952703080C
:104C4800E0E00208A42703087CE30208CE27030853
:104C5800AF27030880E30208652803082DE9F84F09
:104C680080460E46174628F005FB0446F0B9404832
:104C7800404FDFF82081FFF777FD0C25204604F030
:104C880069FD3368184205D005FB047340469968EE
:104C9800FFF76AFD0134182CF0D1336813B9364890
:104CA800FEF7D0FCBDE8F84FFEF738BD02463349A1
:104CB8004046FEF7B3FF0546B0B931482D4EDFF840
:104CC800C880FEF7BFFC2C460C25204604F042FDA8
:104CD800384205D005FB046340469968FFF744FD58
:104CE8000134192CF1D1DDE798F800302D2B03BFE2
:104CF80008F1010804F1FF34012500254FF0000AEE
:104D080047F0807B1B4B0C2202FB0A324046D2F84C
:104D1800089022464946FEF781FFF8B9504604F04C
:104D280019FD1BEA000F19D075B1BAF1180F1CBF95
:104D38003768074337601348FEF784FC4946124832
:104D4800BDE8F84FFFF771BABAF1180F1CBF356804
:104D5800854335600D48FEF775FCEFE70AF1010A57
:104D6800BAF1190FCED10A48BDE8F84FFFF7D4B908
:104D7800BC270308F0FC0208C62703089F2703087E
:104D8800A4270308D2270308CE270308DB27030834
:104D9800AF270308CD2703086FF07F4200495DE77E
:104DA800681A002040F20222004957E7701A0020D2
:104DB8002DE9F047424D074628F05CFA414B95F83B
:104DC8002A801E680446B8F1000F15D0D5F82C903B
:104DD800C4B93D483D4D3E4FFEF734FC012655F819
:104DE800241059B106FA04F313EA090F02D0384621
:104DF800FFF7BAFC0134F2E7B146E9E7BDE8F0474E
:104E0800FEF78CBC224633493846FEF707FF78B9CF
:104E18003148324C324DFEF715FC54F8041F002976
:104E2800ECD00B78002BF8D02846FFF79DFCF4E770
:104E3800B8F1000F03D10123EE6285F82A303B78E0
:104E4800DFF888A02D2B03BF013704F1FF344FF0A2
:104E580001094FF000094FF000085AF8286026B9F8
:104E68002048BDE8F047FFF757B922463146384693
:104E7800FEF7D4FE08BB012303FA08F2110604D595
:104E88001948BDE8F047FEF75DBC9305F8D4EB6A16
:104E9800B9F1000F0BD023EA02031448EB62FEF7C6
:104EA800D1FB31460E48BDE8F047FFF7BEB91343C2
:104EB8000F48EB62FEF7C6FBF3E708F10108CCE701
:104EC800F80F0020904A0020E3270308ECE30208CB
:104ED800ED2703089F270308A4270308E8E302082F
:104EE800CE270308AF270308F1270308D2270308B2
:104EF800DB2703082DE9F04F85B00346FBF73FFA9F
:104F0800064620B1FFF780F905B0BDE8F08F03AA87
:104F18008149DFF84CB2184628F0C2FFB0468246F5
:104F28003446B14635464FF0FF37BAF1000F26D167
:104F38007A483946FFF718FC794B93F9062078B27E
:104F4800824200F0C68093F90E20824200F0C080B1
:104F5800002D14BFA8464FF46148002C08BF032455
:104F68000022E4B2019200944346114625F038F835
:104F7800074600283CD16B48FEF7E4FBC4E7B8F1CC
:104F8800030F07D8DFE808F0020F14245046FEF795
:104F9800D7FE074603AA6049002028F081FF08F1E0
:104FA80001088246C1E75046FEF7CAFE0546F1E70A
:104FB8005D495046FEF756FE08B144F001045946D3
:104FC8005046FEF74FFE0028E4D044F00204E1E723
:104FD800504628F04FF9554902465046FEF71EFE46
:104FE80020B15046FEF7ACFE8146D3E70126D1E753
:104FF800414675B94E48FFF7B7FB4E48FEF7A2FB8E
:105008004D4B186803681B6A33B13A464B499847B9
:1050180002E04B48FFF7A8FB4A4B4B494B48464C2C
:10502800002E18BF1946FFF700F916B9B9F1000F9D
:1050380006D020680368DB6913B14A46444998479B
:105048002468204606F0CCFD384606F0C9FD00214C
:105058000846FDF703F900210120FDF7FFF8204677
:10506800FCF723FBA0B101210020FDF7F7F820464B
:10507800FCF715FB05463846FCF714FB0028FAD068
:1050880029463846FCF714FB00210846FDF7E6F8E8
:105098003846FCF70AFB0028E1D001210020FDF783
:1050A800DDF83846FCF7FBFA05462046FCF7FAFA25
:1050B8000028FAD029462046FCF7FAFA00210846CB
:1050C800FDF7CCF8CBE7B9682248FFF74DFB0EE0B7
:1050D80008331F68002F3FF43BAF002DF3D029465B
:1050E8001D48FFF741FB29463846FBF770F85CB1CD
:1050F8003979A14208D019482246FFF735FB3B68A9
:10510800E1B29B6938469847FB6A0BB10023FB6202
:10511800002D81D171E700BF112703081628030865
:10512800984000201F2803080A28030810280308AD
:1051380034280308C228030830120020D7010008C9
:1051480051280308FD27030865280308E5280308F4
:105158003D2200088928030866280308A4280308B4
:105168000D2803082DE9F041037903F06002202A95
:105178002CD002D852B1BDE8F081402A4AD0602A2A
:10518800F9D12748BDE8F041FFF74FB803F007030E
:10519800022B02D0042B09D07BB9B0F80720B0F855
:1051A80005102048BDE8F041FFF73FB8D0F80510DA
:1051B8001D48BDE8F041FFF738B8B0F90720B0F94D
:1051C80005101848BDE8F041FFF72FB84679174D8C
:1051D800174805EBC605FEF735FA95F88C730024D9
:1051E8000123A74203D8BDE8F041FEF797BAD5F8E6
:1051F800886356F824204FEA84084AB113B90D4849
:10520800FEF720FA56F808100B48FFF7ADFA00230E
:105218000134E6E741790948BDE8F041FFF705B8F0
:105228005A2903081E29030808290308E0E0020890
:105238003529030846290308CF2703084929030805
:105248002DE9F0411746027902F06003402B05462C
:105258000C462BD10026554FDFF8708115E02B79CD
:1052680003F00703022B15D0032B19D0012B14BF11
:10527800A15DA1573846FFF777FA6B79013BB34236
:1052880002DD4046FEF7DEF901366B79B342E6DC13
:10529800BDE8F08134F816103846FFF765FAECE7F8
:1052A80034F916103846FFF75FFAE6E702F007020E
:1052B800042A6DD8DFE802F0031F282A2D0024787D
:1052C800202B3ED0602B4CD0002BE1D1B5F80560E7
:1052D800B5F8078035482146FFF746FAA6424EDC66
:1052E800A0454CDB002FD3D0424631463048BDE8BC
:1052F800F041FFF739BA94F90040202B21D0602BF8
:105308002FD0002BC4D14BE02488D9E7B4F9004052
:10531800F3E72668202B344613D0602B21D0002BCE
:10532800B6D131462348FFF71FFAD5F805108E424B
:1053380025D8002FACD02048BDE8F041FFF714BABB
:1053480000246A791D4B03EBC20393F88C23A24215
:1053580015DDD3F8883353F82400BDE8F041FEF793
:1053680071B96A791441E30704D51548BDE8F041DD
:10537800FFF7FAB91348BDE8F041FFF7F5B9FEF7B2
:10538800CDF9224629681048BDE8F041FEF740BF34
:10539800202BD5D0602BEDD0002B7FF479AF1C46A5
:1053A800B5F90560B5F9078094E700BF322903080D
:1053B8007A2903081B29030874290308E0E0020876
:1053C8006F2903088129030885290308722903081E
:1053D80038B50D460446FBF75BFB2A4601462046D6
:1053E800BDE838402CE72DE9F74FDFF8C4B0814617
:1053F8008A460025D8462B4B0D2418686C43FEF7C7
:10540800D6F804EB0B031B7903F018034B4504D0C3
:10541800B9F1000F3ED1182B3CD10D2303FB0582B7
:105428000093B2F80900FBF71CFB444407462046EA
:10543800FAF7ADFFD7E901210646024401442046A8
:10544800FAF7DEFF1AF0100F0246009B00D008BBE7
:1054580003FB05831AF0200F1B680FD072B9194699
:10546800114800930192FFF77FF97968019A314456
:105478002046FFF7E5FEFEF751F9009B0B48194659
:10548800FFF772F9B968002231442046FFF7D8FEC9
:10549800FEF744F90135B5F5B87FACD103B0BDE8E6
:1054A800F08F00BF2C1200209F290308A0290308B1
:1054B80024EA0208052838B50D460CD8064C607059
:1054C8000648FEF7C1FEFEF729F929461020FFF726
:1054D8008AFFFF23637038BD000000206528030899
:1054E800022838B50D460CD8064C20700648FEF741
:1054F800D7FEFEF713F929460820FFF774FFFF23AC
:10550800237038BD00000020652803080CB407B5D7
:1055180010F020000BD079B92320FEF78BF805A9ED
:1055280004980191FEF7CAFDFEF7F8F8012003B0D0
:105538005DF804EB02B070470020F8E70CB4C3062E
:1055480007B500D561B905A904980191FEF7B6FD24
:10555800FEF7E4F8012003B05DF804EB02B07047F1
:105568000020F8E72DE9F04F354C87B08046354AE2
:105578002378608802EB8303D3F8E890FBF771FA8D
:10558800D0E901A30493304B1B7813B9CDF810A0D0
:105598009A4608F04003DFF8BCB005930026A379CB
:1055A800002B08BF01239E4206DB284B08349C428F
:1055B800DDD107B0BDE8F08F6279237906FB0323BC
:1055C800049A0136D55CBAF1000F11D1B5FA85F706
:1055D8007F090DB305F00F032D0940350293CDE97E
:1055E80000654B465A4639464046FFF7A7FFD6E7BF
:1055F8001AF80330EA1A57425741C3B103F00F02B1
:105608001B0940330292CDE900635A464B4639469E
:105618004046FFF77BFFDCE7059B002BBFD10096D8
:105628004B460B4A39464046FFF788FFB7E70096D6
:105638004B46074A39464046FFF768FFC9E700BFAF
:10564800BCE20208E0E00208F80F00206CE3020860
:10565800C0290308AA2903082DE9F04F87B005AA35
:105668008C4928F01DFC064628B94120FFF77AFF2F
:1056780007B0BDE8F08F8849DFF86082FEF709FBC4
:1056880088BB8648864C874E874FFEF75BF804F543
:105698009875A3792168A28808EB830301F1384142
:1056A800B2FA82F2890A4131D3F8E830C2F11F0216
:1056B8003046FFF759F8E17911B13846FFF754F849
:1056C8000834FEF72BF8A542E3D1724905AA002059
:1056D80028F0E6FB7549FEF7DCFA0028C8D16E48C9
:1056E800FFF74FF8C4E708F5EE770024B94617F836
:1056F800343008EB8303E500D3F8E8A0504627F0E0
:10570800B9FD514602463046FEF788FA38B10134F1
:10571800162CECD131466648FEF7FEFCA8E705AA30
:105728005C4928F0BDFBA8440746FEF709FB98F83A
:10573800E2310646002B40F09880002800F39F8055
:10574800A944B9F80200FBF78CF93D78002D00F068
:105758008980F3B2019399F8046099F80530019AA9
:10576800D0F804805349384602FB0636FEF791FA12
:1057780060B908F8060018F80680B8F1000F16D1CD
:105788004D48FDF7DFFF73E7012372E0602D8CBF02
:10579800613D413D072D65D8781CFEF7D1FA0F28E9
:1057A80060D8013540EA051508F80650E3E7404699
:1057B800FCF73EF98146002854D04FEA18134033CD
:1057C80002933E4F08F00F030026039300252EE0B6
:1057D8007888FBF746F97A793B7905FB0323426819
:1057E800D15C414522D1B44204D101998D421DD0EA
:1057F8000021D154DDE9021231485FFA85FB5FFAD6
:1058080086FAFEF7B1FF59465046FFF703F8B4424F
:1058180009D12C48FEF7A8FF50465946FEF7FAFF73
:105828002948FEF7A1FF2948FDF78CFF0135BB7910
:10583800002B08BF01239D42CADB0136162E07F153
:105848000807C3D1D9F80010B9F80420204801F19D
:105858003841B2FA82F2890AC2F11F024131FEF7D9
:10586800E4FC05E7FEF7D0FC02E7002801DD9E42D4
:1058780007DD012217491848FEF74EFCF8E6012813
:1058880082D105AA0349002028F00AFB013E0746F9
:1058980056E700BF112703086D250308D42903081C
:1058A800783D0020D729030831290308E229030895
:1058B800E6290308CF290308082A0308BCE20208DE
:1058C8000E2A0308322A0308352A03083D5903081B
:1058D8003F2A0308022A03088E240308E0E002088E
:1058E8002DE9F04F4A4085B098461D4FD3430646F0
:1058F8000D4600240393204603F02CFF0E9B18420C
:1059080028D0039B174ADFF860A0034214BF4FF06A
:1059180001094FF0000910EA050302934FF00C0348
:1059280003FB04234946D3F808B0CDF800B014BFF0
:105938003A46524643463046FFF7E8FD029ACDF80C
:1059480000B04346002A14BF52463A4649463046FC
:10595800FFF7F4FD0134182CCDD105B0BDE8F08F68
:10596800972A0308F0FC02084B2A030870B506467C
:1059780027F080FC114C054690B1112200212046E9
:1059880028F057FB2A460E49304628F07EFB38B1EE
:10599800102D2A46314628BF1022204628F087FBC2
:1059A8002378064A002B08BF0121054B1CBF0021A4
:1059B80013460120034ABDE87040BFE5902B002044
:1059C800D65903085A2A030870B5054627F052FC31
:1059D800044690B1112200210F4828F02AFB2246E4
:1059E8000E49284628F051FB38B1102C224629468A
:1059F80028BF1022084828F05AFB094B13F8112F2A
:105A0800002A064A06BF012113460021054A012043
:105A1800BDE8704092E500BFA12B0020D6590308CD
:105A2800902B0020522A03082DE9F04F002489B05A
:105A3800834692460D4626464FF019094FF4617881
:105A4800BAF1000F22D004EB84030AEB0307052206
:105A580039462846079328F0B9FA3A79079B19FB83
:105A680002820492FA781AF8033019FB0282039230
:105A7800BA780292B0FA80F67A78019276090093A1
:105A8800104A234631465846FFF740FD2B790D4A08
:105A980019FB03830493EB7819FB03830393AB7817
:105AA80002936B78019315F8053B00933146234622
:105AB80058460134FFF742FD0A2CC1D109B0BDE8B0
:105AC800F08F00BF622A03082DE9F0478AB08246AA
:105AD800FAF755FC064638B1002247490120FFF77E
:105AE800A3FF0AB0BDE8F0875046FEF729F9092858
:105AF80004467ADC850005EB00080AF101008DF800
:105B08001F60FBF739FC3C4F824608EB07093E460D
:105B180050B1FEF715F90D2806D89DF81F3008F882
:105B2800070001338DF81F305046FBF725FC8246ED
:105B380058B1FEF705F9052807D82B1933445870D2
:105B48009DF81F3001338DF81F305046FBF714FCC9
:105B5800824658B1FEF7F4F8082807D82B193344C1
:105B680098709DF81F3001338DF81F3008F103013C
:105B78000DF11F0231445046FEF7E5F89DF81F204D
:105B8800052A2AD1002308A9484608938DF824300D
:105B980028F01CFA2B19334493F801C020B1BCF14A
:105BA800000F1AD09B78C3B1254472194FF4617065
:105BB8001179192313FB01010491D17813FB010317
:105BC800039393780D4ACDE901C30021735D0093D7
:105BD80008462346FFF7B2FC83E7002348F807305E
:105BE80089F80430FEF710FB7BE7092332460449A5
:105BF8000448FEF791FA74E784170020622A030824
:105C0800022A03088E2403082DE9F74FDFF864A061
:105C180081468B4617460E46002447B307EB840897
:105C280004224146304628F0D1F9B8F802300193F1
:105C3800B0FA80F537F8243000936D0923465246B0
:105C480029464846FFF762FC738801933BF82430E5
:105C5800009352462346294648460134FFF76EFC16
:105C6800042C06F10406D8D103B0BDE8F08F3D46F8
:105C7800EAE700BF782A0308F7B50546FAF77FFB7D
:105C8800064630B12A490022012003B0BDE8F040A1
:105C9800BAE728492846FDF7FCFF38B9244B264ABD
:105CA800C3E90022C3E9022203B0F0BD2846FEF78B
:105CB80047F80328044632D82846FBF75DFB074619
:105CC80060B1FEF73DF8012605463846FBF754FB60
:105CD80040B903B0BDE8F040FEF796BA40F2EE25B1
:105CE8000646F2E7FEF72CF8002EF2D0A5F2EE22D7
:105CF80040F2DC539A42ECD8A0F2EE229A42E8D85D
:105D08000B4B0E4A23F8245003EB840300215880E0
:105D1800CDE9005023460846FFF710FCC4E70849C0
:105D280008480323324603B0BDE8F040FEF7F4B953
:105D3800503A002010280308E803D007782A0308FF
:105D4800652503088E2403082DE9F04F2DED088BF7
:105D5800DFF80C9193B0804692460D461446002613
:105D680095ED008AB5EE408AF1EE10FA70D0D5EDC7
:105D7800019A95ED029AD5ED038ABAF1000F3ED04B
:105D880094ED000A94ED01BAD4ED02AA94ED03AAA9
:105D9800B4EE408AF1EE10FA5FD1F4EE4B9AF1EED0
:105DA80010FA5AD1B4EE6A9AF1EE10FA55D1F4EE1F
:105DB8004A8AF1EE10FA0CBF012700270FA8FBF75B
:105DC8004BFBB0EE4B0A83460CA8FBF745FBB0EE45
:105DD8006A0A059009A8FBF73FFBB0EE4A0A04904F
:105DE80006A8FBF739FB059B049A03900292CDE9BC
:105DF80000B34A46334639464046FFF787FBB0EEC4
:105E0800480A0FA8FBF728FBB0EE690A07460CA85A
:105E1800FBF722FBB0EE490A834609A8FBF71CFBF7
:105E2800B0EE680A049006A8FBF716FB049B0390E3
:105E3800CDE901B3009733464A4600214046013672
:105E4800FFF77CFB082E05F1100504F1100487D13B
:105E580013B0BDEC088BBDE8F08F0027AEE700BF9C
:105E6800892A03082DE9F0474B4FDFF84881DFF80E
:105E7800489104462046FAF782FA064628B10022DD
:105E880046490120BDE8F0475EE70522394620462D
:105E9800FDF7C4FE58B9414B00221A601A611A6214
:105EA8001A631A641A651A661A67BDE8F08704222D
:105EB80041462046FDF7B2FE0546204615BBFBF7D6
:105EC8005BFA06460028F0D027F0D4F92C465FFA92
:105ED80080FA59F8245025B93148BDE8F047FEF753
:105EE8001BB9524629463046FDF798FE40B9204670
:105EF80026F0EAF929462B482B4CFEF796F9B9E724
:105F08000134E6E7FDF71CFF072805463BD8204685
:105F1800FBF732FA064648B3FAF724FB1F4B03EBAC
:105F2800051383ED000A01243046FBF725FA0646DF
:105F380038B1FAF717FB194B03EB051383ED010A88
:105F480001343046FBF718FA064638B1FAF70AFB6F
:105F5800124B03EB051383ED020A01343046FBF7BD
:105F68000BFA28B9BDE8F047FEF74EB90446DBE75F
:105F7800FAF7F8FA094B032C03EB051585ED030A2C
:105F88003FF47DAFEEE73246072308490848BDE8ED
:105F9800F047FEF7C1B800BF10280308A05800203A
:105FA800AF270308A22A030865280308022A030862
:105FB8008E2403089D2A030880E302082DE9F04F88
:105FC800834689B092460D46144600264FF01909BB
:105FD8004FF46178BAF1000F45D00A2221462846CD
:105FE80027F0F4FF23890793E38806932379059321
:105FF800E3780493A3781D4A19FB0383039363781A
:1060080019FB0383029323780193B0FA80F763792D
:1060180000937F09334639465846FFF777FA2B89AC
:106028000793EB8806932B790593EB780493AB7869
:106038000E4A19FB038303936B7819FB03830293BE
:106048002B7801936B7900933946334658460136CD
:10605800FFF774FA1E2E05F10A0504F10A04B9D1F6
:1060680009B0BDE8F08F5746D9E700BFAC2A03084E
:10607800F0B58BB00746FAF782F9044630B1002232
:106088005B490120FFF79AFF0BB0F0BD3846FDF7DA
:1060980057FE1D28054600F3A3800A264643781CB0
:1060A8008DF82740FBF768F9514C074650B1FDF7CA
:1060B80047FE032806D8A31958719DF827300133E5
:1060C8008DF827303846FBF757F9074658B1FDF7E2
:1060D80037FE0D2807D80A236B43E0549DF8273074
:1060E80001338DF82730711C0DF127022144384601
:1060F800FDF729FEFBF740F9074660B1FDF720FEE2
:10610800222808D80A2303FB0543D8709DF82730B6
:1061180001338DF827303846FBF72EF9074660B172
:10612800FDF70EFE0D2808D80A2303FB0543187156
:106138009DF8273001338DF827309DF82730062B3E
:1061480007D0A2190023A35153601381FEF75CF80E
:106158009AE70A2606FB054600233846F380338172
:10616800FBF70AF9074638B1FDF7EAFD9DF8273035
:10617800F08001338DF827303846FBF7FDF850B131
:10618800FDF7DEFD0A2303FB054318819DF8273040
:1061980001338DF82730174B4FF0FF321A600A226F
:1061A8006A43A3184FF4617619890791D988069133
:1061B80019790591D97804919878192111FB006013
:1061C8000390587811FB00610291A25C01925B79FF
:1061D800009300212B46084A0846FFF7AFF953E71A
:1061E8001D23224605490648FDF796FF4CE700BFE8
:1061F800A415002090010020AC2A0308022A0308F5
:106208008E2403082DE9F04F89B002F11003DFF85E
:10621800BCA02D4EDFF8B8B00793814690460D46D6
:10622800144695F902309AF906209A4203D09AF951
:106238000E209A423CD1B8F1000F42D008222146E4
:10624800284627F0C3FE627994F9023056F82220D6
:106258000492A27956F822200392227956F8222035
:106268000292E27856F822200192B0FA80F722884A
:1062780000927F095A4639464846FFF747F96A7936
:1062880095F9023056F822200492AA7956F822206D
:1062980003922A7956F822200292EA7856F82220A8
:1062A80001922A88009239465A464846FFF746F92D
:1062B800079B0834A34205F10805B2D109B0BDE82F
:1062C800F08F4746DBE700BFB81D03089840002061
:1062D800D02A03082DE9F04188B00346FAF74FF8B1
:1062E800044630B146490022012008B0BDE8F0411B
:1062F80088E7CDE9060018465E1C414DFDF720FDF4
:1063080095F9023040B2834276D095F90A3083423B
:1063180071D025463046FBF72FF8074628B1FDF720
:106328000FFD0134ADF81800E4B2DFF8D88000267C
:106338003846FBF721F8074600B3FDF701FD0022B8
:1063480058F822108842D3B203D00132102AF7D16C
:10635800002358F82320904210D1022E1AD0032E81
:106368001DD05A1E012ED2B20FD00B2A03D88DF899
:106378001B300134E4B20136042ED9D1052C14D8CF
:1063880008B0BDE8F041FDF73FBF042AF3D88DF807
:106398001C30EEE7052BEED88DF81E30E9E79A1E83
:1063A8000D2AE8D88DF81D30E3E706AB03CB154A74
:1063B80069609DF81D10286052F8211004919DF81D
:1063C8001E109DF91A3052F8211003919DF81C10E7
:1063D80052F8211002919DF81B1052F821200192C9
:1063E8000021BDF8182000920846074AFFF7A6F8D2
:1063F80008B0BDE8F08108358DF81A00012489E756
:1064080022590020B81D0308D02A03082DE9F04FAF
:10641800DFF8DCA087B0814690460D46144600267A
:10642800B8F1000F61D006222146284627F0CEFD9C
:10643800B0FA80F7207812F0B9FA834660797F09BC
:1064480012F0B4FABBF1000F1DD09BF80810A27827
:1064580094F803B094F801C04FF4617E192313FB3C
:1064680002E213FB0BE394F804E000B1007ACDE9F3
:106478000223CDE904E0CDE9001C334652463946F3
:106488004846FFF743F8287812F090FA834668796F
:1064980012F08CFABBF1000F1DD09BF80810AA78F7
:1064A80095F803B095F801C04FF4617E192313FBEA
:1064B80002E213FB0BE395F804E000B1007ACDE9A2
:1064C8000223CDE904E0CDE9001C334652463946A3
:1064D8004846FFF733F80136142E05F1060504F196
:1064E80006049DD107B0BDE8F08F4746CBE700BF53
:1064F800ED2A03082DE9F04186B00746F9F73FFF7A
:10650800044638B1002253490120FFF77FFF06B047
:10651800BDE8F0813846FDF713FC1328054600F363
:10652800918006264643781C8DF81740FAF724FF19
:10653800484C074660B1FDF703FCC0B212F01AFAE6
:1065480030B10378A3559DF8173001338DF8173013
:106558003846FAF711FF074660B1FDF7F1FB0D2841
:1065680008D8062303FB054358709DF817300133FC
:106578008DF81730B11C0DF1170221443846FDF78C
:10658800E2FBFAF7F9FE074660B1FDF7D9FB0128EF
:1065980008D8062303FB054318719DF8173001330B
:1065A8008DF817303846FAF7E7FE78B1FDF7C8FBE3
:1065B800C0B212F0DFF948B1062303FB05430278A5
:1065C8005A719DF8173001338DF817309DF8172050
:1065D800042A4FF0060327D103FB054300221A7152
:1065E8005A7120F06FFF06236B43E618E05C12F047
:1065F800DDF9F278B778192380464FF46174707921
:1066080013FB074713FB024412F0D0F9017A7378A1
:1066180098F80820039131790F480097CDE9014196
:106628002946FDF702FE72E7052A04D103FB05435C
:1066380000225A71D5E7062AD3D0A2190023A35104
:106648009380CEE71323224604490548FDF764FDED
:106658005DE700BF3C340020ED2A0308022A030846
:106668008E2403080EB400B584B005AB019053F82E
:10667800042B0649039301A8FDF758FC019B00224F
:106688001A7004B05DF804EB03B070477509000890
:106698002DE9F04F1E468DB007460B889246002A1A
:1066A8005ED115461446B3F5FA6F39D391F80280D6
:1066B80008F1FF320B2A33D891F803C00CF1FF32EE
:1066C8001E2A2DD891F804E0BEF1170F28D891F8AA
:1066D8000590B9F13B0F23D888793B2820D80A893F
:1066E800B2F57A7F1CD21A4643464FF001085EBBCA
:1066F80009890491002CB4BF2D212B21002CB8BF8F
:106708006442CDE90290CDE905140795CDE900CEA4
:1067180038464449FFF7A6FF40460DB0BDE8F08F64
:1067280000234149ADF828304FF0010C18468DF888
:106738002A30ADF82C3099469E461A46984609915B
:10674800634609A9002ED3D0CDE90290CDE900CE49
:1067580038463649FFF786FF40460DB0BDE8F08F52
:10676800A3F5FA638D7891F80380DFF8CC9091F85F
:1067780004E02F4C487991F806C003F0030202EBBD
:106788004202013D05EB82059A0839F81590294D1A
:1067980008F1FF3340F2B55808FB02334B4403EBD2
:1067A80043030EEBC30384FB0A24C3EB03134FEA32
:1067B800EA7200EB830354446544C2EB6414C3EBF0
:1067C800031305EB8303B1F80880C4EB04154FF4F9
:1067D8007A7BAAEB85054FF00009CBFB03892DB224
:1067E800002D4FF47A724FF0000340464946B8BF77
:1067F8006D4226F0FBFF3C230AFB030A4FF47A7232
:1068080000234046494626F0F1FF002392B2CBFB15
:106818000A2309A8F9F7F2FF24B209A9BDF8243020
:1068280041E700BF4C2D0308000001012C2D03088F
:106838008988888880436D38E0E00208F0B54822EE
:1068480091B04C494C48FDF78FFFFCF767FF4B4A66
:106858004B494C48FDF788FFFCF760FF4A4B4B4A11
:106868004B48D21A4B4B198DFDF7DFFC4A4B4B486E
:1068780019684FF47A73B1FBF3F1FDF775FF05A8BA
:10688800FDF7BCFA58B1464A05A90023B2F9002021
:1068980008A8FFF7FDFE08A94248FDF765FFFCF7C9
:1068A8003DFF4149D1F89C20002A53D007EE902A99
:1068B800DFED3E6AB8EEE77AC6EE877AFDEEE77A54
:1068C800CDED037A3A4B1B885BB107EE903ADFEDCA
:1068D800376AF8EE677A86EEA77AFDEEC77A17EE82
:1068E800903AC96959B107EE901ADFED306AF8EEAF
:1068F800E77A86EEA77AFDEEC77A17EE901A2D484A
:106908002D4E00882D4F6428CDE900310146039BA8
:106918002B48A8BF6421FDF788FC2A4B2A491A781E
:106928002A4B09882A4803EB82032A4AD3F8D83429
:106938001278FDF77AFC00212748FDF776FC2748F6
:10694800FCF780FE264B1C6801252CB9FCF7E6FEF7
:1069580011B0F0BD0392B5E794FAA4F3B3FA83F348
:1069680005FA03F256F82310384624EA0204FDF724
:10697800FBFEEAE7062B03080B2B03080020001098
:10698800000800001E2B030800F00308000004089C
:10699800422B0308F80F0020603D00206C2B0308F1
:1069A8005C2A0020862B03089401002000247449E7
:1069B8008614002098130020C0070308CE27030878
:1069C800992B03087E25002078250020E0E00208A6
:1069D800DF2B03087F250020062C0308152C03084D
:1069E800B029002010B44C09012250F8243001F0DD
:1069F8001F0102FA01F123EA010340F824305DF88F
:106A0800044B704710B44C09012250F8243001F0AF
:106A18001F0102FA01F10B4340F824305DF8044BE2
:106A280070474B0901F01F0150F82320012303FA96
:106A380001F1114214BF18460020704770B5448810
:106A48000546C4F30B0422460846002127F0F1FA54
:106A58002969094A9142034602D3084A914204D35C
:106A680041B11846BDE8704008472246BDE870406D
:106A780027F0BBBA70BD00BF4C70030874710308DF
:106A880038B5064C064DAC4206D26168204614342F
:106A9800FFF7D4FFAC42F8D338BD00BFEC6B030856
:106AA8004C7003082DE9F04F0F468DB0C2490646D9
:106AB800FDF709F90546002840F0FD81BF49304639
:106AC800FDF701F90546002840F0F781BC4930463A
:106AD800FDF7F9F80546002840F0F181B94930463C
:106AE800FDF7F1F80546002840F0EB81B64930463D
:106AF800FDF7E9F8002805460ABF012408243546B1
:106B08000FB144F01004B1492846FDF7DCF800281D
:106B180000F0D98144F02004FAF788FCFFF7B0FFB1
:106B280014F0090F00F048820020FDF725FF14F447
:106B38008073039340F0D181A548FCF703FE04F06D
:106B48001803182B40F0CC81A248FCF7FBFD012369
:106B5800029304F48473082B02D10020FDF766FD2C
:106B680014F080050BD19C4B1A78002A9B4A06BF6B
:106B78000121134600219A4A2046FEF7DFFC2046F1
:106B8800FEF7F0FC002D40F02882964F964B3E7899
:106B98001B78964D964AF01A464205EB8303464108
:106BA800D3F89C3231462046FEF7B0FC3B78904A39
:106BB80005EB83053146D5F89C328E4D2046FEF70D
:106BC800BDFCD5ED007A8C4AF5EE407AF1EE10FA6C
:106BD8000CBF012100212046FEF7B0FC2A46874958
:106BE8002046FFF7B1F8864B1F68864B93F82A209A
:106BF80002B1DF6A844BDFF814A2D3F80090DFF803
:106C080070B200265AF82650002D40F06C81DFF84B
:106C180064A22E4669EA070B7C4B53F82650002DD8
:106C280040F081817A4F7B4E6FF07F4300933A6842
:106C38003168794B2046FEF753FE40F20223009359
:106C4800BA68B168754B764F2046FEF749FE75481D
:106C5800DFF824C201262B5CEA5D0CA919440DF16A
:106C6800300E01F8202C15F80C108E440EF8102C5C
:106C780016B1591A4E424E410135082DEBD1314615
:106C8800002508AB684A8DF8185020468DF8285022
:106C9800FEF73CFC04AB3146634ADFF8E0B1DFF8AD
:106CA800E0912046FEF74AFC604A61492046FFF71A
:106CB800A9FA604A60492046FFF7A8FB5F4A604985
:106CC8002046FFF77BF95F4A5F492046FEF79CFFA5
:106CD8005E4A5F492046FEF7A7FE01265D4B5E48E7
:106CE800DFF8088102229919304427F06FF91BF860
:106CF80015304344B0FA80F793F8DD2019F81530C1
:106D0800022B4FEA571740F0328116F80B304FF03C
:106D1800190A40F2EE211AFB0313CDE90023394684
:106D28002B464E4A2046FEF7F1FB16F809304B4A2F
:106D380040F2EE211AFB0313019319F81530984419
:106D4800394698F8DD30009320462B46FEF7F6FBCF
:106D58000135122D06F10206C0D11F4B404E13F823
:106D6800112F002A1D4A06BF0121134600213D4A62
:106D78002046FEF7E3FB21460020FEF734FB14F023
:106D8800080F214600F010810020FEF7A9FB2146DC
:106D98000120FEF7A5FB344D21460220FEF7A0FB9B
:106DA80033782B70039B13B93048FDF779FAFF232A
:106DB8002B70002766E000BF2B2C0308322C030839
:106DC8003A2C0308402C0308E2290308492C03083D
:106DD800572C0308632C0308F82D0020D659030804
:106DE8005A2A0308583B0020043A0020E0E0020831
:106DF800732C0308A05800207C2C0308145B002087
:106E0800B85B0020F80F0020904A0020ECE302084D
:106E1800681A0020841A0020A22C0308A92C030851
:106E2800A01D0308D45A00202D250308225900204C
:106E3800005B00203C340020B83A0020A415002054
:106E4800081B0020503A0020403A002084170020F8
:106E5800D41A0020833A00205F3A0020482503080E
:106E6800F85B0020522A0308000000206528030868
:106E78008B2C0308972C0308E4590020843A00203F
:106E8800603A0020F8B221460137FEF713FB062FBF
:106E9800F8D173786B70039B002B7CD15148FDF7B8
:106EA800D3F95148FCF7CEFBFF236B70FAF7A8FA29
:106EB8000DB0BDE8F08F012422E6022420E6042468
:106EC8001EE681241CE649492846FCF7FCFE0028FA
:106ED8003FF422AE44F480741EE60023029338E6A1
:106EE8000123029335E62B78DBB14FF0010808FA4D
:106EF80006F869EA070313EA080F14BF0121002105
:106F08002B465A462046FEF701FB67EA090313EAB7
:106F1800080F5A462B4614BF012100212046FEF7D0
:106F28000DFB01366EE62B78FBB14FF0010808FA2D
:106F380006F819EA080F0BD067EA090313EA080FE5
:106F480052462B4614BF012100212046FEF7DEFAE7
:106F580018EA070F09D01BEA080F2B46524614BF40
:106F6800012100212046FEF7E9FA013654E6009295
:106F78002B4639461E4A2046FEF7C8FA19F815303E
:106F88001B4A9844394698F8DD30009320462B4632
:106F9800FEF7D4FADCE6FF236B70029B002B85D04A
:106FA8001448FCF7CFFB81E73078FEF799FA2146C1
:106FB8007078FEF77FFAF0E7A20705D50E4B214659
:106FC8001878FEF78DFA71E763077FF56FAF0A4B04
:106FD80021465878FEF76EFA68E721461820FEF732
:106FE80002FADAE7652803086E2C0308522C030816
:106FF80058250308B02C0308F85B0020012151E54F
:1070080000214FE52DE9F74F3A4B3B4C1A785B7856
:10701800009022706370FAF709FAFFF731FD002536
:10702800DFF8D8B0A8460D27344B00996F43DE1916
:10703800D6F800904846FCF715FE00283DD0B8F178
:10704800000F01D0FCF76AFB49462D485F44FDF765
:107058008BFB00213046FEF7BBF9FCF75FFB3B7961
:1070680003F01803082B3AD0102B3CD03046FEF71B
:1070780079F80D2303FB05B3B3F80900F9F7F1FC20
:107088000746C0B13046F9F782F9D7E901218246AF
:10709800024401443046F9F7B3F960B90190494612
:1070A8001848FDF761FB7968019A51443046FEF7AC
:1070B800C7F8FCF733FB08F101080135B5F5B87FCF
:1070C800B1D1FAF79DF9FF2323706370B8F1000F6F
:1070D8000DD10D4803B0BDE8F04FFDF71DB80B48C2
:1070E800FDF7DEF8C2E70948FDF7AEF8BEE703B0E2
:1070F800BDE8F08F245C00200000002024EA02088C
:10710800A4290308BA2C0308AF2703086528030835
:107118002DE9F74F814626F0ADF8054628B101283C
:1071280021D199F800302A2B1DD17C48DFF8048240
:107138007B4FFCF707FB00244FF00D0909FB048681
:1071480038463168FDF710FB291C18BF012130466D
:107158000134FEF73DF9FCF7E1FAB4F5B87FEDD15B
:1071680003B0BDE8F08F3D21484626F079FF00289E
:1071780000F0CF80074617F8013C202B07F1FF32BB
:1071880032D0A7EB09070130054601302B78202BB8
:10719800FAD0DFF8A0A14FF00008D346FFB20D23C4
:1071A80003FB08A42668304626F064F831460246F8
:1071B80001904846FCF732FD0646002840F09D80C5
:1071C800019BBB4240F09980237903F0600120299C
:1071D80051D00BD8F1B15348FCF79EFF204603B0BD
:1071E800BDE8F04FFDF7BEBF1746C4E7402958D0A9
:1071F8006029F0D14C4A02EBC606002796F88CA30A
:10720800B9463B46574502D2B9F1000F35D0002B9D
:10721800E1D00EE003F00706042E284618D125F029
:107228007FFFD4F8053083420146D4D32046F9F7CE
:1072380045FC0D2303FB08B83C48D8F80010FDF7BF
:1072480093FA0021204603B0BDE8F04FFEF7C0B81E
:10725800FCF776FDB4F805500146B4F80700AAB269
:1072680083B21EB1022E1CBF2AB203B29142B2DB16
:107278009942B0DCDAE76679BCE7D6F8882352F899
:10728800270060B129460193FCF703FD019B30B943
:10729800394620464FF00109F9F710FC4B460137F3
:1072A800B0E74FF00D0994F805A009FB08B9564559
:1072B800BFDA002DBDD02F4601353B78202BFAD000
:1072C8002046F9F7E5FB99F8043003F00703022B91
:1072D80005460CD0032B0AD03846FCF731FDA855DB
:1072E8002C21384626F0BCFE0136451CDFE738461F
:1072F800FCF726FD25F81600F2E708F10108B8F5B5
:10730800B87F7FF44CAF0A4803B0BDE8F04FFCF7F4
:1073180003BF484603B0BDE8F04F73E6CA2C030824
:10732800A4290308E82C0308E0E00208DD2C030880
:10733800AF27030824EA020810B50346F9F71FF837
:10734800044628B9062208491846FCF767FC48B9DC
:10735800FFF796FB054B002018701CB1BDE81040E4
:10736800FCF7E9BE10BD00BF6C2C03088913002090
:1073780010B5184B0446D02C18681CD0C02C0DD161
:107388000121FBF773F8144B186808B1FAF72EFFC0
:1073980021461248BDE81040F8F7B4BF0021FBF7BA
:1073A80065F80D4B18680028F0D121460B48BDE858
:1073B8001040F8F7A7BF0121FBF758F8064B1868EB
:1073C8000028E5D0FAF717FF21460448BDE8104029
:1073D800F8F798BF903F0020983F0020843F002096
:1073E8002DE9F043B64C237B8BB0002B00F088804E
:1073F800814600254021B348D4F808802573FBF75F
:1074080006F900F00303022B00F0158110F02106A5
:1074180047D1AD4F94F83150BB780B2B00F0A081C9
:10742800002D40F03A81F020FFF7A2FF05236A46BD
:107438004521A448F8F70EFF9DF80030AA2B30D15B
:10744800D7F85801DDF801604068236EA065C6F3DF
:10745800031001309D499E4AA66406F00F0C0133C3
:1074680000270928C4F8548028BF092001EB0C1113
:10747800236602F11006E76511F8013B1B1A02F8B2
:10748800013FB242F8D194F8323003F00F03E2180A
:107498000F2092F8341084F832300EF07DFAC4F8D8
:1074A8006480C020FFF764FF94F8303073BBA06E8F
:1074B80038B1FAF7EDFE94F86C3084F86C0003B13B
:1074C80090B394F826307BBB94F83130002B45D12B
:1074D80004F010FA636E7F4AC01A904204D994F8F7
:1074E8003430002B40F0B3807B4B7C4A1B68126819
:1074F800FA33934240F2998028460BB0BDE8F083F6
:1075080003F0FF0594F83030002BD0D004F0F2F9E6
:10751800236DC01AB0F5FA7FC9D9D020FFF728FF2C
:10752800002384F83030C2E7674B6D4A9B780B2BF9
:107538004FF00003536008BF0D21636318BF00219B
:10754800C2E902330F2084F8263084F83130A3646E
:107558000EF022FA94F83130002BB9D05A4F04F0CB
:10756800C9F9D7F858610246D6F800C0206F6521DE
:1075780001FB0CF1101A88420BD9216E226763298E
:107588009ABFC1F1640189B200210023A4F84E100A
:107598002366616FF368511A994203D90123626720
:1075A80084F84C30D4E91501131A8B4221D9B3FB66
:1075B800FCF6012E98BF4218A0206265FFF7D8FE9E
:1075C80094F83230334403F00F03E2180F2092F896
:1075D800341084F832300EF0DFF9C020FFF7C8FE0F
:1075E800E36D1F2B44D8D7F8582112680133C4E93A
:1075F80016233C4B186800283FF47EAF022D43D079
:10760800B4F87830B3F57A7F06D201332846A4F867
:1076180078300BB0BDE8F0832F4B304A1B681268F6
:1076280003F57A7393423FF667AF1BF01FFC2846B9
:107638000BB0BDE8F08394F83130002B40F0AD80FA
:10764800C020FFF795FE002594F830302EE7A36C94
:10765800002B3FF449AF244EE367A6F14C030FCB50
:10766800012586E80F0084F8315003F0B5FE3BE7AA
:107678001E4BD7F858211B789268A265032BB8D106
:107688001B4B00221A80B4E794F87A300022A4F841
:1076980078208BB9FAF7AFFD2EE7F020FFF768FEE8
:1076A80015236A4645210748F8F7D4FD9DF80030B0
:1076B800552B1FD03546F4E6FAF798FD1CE700BFB6
:1076C800F80F0020843F002000000020CCE50208CD
:1076D8002B100020400D0300EC310020603D0020FD
:1076E8002C100020F0310020781000207C2F002082
:1076F800A42F0020DDF80120A36C9A42DAD1FAF712
:10770800CDFFD7F85821236E5268C4F8548001334E
:10771800C4E916262366B9F1000F0DD00AAB53F859
:10772800232DC9F8002059689A68DB68C9F8041045
:10773800C9F80820C9F80C3094F83230013303F046
:107748000F03E2180F2092F8341084F832300EF04C
:1077580023F994F831300225002B3FF46DAEA0E6F2
:107768004DB3F0206E46FFF703FE25233246452130
:107778008748F8F76FFD9DF80030582B6AD0AA2B80
:1077880068D0562B66D0002594F83030002B7FF453
:10779800BDAEC020FFF7ECFD89E694F83230013326
:1077A80003F00F03E2180F2092F8341084F83230F7
:1077B8000EF0F2F844E7F0206E46FFF7D9FD1B23E0
:1077C800324645217248F8F745FD9DF80030AA2B4E
:1077D80040D03BD9BB3B012BD5D8D7F85821236ED5
:1077E8005268A2659DF80B20C4F854800133FF2A23
:1077F800C4E917535CD00AAD04F1340755F81D0DE0
:107808006968AA68EB680FC74FF0FF33626CDDF850
:107818000110CDF80520CDF80B3001226B60AB606C
:10782800EB602B616B612B83E020A16484F830202E
:10783800C4F86480C4F85080FFF79AFD32462523C7
:1078480005215348FBF716FE00255FE6562B01D0AD
:10785800582B98D1DDF80520636C9A4293D1DDF856
:107868000120A36C9A428ED1FAF718FF236ED7F83D
:1078780058119DF800204968C4F854800133002548
:10788800582AA165C4E9175315D094F83030002B55
:107898007FF43CAE94F83230013303F00F03E21862
:1078A8000F2092F8341084F832300EF075F86BE738
:1078B8000DF10B05A8E7B9F1000F16D00AAB53F884
:1078C8001F0DC9F800009A685968C9F80820DA68D5
:1078D800C9F804101869C9F80C2059699A69C9F8D7
:1078E8001000C9F81410C9F8182094F84C300BB9D6
:1078F8000225CAE7274BA08C1B88B4F84E1097F8CE
:1079080054918DF80B301A0A8DF80C20020AB9F13F
:10791800400F4FEA11238DF810204FF0FF324FF03F
:10792800000528BF4FF040098DF80F008DF813109F
:107938008DF81430AA21FE23CDF81920CDF8152092
:10794800CDF81D20CDF82120E020FC228DF8001074
:107958008DF809508DF80A508DF80E508DF8125098
:107968008DF80D208DF81130FFF702FD4B46324699
:1079780005210748FBF77EFD1522012384F84C50AA
:10798800C4F8508087F8542184F830300225BDE5CA
:10799800843F0020782500202DE9F0410646807BB1
:1079A8008846FAF745F80546002839D04F4F307B0E
:1079B8003378BB70002849D14D4B4E4C1860F07A93
:1079C800002876D1A066BB780B2B5AD008234A4EE4
:1079D80088F800302846C7F8586121F07DFF06F185
:1079E800100021F043FF0021E36FDBB984F8313048
:1079F800424B1A780AB903221A700F200DF0CCFFF7
:107A0800C020FFF7B5FC03F075FFD7F85821236EA7
:107A18005268A26501330022C4E91723606501207A
:107A2800BDE8F081364DA36405F14C030FCB85E822
:107A38000F0094F8323003F00F03E118012291F897
:107A4800341084F8323084F83120D1E7F9F7F0FFA8
:107A5800274C2060002841D0002205218171C27185
:107A68000121F9F72DFE737B2068224C1A1C18BFE0
:107A7800012284F87A200028A1D063BBFAF7B6FB6C
:107A88009DE70E221F4B204988F800201F4A0968ED
:107A98001B6812681E4EC7F858614B405340284671
:107AA800636421F019FF06F1100021F0DFFE0D21BB
:107AB8009AE7F9F7BDFF0646A06630B127220023F2
:107AC8008271C3712021F9F7FBFD3046FAF7E0FB1C
:107AD80084F86C0077E7FAF78EFB70E7737B054C48
:107AE800003318BF012384F87A3068E700000020CB
:107AF800F0310020F80F002010E702087C2F00204A
:107B08002C100020ACF7FF1FB0F7FF1FB4F7FF1FC2
:107B1800CCE6020838B5064C0D4601466068F8F711
:107B28007BFB29466068BDE83840F8F775BB00BFA5
:107B3800584300202DE9F843DFF8D080DFF8D090D3
:107B48002E4E04214046FAF717FDD8F80800FAF738
:107B58004DFB00210520FFF7DDFF00210620FFF780
:107B6800D9FF99F80010042041F00101FFF7D2FF76
:107B780033888BB1224F234D3C4615F8011FFF294E
:107B880008BF20210720FFF7C5FF2B7804F8013B29
:107B98003288E31B9A42F0DCFF210720FFF7BAFF87
:107BA80099F800100420FFF7B5FF3388DBB1164FB2
:107BB800002403E033880134A34214DD17F8015B85
:107BC800FF2DF7D1C4F307210520FFF7A3FFE1B28A
:107BD8000620FFF79FFF29460720FFF79BFF338802
:107BE8000134A342EADCD8F80800FAF704FBD8F815
:107BF80004000221BDE8F843FAF7E4BC5C07002062
:107C0800382000202F1E0020301E0020584300205E
:107C1800AC29002070B5134BC1F1030141EA800083
:107C280093F85C21C5B2AA421AD00F4E83F85C5172
:107C380030460421FAF7A0FCB068FAF7D7FA102406
:107C4800E0B229460134FFF765FF202CF8D1B0686F
:107C5800FAF7D1FA70680221BDE87040FAF7B2BCB1
:107C680070BD00BF0000002058430020F8B5374C15
:107C780004212046FAF780FCA068FAF7B7FA344BDB
:107C88001B78012B59D048D3022B39D1314F082307
:107C98003B704FF4C373304E304D33800221FF23C5
:107CA800002085F85C31FFF7B5FF04212748FAF773
:107CB80063FCA068FAF79AFA39780020FFF72AFFE0
:107CC800274B02201978FFF725FF264B0320197848
:107CD800FFF720FF244B197804200143FFF71AFF10
:107CE800A068FAF788FA60680221FAF76BFC328814
:107CF8001E48002126F09DF995F85D313BB9F8BD85
:107D0800144F3B785B06C4D54FF4F073C3E7FFF715
:107D180011FF002385F85D31F8BD0021A020FFF791
:107D2800F9FE00F00603022B0A4F03D000F005000D
:107D3800012808D008233B70ABE7064F48233B7067
:107D48004FF4F073A7E748233B70DDE75843002062
:107D5800944300209C0700205C07002000000020BE
:107D68009B4300209C430020AC29002038200020A1
:107D78002DE9F047404C414D414E04212046FAF789
:107D8800FBFBA068FAF732FA00218020FFF7C2FE59
:107D98000746A068FAF72FFA60680221FAF712FC82
:107DA8002B78D6F80080BB420DD1364B1F7847B9E7
:107DB800DFF8D890D9F89030A8EB0303B3F57A7FB1
:107DC80004D8BDE8F087BDE8F0474FE70421204616
:107DD800FAF7D2FBA068DFF8B8A0FAF707FA394635
:107DE800A020FFF797FE0746A068FAF704FA606834
:107DF8000221FAF7E7FB9AF80030192B0CD12B78FF
:107E0800214A03F04003002B07F007010CBF0D20A7
:107E1800102013805180D080790706D50023C9F837
:107E28009430C9F89080BDE8F08707F00507012F66
:107E38001AD0002FF5D12B785B06F2D5D9F89430FB
:107E4800B3B13268D31A642BEBD9FFF70FFF9AF856
:107E58000030192BE5D1B9F898300B4A01339BB2A1
:107E6800A9F898309380DCE72B785A06E6D5D8E74E
:107E78003368C9F89430D4E7584300209C070020A1
:107E8800603D002094430020B41C0020F80F00201F
:107E9800B01C0020074A00235168814202F11C02ED
:107EA80004D001330C2BF7D100207047581CC0B206
:107EB800704700BF0400002001382DE9F0434FEA65
:107EC800C00C394EDFF804E1384FDEF81490DFF8C3
:107ED8000081ACEB000406EB840483B06568BD4206
:107EE8000CBF01270227A56847EA09074545CEF8D0
:107EF8001470E16063613ED02D4B9D423DD0143338
:107F08009D423CD014339D4232D014339D4239D027
:107F180014339D4239D014339D4239D003F562732E
:107F28009D423AD014339D4239D014339D4232D009
:107F380014339D4235D01F491F4B8D420CBF1D463F
:107F48000025ACEB000C06EB8C069209747CF561FD
:107F58000021012301A88DF804408DF805208DF833
:107F680006108DF8073020F0C3FD03B0BDE8F0839C
:107F78004FF40055E5E70225E3E72025E1E74FF454
:107F88000075DEE74FF40035DBE74FF40015D8E75E
:107F98004FF00075D5E7094DD3E7094DD1E7094DF5
:107FA800CFE7094DCDE700BF0000002000000240E8
:107FB8001C00024058040240000002100002001099
:107FC80002000010200000100020001000100240E5
:107FD800080002400A4B0138C0EBC00003EB8000E8
:107FE80070B4084C084E43686569B3420CBF01235E
:107FF80002232B4363610176427670BC704700BF51
:108008000000002000100240000002402DE9F04F5F
:10801800544C54F8204083B0002C5FD0E56DA1602B
:108028001F469046504B6A686265236004F16202FD
:1080380004F1E2036261A36180224FF48073C4E912
:1080480003238146287E20F085FBE86860B1FFF7AE
:1080580021FF09F10102D2B20C21FFF7BBFF636DCA
:10806800EA68A26324332365A86898B1FFF712FF72
:1080780009F101020646D2B20B21FFF7ABFF2346F6
:10808800EA7E3A493046FFF717FF636DAA68E26354
:108098002833E36494F86100F9F7CAFC064694F8BB
:1080A8006000F9F7C5FC3A07824695F819B019D56A
:1080B800C6B117F0110F4FF00B0309F10100F07171
:1080C80014BF4E213E21B3715A463046F9F776FD6A
:1080D800FB0743D5A36B6BB3E36B5BB3204603B0DD
:1080E800BDE8F08F17F0010F0CBF2E274E2718F0B0
:1080F800020F0AD04EB10B2209F10103B271F371DC
:1081080030465A463946F9F759FD18F0010FE1D0C3
:10811800BAF1000FDED00C2309F101008AF807003C
:108128008AF806305A4639465046F9F747FDA36B98
:10813800002BD1D12B7FAA7E8DF804209B0900212A
:10814800012201A88DF805308DF806108DF807205A
:1081580020F0CEFC204603B0BDE8F08F3046FAF799
:1081680045F8B7E72C1A002054E70208650D000807
:108178000348D0F8403113B100F59C701847704798
:10818800000000200348D0F8243113B100F58E70A8
:1081980018477047000000200348D0F8083113B191
:1081A80000F5807018477047000000200348D0F899
:1081B800EC300BB1E4301847704700BF00000020D6
:1081C8000348D0F8D0300BB1C8301847704700BF0B
:1081D800000000200348D0F8B4300BB1AC30184789
:1081E800704700BF000000200348D0F898300BB15A
:1081F80090301847704700BF000000200248C36F46
:108208000BB1743018477047000000200248036E15
:108218000BB1583018477047000000200248436CE3
:108228000BB13C3018477047000000200248836AB1
:108238000BB1203018477047000000200248C3687F
:108248000BB1043018477047000000202DE9F843AF
:108258000501774C63596119002B00F0A080754A1D
:108268006719934204BF01230B730646387A20F03E
:1082780071FA3B7A03F01F015B090122022B02FA13
:1082880001F200F0AE80032B00F0A680012B03D191
:10829800694B996A0A439A62631901361879F9F7A2
:1082A800C7FBF6B2074610B11223C6718371631972
:1082B8005879F9F7BDFB10B11323C671837163199F
:1082C8009879F9F7B5FB10B11423C6718371661953
:1082D8000E21F2793846F9F771FC7079F9F7A8FBA5
:1082E800F2790E21F9F76AFCB079F9F7A1FBF27976
:1082F8000E21F9F763FC6359504A934276D04D4AF0
:10830800934200F089804E4A93427AD02C44227BD3
:10831800002A46D000252E4699884A4A21F48051E1
:108328000904090CA2F86851A2F866619980B3F8AB
:1083380004E0B2F86271B2F864C1B2F86A91B2F8B6
:108348006C81B2F86E01B2F860414EF4805EB7F508
:10835800827FA3F804E027D0998821F4706109048A
:10836800090C4CEA010199802743198849EA070456
:1083780048EA040401F4415120430843304345EAE4
:1083880000011980998BB2F8700121F4006212047F
:10839800120C9A8318821A8842F040021A80BDE8AB
:1083A800F88301250226B7E744EA0904198844F44A
:1083B800827448EA0404044301F44150044346EA41
:1083C800040028431880998821F470610904090C75
:1083D8004CEA01019980D5E7174B19690A431A61DC
:1083E8005AE7154BD9680A43DA6055E702F5604247
:1083F800D16841F48051D160D16821F48051D160B5
:1084080084E702F5EA32116941F40041116111690A
:1084180021F40041116179E702F5EC32116941F468
:1084280080411161116921F4804111616EE700BF3B
:108438006443002000380040001002400030014032
:10844800003C0040000000201749184B184A194802
:1084580010B4D1F8884044F47004C1F888401C680E
:1084680044F001041C605C6822405A601A6822F0DB
:10847800847222F480321A601A6822F480221A6008
:108488005A6822F4FE025A60DA6A22F00F02DA62AF
:108498001A6B002410404FF0006218639C608A60D9
:1084A8005DF8044B704700BF00ED00E0001002408B
:1084B8000CC07FF8CCFC00FF7047704770B50C4CBF
:1084C80023689BB15A68821A002A0FDB05460026EA
:1084D80003E05A68AA1A002A08DB99681E731A680A
:1084E8002160184690472368002BF2D170BD00BF69
:1084F80040110020436A8269D154436A0169C26B02
:1085080001338B4228BF002343623AB370B4EFF3C0
:108518001183502282F31288C66B3268D20704D5C1
:10852800DBB283F3118870BC7047716869B9D0E910
:108538000942944218D085691544F56018D9A21AE1
:1085480072608462002280F85820326842F001028A
:10855800DBB2326083F3118870BC7047426D1368D8
:1085680043F0800313607047012280F85820D7E752
:108578000469A21A72608162E4E7034610B4846B4E
:10858800D968406954B19A6C8C1A013A005D5DF85B
:10859800044B08BF0A46C0B29A6470471A6A805CE6
:1085A80001328A4228BF2246C0B21A625DF8044BE3
:1085B8007047C36B13B190F858007047D0E90903AE
:1085C800181AB0FA80F040097047D0E90912036917
:1085D800914238BFC9188A1AC16B013B19B1496861
:1085E8000A449A4201D2981A704700207047836B58
:1085F80043B1826C5B689A4291BF981AC0689B1A13
:10860800C0187047D0E907239A422FBFD01AC06814
:108618008018C01A704710B50E2204460021063093
:1086280025F007FD1423A3700523E3706371E3723B
:108638006373012323805223042100220220A374A0
:1086480064232171A271A0722173A273238210BDC9
:1086580008B51DF00FFA084B1B7943B1012B0AD15D
:108668000649074B0748084A0860DA6002E0044BED
:10867800054ADA60FEE708BD40110020FC9F002093
:1086880000ED00E0EFBEADDE0400FA052DE9F04F85
:108698002DED028BA0F10A0385B00C46ED2B00F2FC
:1086A800F686DFE813F0DA01F406F406F406F406B9
:1086B800F406F406F406F406F406F406F406F406E2
:1086C800F406F406F406F406F406F406F406F406D2
:1086D800F406F406F406BC01F406F406F406AD014B
:1086E800F406F406F406A001F4063001F406F406D4
:1086F800F4061D01F4064103F4061C03F4060803FE
:10870800F406F406F4060203FB02F406E802F40693
:10871800F406E102F406F406F406F406F406CF02C1
:10872800F406F406F406F4065F05F4063E05F406BE
:10873800E4062305F406F406F406F406F406F40643
:10874800F406E004F4069904F4062304F406650329
:10875800F406D206F406F406F406F406B80675061E
:10876800F40622060F06F406F406F705D505F40606
:108778007F05FF00F406F406F406F406EE00F4069E
:10878800F406F406F406F406F4069A028302A90233
:10879800F406F406F406F4067402F406F4066C0211
:1087A800F406F406F406F406F406F406F406F406F1
:1087B800F406F406F406F406F406F406F406B8061D
:1087C800F406F406F406F406F406F406F406F406D1
:1087D800F406F406F406F406F406F406F406F406C1
:1087E800F406F406F406F406F406F406F406F406B1
:1087F800F406F406F406F406F406F406F406F406A1
:10880800F406F406F406F4065D02F406F406F4062B
:10881800F406F406F406F406F406F406F406F40680
:10882800F406F406F406F406F406F406F406F40670
:10883800F406F406F406F406F406F406F406F40660
:10884800F406F406F406F406F406F406F406F40650
:10885800F406F406F406F406F406F406F406F40640
:10886800F406F406F406F406F406F406F406260202
:10887800F4061B02F406F406F406F406F406F406FD
:10888800EC01AD4952232268501C2060137011F886
:10889800013F002BF7D10125284605B0BDEC028B1E
:1088A800BDE8F08FA54800220168256802EB420365
:1088B8005B0019446E1C097A2660297001682568D6
:1088C80019446E1C497A26602970016825680B4492
:1088D80001329B7A691C052A21602B70E4D1DAE702
:1088E800202500212046FAF7DFFF013DF9D1236852
:1088F80093495A1C22601D702268C978531C236052
:1089080001251170C8E78F4D0B682A7A8E4E591CC5
:1089180021601A70E98A2046FAF7DDFF698A204645
:10892800FAF7D9FFA98A2046FAF7D5FF23686A7BA8
:10893800591C21601A70E98B2046FAF7CCFF298C64
:108948002046FAF7C8FF23682A7E591C21601A704E
:108958002368AA7E591C21601A702B7F03EB8303BE
:10896800590001F57A712046FAF7B5FF2368327885
:10897800591C21601A7071682046FAF795FF236820
:10898800327A591C21601A702368EA7E591C2160CA
:108998001A7023686A7E591C21601A70236895F83A
:1089A8002520591C21601A70236895F82620591C27
:1089B80021601A70236895F82720591C21601A70C5
:1089C800236895F82920591C21601A70236895F8A6
:1089D8002A20591C21601A7022680021531C236028
:1089E8000125117058E70A68584B501C1978206007
:1089F800117022685978531C2360012511704BE7C8
:108A0800534D08462988FAF766FFA9882046FAF7E1
:108A180062FF29892046FAF75EFF01253CE74D4DA4
:108A280005F1780628780FF0C1FF2368027A591CEF
:108A380021601A7023686A78591C21601A702368AB
:108A4800AA78591C21601A702368EA780635591CDF
:108A5800AE4221601A70E5D11DE73F4D284624F04B
:108A680009FC00283FF417AF2B460544226813F889
:108A7800011B501C9D4220601170F7D10BE701A823
:108A8800FBF7BCF900283FF406AFBDF804102046F8
:108A9800FAF721FF23689DF80620591C21601A70F7
:108AA80023689DF80720591C21601A7023689DF8D7
:108AB8000820591C21601A7023689DF80920591C48
:108AC80021601A7023689DF80A20591C21601A70C9
:108AD8002046BDF80C10FAF7FEFEDCE61F4D0846EE
:108AE800A989FAF7F8FE69892046FAF7F4FE012504
:108AF800D2E60B68174D591C1422216005F178063F
:108B08001A7028780FF052FF074668790FF04EFF69
:108B180023683A7A591C21601A7023682A79591CEB
:108B280021601A702368027A0635591CB542216003
:108B38001A70E6D1AFE600BFD4FC0208D8220020A4
:108B480050220020E4590020B4340020043A0020C8
:108B58005C1A00203C340020902B00204C2A002076
:108B68000B68754A591C1278216001A81A70FBF726
:108B780045F92268531C2360012510708CE66F4B61
:108B88001B6813F0006340F05E851D4684E66C4D5B
:108B98000846698AFAF79FFEA98A2046FAF79BFEDB
:108BA800E98A2046FAF797FE012575E60A68654BBB
:108BB80065491878551C2560107022685878551C2E
:108BC8002560107022689B78501C20601370204626
:108BD800C988FAF780FE01255EE65B4D08462988BC
:108BE800FAF779FE69882046FAF775FEA9882046C3
:108BF800FAF771FE01254FE60B68544A5448D179BB
:108C08005D1C2560197023685D1C25601970236838
:108C1800807850495D1C2560187023680978581CB5
:108C28002060197023680021581C2060197023687F
:108C3800D279581C20601A702268531C23600125C1
:108C4800117029E60B6800255A1C0A60204629463F
:108C58001D70FAF729FE29462046FAF725FE29460F
:108C68002046FAF721FE16E6084608223A49FAF79E
:108C780011FE012510E60B68384A39495278581C0C
:108C880020601A7023680022581C20601A7022681D
:108C98000979531C236001251170FDE50A6801213B
:108CA800531823600D461170F6E508460021FAF7BF
:108CB800FBFD0125F0E52B4D2B4E05F1100795F92D
:108CC800023096F906209A4200F0448496F90E2064
:108CD8009A4200F03F840835AF42F0D1DBE5234BE0
:108CE80003F5967522685979501C20601170226826
:108CF8001978501C2060117022685978501C206027
:108D0800117022689978501C206011702268D978F7
:108D1800501C20601170226819790A33501C9D423A
:108D280020601170DED1B6E50A680B4BD97B531C65
:108D3800236001251170AFE57C2F0020904A0020A8
:108D4800A84B0020A030002024390020B430002097
:108D5800403B0020AF300020E4590020A83000201C
:108D6800281E00202259002098400020A415002029
:108D780000212046FAF7AFFD00212046FAF7ABFDA7
:108D880000212046FAF7A7FD2368914D00265A1CBA
:108D980022601E7023682A68591C92F846202160B8
:108DA8001A7023682A68591C92F8472021601A70A3
:108DB80023685A1C22601E7023685A1C22601E7089
:108DC80023685A1C22601E7023685A1C22601E7079
:108DD8002B682046198FFAF77EFD2B682046D98E1E
:108DE800FAF779FD2A68236892F82D20591C21602A
:108DF8001A7023685A1C22601E702B682046598EF0
:108E0800FAF769FD2B682046998EFAF764FD31461A
:108E18002046FAF760FD2A68236892F85120591C09
:108E280021601A7023685A1C22601E7023682A6801
:108E3800591C92F8552021601A7023682A68591C19
:108E480092F8532021601A7023685A1C22601E7001
:108E580023682A68591C92F84F2021601A702368E9
:108E68005A1C22601E702B6820469989FAF733FD38
:108E78002B682046598AFAF72EFD2B682046198B55
:108E8800FAF729FD2A68236892F83020591C2160D6
:108E98001A702A68236892F86E20591C21601A708B
:108EA8002A68236892F86F20591C21601A702A6872
:108EB800236892F87020591C21601A702A68236868
:108EC80092F87120591C21601A702A68236892F858
:108ED8007220591C21601A7023685A1C22601E7067
:108EE8002268531C236001251670D5E4394E0B689F
:108EF800B279374D591C21601A702B682046598861
:108F0800FAF7E9FC2B6820461988FAF7E4FC71891E
:108F18002046FAF7E0FCB1892046FAF7DCFC2B681A
:108F280020469988FAF7D7FC2B682046D988FAF7A3
:108F3800D2FCF1892046FAF7CEFC318A2046FAF7AE
:108F4800CAFC2A68236892F82620591C21601A70E6
:108F58002368B278591C21601A7023680022591CB2
:108F680021601A70F1882046FAF7B5FC318920464D
:108F7800FAF7B1FC2368727D591C21601A702368C6
:108F8800B27D591C21601A702B682046B3F84C102A
:108F9800FAF7A1FC23682A68591C92F8602021601E
:108FA8001A70B18B2046FAF796FCF18B2046FAF737
:108FB80092FC2B682046B3F86210FAF78CFC2B68F9
:108FC8002046B3F86410FAF786FC012564E400BF74
:108FD800D8220020D04300200B68A34EA34A717802
:108FE800A34D581C2060197023681278591C216001
:108FF8001A7023682A79591C21601A702368AA7884
:10900800591C21601A7029882046FAF764FC298ABD
:109018002046FAF760FC23680022591C21601A7068
:109028002368EA78591C21601A7023683279591C20
:1090380021601A702368F278591C21601A7023681D
:109048003278591C21601A70718B2046FAF743FC5C
:10905800718A2046FAF73FFC2268317D531C236051
:109068000125117018E4834B1E6800238DF8043025
:10907800002E00F0A78201A9304616F09BF833684D
:1090880030465B68984733689B680746002B00F0BA
:109098000A833046984706462368774D5A1C226053
:1090A8001F7023682A78591C21601A7023686A780F
:1090B800591C21601A702368AA78591C21601A70FB
:1090C80023689DF80420591C21601A70A98820463D
:1090D800FAF701FC23685A1C22601E702268297A5C
:1090E800531C236001251170FFF7D6BB0A68634B38
:1090F80063490125501C206015702268987856191C
:10910800266010702268501920601570226809784E
:1091180050192060117019882046FAF7DCFBFFF718
:10912800BBBB584F3B78002B3FF4B5ABDFF86081F1
:1091380000254646236818F81520591C21601A7026
:10914800717801EB810101EB810101F2EE212046EA
:10915800FAF7C1FB3B780135AB4206F10206E9DCC0
:10916800FFF799BB484D0B682A79591C21601A7082
:1091780023686A79591C21601A7029882046FAF7F1
:10918800AAFB2368AA79591C21601A7069882046AD
:10919800FAF7A1FB2268E979531C236001251170B5
:1091A800FFF77ABB394D0B682A68591CD2782160C1
:1091B8001A702B6822689979531C23600023117058
:1091C8002A6821681A440133527A481C032B20600C
:1091D8000A70F5D12A682368127B591C21601A701D
:1091E8002A6823681278591C21601A702A68236833
:1091F8005278591C21601A702B682046D989FAF7D1
:109208006AFB2A682368127A591C21601A702A6836
:1092180023685279591C21601A702A6823681279C8
:10922800591C21601A702A682368D279591C216058
:109238001A702A682368127C591C21601A702B68DE
:109248002268597C531C236001251170FFF724BB49
:1092580000212046FAF728FB20460021FAF73BFBBD
:109268000125FFF719BB00BFD0430020983000202C
:10927800A84B0020602200205E2500204C250020FD
:1092880084300020642F0020B4390020DC36002010
:10929800843A0020CC4D08462988FAF71CFB6988D7
:1092A8002046FAF718FBB5F90430C84AD91782FBEB
:1092B8000323C1EBA301204689B2FAF70CFB012571
:1092C800FFF7EABAC24F3B78002B3FF4E4AAC14E3D
:1092D800002536F9021B204689B2FAF7FCFA3B78DA
:1092E8000135AB42F5DCFFF7D6BADFF824A3DFF887
:1092F80024B3B94EB94F9FEDBA8ADFF81C83DFED6E
:10930800B98ADFF818930AF1C0050EE0FCEEE77A97
:1093180017EE903A99B220460AF1180AFAF7DBFAE2
:1093280055450BF1040B3FF4B6AA9AF81110002921
:10933800F1D03378DBED007A012BE7D13B68DB0411
:1093480040F12681F5EE407AF1EE10FA00F06A81DC
:10935800F4EEC87AF1EE10FA00F16481BDEEE77A16
:10936800F4EEE87AF1EE10FA17EE103A00F28B817B
:10937800A3F130026FF4F97303FB02F389FB0312C4
:109388001A44D917C1EB622101F2DB5189B2C2E755
:10939800954B1B8BB3F5006F00F21181B3F5806F0D
:1093A80000F26E81B3F5007FB7EE008AF6EE007A20
:1093B80028BFB0EE678A8D4D05F10C06B5EC010AA1
:1093C80020EE080A24F0B6FD81B22046FAF783FAA7
:1093D800AE42F3D1864D874F05F10C06B5EC010A74
:1093E800D7ED077A80EE270A24F0A4FD81B2204643
:1093F800FAF771FAAE42F1D100212046FAF76BFA7A
:1094080000212046FAF767FA20460021FAF763FAA6
:109418000125FFF741BA002306461D46DFF8008202
:10942800CDE90133994601E0282D38D02946404638
:10943800FDF7F7FAEFB201350028F5D038460FF0FE
:1094480029FA38BB09F10109EEE70B686A4A591C89
:10945800927821601A7023680122991821601A7085
:1094680021688B18236015460A70FFF715BA0B6838
:1094780000255A1C0A601D700B685A1C0A601D7072
:109488000B685A1C0A6029461D70FFF7E5BB0025CA
:10949800FFF702BA494601A8FDF7B4FAD2E7574BDD
:1094A800574DB3F89C102046FAF715FA00212046CC
:1094B800FAF711FA534B19684B0103F02002C1F374
:1094C80040031343C1F3800243EA4203C1F3C002DD
:1094D80043EA8203C1F3401243EAC20301F01001D8
:1094E80019432046FAF7F7F901A904222046FAF7AA
:1094F800D1F923682978444A581C206019701188CA
:109508006429A8BF64212046FAF7E5F9962E00F0F1
:109518008F8000212046FAF7DEF92168B9F1190396
:1095280048BFA9F11203A3F3C4034A1C22602046D2
:109538001A460B7002A9FAF7ADF92368334A581C8A
:1095480015212060197020461168FAF7ADF9012538
:10955800FFF7A2B92268511C2160137029882046A0
:10956800FAF7B9F92368EA78591C21601A70236858
:109578002A79591C21601A702368AA79591C21601C
:109588001A7023686A79591C21601A70FFF7A3BB07
:10959800F4EEC87AF1EE10FA47DBFDEEE77A40F216
:1095A800E73217EE903A303B02FB03F388FB0321C6
:1095B800DB17C3EB612101F2E93189B2ABE6B4EE06
:1095C800008AF8E6FF2767E51C1E002067666666C6
:1095D800642F0020D4290020C24B0020904A00208C
:1095E8000000404200E08244842A0020B02A002083
:1095F800FC430020084400204C2A0020940100204D
:10960800245C0020482A002098130020B02900205C
:10961800E84A002034260020DB9B91412105348351
:10962800F013002040F2DC5175E64FF47A7172E6CF
:1096380023680322591C21601A7023686A78591C10
:1096480021601A7069E70B68184E591C327821603E
:109658001A703378002B3FF41EA90025E8B213F0E6
:10966800DFFE23684278591C21601A7081892046E0
:10967800FAF731F933780135AB42EFDCFFF70BB974
:10968800B5EE008A97E6A3F5836240F2F31303FB75
:1096980002F389FB03121A44D917C1EB622101F2C4
:1096A800DD5189B237E61846F5E400BF205900209D
:1096B80038B5084D002415F8013BFF2B184605D096
:1096C8000FF0E8F801462046F8F7A2FD0134042C13
:1096D800F1D138BDA4430020064B1B7803B1704775
:1096E800054B1B685B05FAD5044B1B78002BF6D19C
:1096F80018F090BE4D270020904A0020B03000207E
:10970800064B1A68904203D09A68904204D10833F5
:109718000022C2629A801A60704700BF98400020F9
:109728000A4A0B491388184210B50C4609D1138907
:1097380018404FF0020307D0012002EBC00023704D
:1097480010BD00200123F8E70B70F9E7225900202B
:109758004C14002018280BD8064B00EB400003EBF4
:109768008000007F28B10123013803FA00F0704718
:1097780000207047D4FC0208024A1368184310609E
:10978800704700BFB02900202DE9F04FE04D2DEDC6
:10979800068B2B7891B0044643B1DFF8CCA3DAF8F6
:1097A8000C305046984780F001002870D94B1A7841
:1097B800002A00F04882D849D848D94E0D7804F5D7
:1097C800EC425F320260002032681870002D00F011
:1097D800F581944201D9013D0D7020460CF054FBEF
:1097E800002800F03082CF4DCF4AD5F89030C5F828
:1097F8009040E41A47F230539C421668CB48CC4953
:10980800B6F80EC0CB4FA8BF1C46B4F57A7FB0F9A6
:109818000630B8BF4FF47A740C8063454FF00104EA
:109828003C7080F22882C44A4FF07E511160C34ACE
:10983800C349B0F900804E8A92F9044092F800E0DA
:1098480092F801C0002CA8EB060214BF01274FF0C4
:10985800FF37002AB8BF5242B2F5FA7FA8BF4FF4CB
:10986800FA727245C6BFA2EB0E0207EE902ADFED30
:10987800B57AB54CC8BFF8EEE77A4645B0F902802C
:10988800C4ED007AA8EB0602C4BFF1EE677AC4ED16
:10989800007A002AB8BF5242B2F5FA7FA8BF4FF447
:1098A800FA729645BABFA2EB0E0207EE902ADFEDD8
:1098B800A57AB0F90400B8BFF8EEE77AB045A0EB96
:1098C8000602C4ED017ABCBFF1EE677AC4ED017AF5
:1098D800002AB8BF5242B2F5FA7FA8BF4FF4FA7215
:1098E800944580F2E181A2EB0C0C07FB0CFC07EE1F
:1098F80090CAF8EEE77A954AC4ED027A8642106873
:10990800C4BFF1EE677AC4ED027A10F4805000F01B
:109918009F81B3F5FA6FA8BF4FF4FA63B3F57A7F66
:10992800B8BF4FF47A73A3F57A71894B1A78002A75
:1099380040F09781874FDFF834C287FB0123CA17AD
:10994800C2EB63135A1C6FF0630E3CF912203CF90A
:1099580013C00EFB0313A2EB0C0203FB02F387FBFD
:109968000327DB17C3EB671363441BB207EE903A78
:10997800B8EEE78A84ED038A002840F0B581764B7B
:109988001B885A0640F10F8140F603027349D4ED53
:10999800011A91ED018AD1ED033A91ED029AD1EDC8
:1099A800005A94ED002A13406D4A08BFD4ED022AEC
:1099B80092ED014A92ED026AD2ED006A92ED030A35
:1099C80018BFDFED602A674A38EE635A74EE460A1C
:1099D80076EE807A65EE200A75EEC94A35EE89AAD8
:1099E80076EEC09A64EEA74AB0EE603AAAEE293A3B
:1099F800B0EE645A38EE237A74EE067AAAEE295A43
:109A0800A7EE273AA7EE675AB0EE601A97EE271A24
:109A180033EE243AF6EE008A75EE88AA28EEC33AA9
:109A280035EE605A76EE840AB0EE417AAAEE691AEB
:109A3800AAEEA03A77EE647A76EE400A73EEC9AAE7
:109A480025EE285AEAEE297AAAEEA05A71EE244A9F
:109A580036EEC44A63EE036A73EE893A64EEA84AA6
:109A680075EEC85A36EE006A67EEA87AB0EE667AE6
:109A7800E3EE844A95EE057AE5EE056AE5EE867A28
:109A8800B1EE648AF0EE665AF0EE476AB1EE674AC4
:109A9800E8EE246A63EE270A67EEA43AE4EE275A52
:109AA800B1EE450AB0EE606AB0EE631AA4EE277A0A
:109AB80023EE244AE7EEA76AA5EE246AA0EE031A6D
:109AC800E8EE245AB0EE448A31EEA19AE0EE240A78
:109AD800A5EE278A66EEA16A72EE028AE5EE033ADF
:109AE80061EE211A26EE096AA4EEA47AA0EE274AAE
:109AF800A2EE256AE8EEA06AE2EE081A73EEA33A2F
:109B080027EE227A34EE044AF0EE005A30E000BF25
:109B1800A62F0020AC2F0020F0330020A82F002013
:109B2800EC33002040110020DC360020D42900202E
:109B38008614002084140020D8360020A03000208D
:109B4800E45900200000000030320020904A002034
:109B5800A81300201F85EB5108260020140F0020B1
:109B6800240F0020340F0020642F00200C3A00201E
:109B7800E2EEA36AA4EE226AA1EEA57AC5ED266AF2
:109B8800C4ED016A85ED256A84ED006A85ED277AC2
:109B980082ED005A82ED013AC2ED027AC2ED034A23
:109BA800002B00F0DA81684B1B78DB077FD411B0FB
:109BB800BDEC068BBDE8F04F06F01EBA94427FF666
:109BC8000CAE624B1E78002E00F0E280DFF8B8A1E0
:109BD800DFF8B0B1DFF8A881DFF8B091574628E088
:109BE80018F805109847032D03462ADCC8B109EB7D
:109BF800850339F825105A88401A4FF47A7303FB05
:109C080000F0521A40F6CA0390FBF2F000F57A70A1
:109C18009842A8BF184640F2EE239842B8BF1846AB
:109C280000B24A4B2BF8020B1E780135B54280F280
:109C3800AF80072D3846DAF80430D1DDE9B298470D
:109C4800034618B2EDE711B0BDEC068BBDE8F08F06
:109C58008A8A934238DA3E4B1A780146002A3FF442
:109C680069AE5B783B4A01FB03F382FB0321DB17F8
:109C7800C3EB61115EE6B3F5FA6F327B9FED367A7E
:109C8800BFBFA3EB0C014A43CCF5FA6192FBF1F29A
:109C9800C2F1640207EE902AF8EEE77A2F4A67EEDF
:109CA800877AC2ED007AC2E5DFED2D7A23E62D4AE8
:109CB8002D4B1178186801F0010111B0BDEC068B2D
:109CC800BDE8F04FF8F79CBAB3F5FA6FD4BFC2EB12
:109CD8000303C2F5FA634FF47A71C2F5FA6201FB25
:109CE80003F3B3FBF2F120E6204BDB78002B7FF483
:109CF80046AE1F4B1F481F7B1521FCF792FE002F15
:109D080040F0338100283FF43AAEDFED1B7A1B495F
:109D180078EE677AC6F5FA63FDEEE77A1AB217EEBF
:109D2800903A1BB21B0381FB0301DB17C3EBA113A2
:109D380002FB03F343F30F33334407EE903AF8EE94
:109D4800E77AC4ED037A1AE6231E0020C434002003
:109D5800A81300201F85EB510AD7233CD8360020D2
:109D6800000000001F3F0020203F0020A425002005
:109D7800243900205C30002000007A44D34D621062
:109D8800E459002048110020642F0020503A002098
:109D9800B94B1A78B94BD3F80090002A40F0E0800C
:109DA8001346B749097804912A2904D1B548B64918
:109DB800007848800A80B54A01251570002E00F009
:109DC800AB81B34AB34F10780390B348DFF800C3B0
:109DD800C18B0191018C0291418A03980A91397BC8
:109DE8000D910746ACFB07714908079201EB410149
:109DF800AA4ADFF8E0A21268DFF8B4B20B95411A5C
:109E0800C8B206F1FF380590CDE90864400042F277
:109E180001010690B8F1030F02F480500C9002EA99
:109E28000102A8BF4FF003080025002B00F0DD80D9
:109E38009B49019831F8151081424FEA4507C0F057
:109E4800D4800298814200F2D08009F596704AF8D1
:109E5800250009B2002A40F0E8802BF807100135E8
:109E68004545E2DDDDE90864AE4227DD8D4FDFF8C8
:109E780040B2069405EB450107EB4107002B00F0C3
:109E880099808749019831F8151088424FEA4508AA
:109E980000F2908002988842C0F08C8009F5967094
:109EA8004AF8250009B2002A40F016812BF808105C
:109EB8000135AE4207F10607E0D1069C734B1B78CB
:109EC800002B40F02B816F4B012204201A70FFF702
:109ED80053FC754A694BD2E901101B68D3601B1A01
:109EE8008B4202D9002382F82130704B1E78644BD4
:109EF8001B780493002E00F02881664A674B117B7B
:109F08001B68654A03F48053B2F81E80578A0029FB
:109F180000F046816649674D83B1ACE1022A40F002
:109F28002781427802EB820202EB820202F2EE22E1
:109F380001339E4221F8022B00F0078115F8132007
:109F480005EB4300002AE9D1DAB2022A40F2608127
:109F5800032A40F00D814246EAE784ED027A22E6C0
:109F6800484B1B7883F001031BE7DFED537A534A14
:109F780038EE678ABDEEC88A18EE103A1BB21B038A
:109F880082FB0312DB17C3EBA213002800F02A811F
:109F9800C6F57A7212B203FB02F343F30F3333446C
:109FA80007EE903A464BF8EEE77A0122C4ED037AC1
:109FB8001A70E4E45AF82510A9EB01010029FFF60C
:109FC80077AF3C4810F815104FEA4508404400297F
:109FD80000F0D080022940F0C880417801EB81016F
:109FE80001EB810101F2EE215CE75AF82510A9EB9B
:109FF80001010029FFF633AF2E4810F815106F0045
:10A008003844002900F0C180022940F0AB80417833
:10A0180001EB810101EB810101F2EE211B4C0020D3
:10A02800207009B2002A3FF418AF1E48254C069E3E
:10A0380094F874E007EB050C00EB4C008153BEF17B
:10A04800000F06D1039E022E7FF607AF0B9984F806
:10A0580074104188B0F804E0124830F81C007144CC
:10A06800014408B2184981FB0041184CA1EBE0718A
:10A07800E05309B2F1E600BF482F0020603D002000
:10A08800B01C0020E80E0020B41C00206430002022
:10A09800F133002024390020E4590020904A0020A0
:10A0A800481100206C110020A4250020C434002091
:10A0B800D4290020843A002000007A44D34D62104D
:10A0C800201500204011002056555555B811002084
:10A0D800ABAAAAAAF43300208B48059C90F8740018
:10A0E80027F8141038B9039C022C7FF6DFAE864897
:10A0F800012180F874107988B7F800C0B8886144E5
:10A10800014408B2814981FB0041814CA1EBE07117
:10A1180024F8080009B2C9E67E4B07937E48062159
:10A12800FCF77FFC00287FF4CEAE7C4A7C4BD168DC
:10A138001B6893605B1AC82B07D97A490B68012002
:10A1480023F004030B6082F82100049B2A2B03D11F
:10A15800754A764BD288DA80079A137801331370E0
:10A16800FFF73BBB3BF8071058E73BF8081099E6A8
:10A178000A88DDE6E9B2022948D90329F5D10C9904
:10A18800002940F09C8001998CE6E9B202293BD96C
:10A198000329E7D10C99002940F0A38001993DE7F4
:10A1A800002B39D16049624D0DE0022A18D142785E
:10A1B80002EB820202EB820202F2EE2201339E429D
:10A1C80021F8022BC1D015F8132005EB4300002A13
:10A1D800EBD1DAB2022A1DD9032A01D14246EDE7B2
:10A1E8000A88EBE7C6F5FA6212B203FB02F343F3FF
:10A1F8000F33334407EE903A4E4BF8EEE77A187077
:10A20800C4ED037AFFF7BBBB0A9907E70A9949E649
:10A218003A468DE63A46D1E7DFF80CA1444DDFF81F
:10A22800F8B089460EE0022B22D1507800EB80006E
:10A2380000EB800000F2EE2009F10109B1452AF88F
:10A24800020B82D015F8193005EB4902002BEAD130
:10A258005FFA89F3022B2ED9032B4FF015015846CC
:10A2680006D1FCF7DEFB00280CBF38464046E3E782
:10A27800BAF80000E0E700230EE0022A19D142787C
:10A2880002EB820202EB820202F2EE2201339E42CC
:10A2980021F8022B3FF459AF15F8132005EB4300C2
:10A2A800002AEAD1DAB2022A07D9032A01D14246A2
:10A2B800ECE70A88EAE73846BEE73A46E6E71521BA
:10A2C8001548CDE90832FCF7ACFBDDE90832002877
:10A2D8007FF459AF0D99019800290A9918BF0146D2
:10A2E800E0E515210C48CDE90E32FCF79AFBDDE9D3
:10A2F8000E3200287FF452AF0D99019800290A996F
:10A3080018BF01468AE600BF401100205655555532
:10A31800B8110020F13300205C300020A425002073
:10A32800603D0020B0290020D4290020B41C002062
:10A33800843A0020201500205F4B60482DE9F04149
:10A34800542201245E4E1C70002123F072FE5D4AE7
:10A358005D495E4D002330460B6013600EF040F9F6
:10A36800214620460EF08AF9214606200EF086F98D
:10A378006F7A574B391C1A8A564B93FBF2F318BF66
:10A388000121642BB8BF64230820C6F890310EF071
:10A3980075F995F80A8018F100014FF0090018BF07
:10A3A80001210EF06BF9AB7B002B4CD04A4C002FEF
:10A3B80053D118F1000118BF0121484D0A200EF0B1
:10A3C8005DF92B68D9074AD49A0764D4012105207E
:10A3D8000EF054F9002107200EF050F901210B204E
:10A3E8000EF04CF921684B0546D4C1F300410D200D
:10A3F8000EF044F9216811F4802104D0384B196813
:10A40800003118BF01210E200EF038F921680F2005
:10A41800C1F3C0610EF032F9012113200EF02EF9BC
:10A42800012110200EF02AF9012111200EF026F941
:10A438002C4B196800314FF0120018BF0121BDE8FC
:10A44800F0410EF01BB9EB7B234C002BAFD12168F8
:10A4580011F48021B1D0002FABD00121ADE7224B00
:10A468001B68642BB8BF642301210220C6F8903012
:10A478000EF004F92B68A7E701210C200EF0FEF876
:10A488001A4B21681B7A083B012B9CBF4FF4FA63D7
:10A49800C6F81033A9E7012103200EF0EFF8144B9A
:10A4A8009B6A642BB8BF642301210420C6F8D0300E
:10A4B8000EF0E4F88AE700BF10180020BC1700204F
:10A4C8009401002024180020B8170020401D002007
:10A4D8002259002040420F00904A0020482A0020BC
:10A4E800C8260020C42A0020F8430020E459002090
:10A4F800842A002008B501210020F7F7AFFE0121CA
:10A508000846F7F7ABFE01210220F7F7A7FE104B2C
:10A518001B7803F00503052B17D000210846F7F731
:10A528009DFE00210120F7F799FE00210220F7F790
:10A5380095FE1EF079F80020F7F751FE0120F7F795
:10A548004EFE0220F7F74BFEF3E71BF029FBE4E78A
:10A5580028180020594B1A6840F2EE239A4210B589
:10A5680000F29880564B5A899989914224BF00225B
:10A578005A81198ADA89914228BF0022998B28BF0B
:10A58800DA81DA8B914284BF00229A839A784D4906
:10A59800012A91F8581032D00A2935D00C2976D1E1
:10A5A8009FED497A494CA278062A97BF4849DFEDC2
:10A5B800496A01EB8201D1ED526A217969B3013A06
:10A5C800032A6CD9444A45499378013B012B9CBF27
:10A5D800002393704B78052B45D803EB4300404A82
:10A5E80003EB800302EB43030A783E48022A036028
:10A5F80041D900230B703C4B3C4A1A6010BD3C48C3
:10A608005A700A29027040D19FED3A7A012AC9D1BD
:10A618000A2950D19FED387AC4E75B78344907EEB0
:10A62800903A0A78F8EEE77A67EE877A07EE102A0A
:10A63800B8EEC77A27EE277AF4EEC76AF1EE10FA79
:10A64800C0DD86EEA77AFDEEC77A17EE903A102B9A
:10A65800A8BF1023012BB8BF0123DBB29A4238BF31
:10A668001A460A70AEE700224A700A781D481C4B49
:10A678000360022ABDD81D4BC2EB0211C2EB810256
:10A6880003EB4202184B1A6010BD0C2913D09FED42
:10A698001B7ABBE74FF00050F9F75AF862E7B7EEBC
:10A6A800000A80EE260A23F045FC2388984228BF3A
:10A6B8001846208086E79FED127A73E7F84300205A
:10A6C800D0430020084400200AD7A339A84B002013
:10A6D800D4FC02086F1203384C250020245C0020AB
:10A6E80094240020DC360020D8220020E822002014
:10A6F800983000205304E9380F506E3A6F1203392E
:10A708006F12833A70B5244924480A784B78CD7B78
:10A718002349244EC2EB0214C2EB840203EB430428
:10A72800002D03EB8403204D204C01EB430300EB89
:10A73800420214BF2821202133602A6021601DF0C5
:10A74800E3F9302200211A481A4C23F072FC2868D9
:10A758001BF0DEF81DF026F9174A184B1079184A35
:10A76800C4F8A0206421C82211FB00210022C3E9FB
:10A778000112C3E90322C3E90522DA6183F8202024
:10A7880083F8212018F0BEF994F8A610B4F8A400B4
:10A79800BDE870401BF0E4BF245C0020E8220020E4
:10A7A80094240020DC360020D822002098060020BF
:10A7B8001017002040110020B4390020A4250020E3
:10A7C800502A00200C290ED8DFE801F01B0D0D0DD2
:10A7D800140D0D0D0E0D0D0D0700C36923F4006354
:10A7E80043EA0222C2617047C36923F008031A438F
:10A7F800C2617047836923F4006343EA02228261DD
:10A808007047836923F008031A4382617047F0B4E4
:10A818000C292BD8DFE801F0752A2A2A502A2A2A7F
:10A828002C2A2A2A0700046AB2F80CC097881668EE
:10A838006A4D24F480540462036A4468C16923F4AD
:10A84800005343EA0C3321F4E641A84243EA0733B4
:10A8580041EA062100F0BC8005F50065A84200F039
:10A86800B78092684460C16102640362F0BC7047BB
:10A87800046AB2F80CC097881668584D24F480749E
:10A888000462036A4468C16923F4007343EA0C2331
:10A8980021F07301A84243EA072341EA060100F0C8
:10A8A800848005F50065A8427FD092684460C16144
:10A8B800F0BCC26303627047046AB2F80CC09788A0
:10A8C8001668464D24F010040462036A44688169DE
:10A8D80023F0200321F0807143EA0C1321F4E641B0
:10A8E800A84243EA071341EA06214BD005F5006563
:10A8F800A84247D0926844608161F0BC82630362D9
:10A908007047046A9389B2F804C01768334E24F07C
:10A9180001040462046A4568816921F4803124F0E5
:10A92800020443EA0C0321F07301B04243EA040332
:10A9380041EA07010ED02A4CA0420BD004F540642E
:10A94800A04207D004F58064A04203D004F58064D7
:10A95800A04210D1D489168A578AB2F806C023F0CB
:10A968000803234325F4407523F0040346EA07044B
:10A978004CEA03032543926845608161F0BC426359
:10A9880003627047D589178AD68823F0800343EA83
:10A99800051324F44064558A23F0400344EA8704ED
:10A9A80043EA061344EA8504A4E7D589178AD688BA
:10A9B80023F4006343EA052324F44054558A23F41E
:10A9C800806344EA071443EA062344EA05146CE763
:10A9D800158A24F4804444EA851442E7002C014097
:10A9E800003401402DE9F84FA02200213148324CB3
:10A9F800DFF8DC90314D324E324FDFF8D88023F04B
:10AA080018FB314A3149DFF8D0C0DFF8D0E002F155
:10AA180090001368A3423DD0B3F1804F3CD0AB42C5
:10AA28003CD0B3423CD0BB423CD063453CD073459C
:10AA38003CD043453CD0DFF8A8A053450AD00AF5DE
:10AA4800806A534508BF092305D018329042E0D1E7
:10AA5800BDE8F88F082309EBC3034FF0010A1B79FF
:10AA680003F01F0B5B09022B0AFA0BFA08D0032B21
:10AA78000BD0012BE9D14B694AEA03034B61E4E7A8
:10AA88008B694AEA03038B61DFE7CB694AEA030370
:10AA9800CB61DAE70023DEE70123DCE70223DAE70C
:10AAA8000323D8E70423D6E70523D4E70623D2E710
:10AAB8000723D0E79C3B0020002C01400004004005
:10AAC8000008004000100040001F0308001002406A
:10AAD800281E0308004001400014004000340140D3
:10AAE800004401402DE9F8432E4D2A69EB6812EA2B
:10AAF800030826D02C4E4FF00047B8FA88F327FAFF
:10AB080003F2D2431B3B2A6108EA0208042B15D83A
:10AB1800DFE803F0352B22190300D6F89C30002B10
:10AB280037D1EB6A1FFA83F9D6F8984034B1236815
:10AB38002046494698476468002CF8D1B8F1000FC0
:10AB4800DBD1BDE8F883B06F696B036889B29847B9
:10AB5800B8F1000FD1D1F4E7F06FA96B036889B29F
:10AB68009847B8F1000FC8D1EBE7D6F88000E96B39
:10AB7800036889B29847B8F1000FBED1E1E7D6F86B
:10AB88008400296C036889B29847B8F1000FB4D1E2
:10AB9800D7E703F1FF3900231FFA89F9C6F89C307B
:10ABA800C2E700BF003401409C3B00202DE9F84378
:10ABB8002E4D2A69EB6812EA030826D02C4E4FF076
:10ABC8000047B8FA88F327FA03F2D2431B3B2A61FD
:10ABD80008EA0208042B15D8DFE803F0352B221900
:10ABE8000300D6F89C30002B37D1EB6A1FFA83F9A3
:10ABF800D6F8984034B12368204649469847646897
:10AC0800002CF8D1B8F1000FDBD1BDE8F883B06FA4
:10AC1800696B036889B29847B8F1000FD1D1F4E79E
:10AC2800F06FA96B036889B29847B8F1000FC8D1D3
:10AC3800EBE7D6F88000E96B036889B29847B8F16A
:10AC4800000FBED1E1E7D6F88400296C036889B209
:10AC58009847B8F1000FB4D1D7E703F1FF390023C3
:10AC68001FFA89F9C6F89C30C2E700BF00340140DA
:10AC78009C3B00202DE9F8432B4D2A69EB6812EA2A
:10AC8800030824D0294E4FF00047B8FA88F327FA72
:10AC980003F2D2431B3B2A6108EA0208042B13D8AB
:10ACA800DFE803F0322920170300736F002B34D13B
:10ACB800EB6A1FFA83F9346F34B12368204649469A
:10ACC80098476468002CF8D1B8F1000FDDD1BDE8D1
:10ACD800F883306D696B036889B29847B8F1000F43
:10ACE800D3D1F4E7706DA96B036889B29847B8F1BE
:10ACF800000FCAD1EBE7B06DE96B036889B29847DA
:10AD0800B8F1000FC1D1E2E7F06D296C036889B290
:10AD18009847B8F1000FB8D1D9E703F1FF390023FC
:10AD28001FFA89F97367C6E7000800409C3B0020BA
:10AD38002DE9F8432B4D2A69EB6812EA030824D061
:10AD4800294E4FF00047B8FA88F327FA03F2D243A6
:10AD58001B3B2A6108EA0208042B13D8DFE803F03A
:10AD6800322920170300F36C002B34D1EB6A1FFA49
:10AD780083F9B46C34B1236820464946984764681F
:10AD8800002CF8D1B8F1000FDDD1BDE8F883B06A26
:10AD9800696B036889B29847B8F1000FD3D1F4E71B
:10ADA800F06AA96B036889B29847B8F1000FCAD155
:10ADB800EBE7306BE96B036889B29847B8F1000F8D
:10ADC800C1D1E2E7706B296C036889B29847B8F182
:10ADD800000FB8D1D9E703F1FF3900231FFA89F929
:10ADE800F364C6E7000400409C3B00202DE9F843CB
:10ADF8004FF080452A69EB6812EA030824D0294EEF
:10AE08004FF00047B8FA88F327FA03F2D2431B3B06
:10AE18002A6108EA0208042B13D8DFE803F0322974
:10AE280020170300736A002B34D1EB6A1FFA83F9E9
:10AE3800346A34B123682046494698476468002C30
:10AE4800F8D1B8F1000FDDD1BDE8F8833068696B3F
:10AE5800036889B29847B8F1000FD3D1F4E7706856
:10AE6800A96B036889B29847B8F1000FCAD1EBE71C
:10AE7800B068E96B036889B29847B8F1000FC1D18F
:10AE8800E2E7F068296C036889B29847B8F1000FC7
:10AE9800B8D1D9E703F1FF3900231FFA89F97362A2
:10AEA800C6E700BF9C3B00201F4B98422CD0B0F156
:10AEB800804F2BD0A3F59433984229D003F58063B3
:10AEC800984227D003F50063984225D003F58063A4
:10AED800984223D003F59033984221D003F540637C
:10AEE80098421FD003F58063984207D003F580632A
:10AEF800984208BF092202D00020704708220B4B55
:10AF080003EBC203187970470022F8E70122F6E73D
:10AF18000222F4E70322F2E70422F0E70522EEE733
:10AF28000622ECE70722EAE7002C0140281E030866
:10AF380070B4104E002332461D46042403E001334A
:10AF4800062B0CD0947930EA040402F11802F6D1E9
:10AF5800A94207D001330135062BEDB2F2D100200A
:10AF680070BC704703EB430306EBC30370BC18794E
:10AF7800704700BF001F030810B40E4C282122465A
:10AF880088424FF0000302F1180207D00133062B64
:10AF98000BD01179884202F11802F7D103EB430371
:10AFA80004EBC3005DF8044B704700205DF8044BC8
:10AFB800704700BF001F03082DE9F041C44A137809
:10AFC800A3F11701022905D9C24911F83300002855
:10AFD80040F09E81C04CC14F94F808C0C04E00217B
:10AFE800084637F83020530803F077334FEA9208C1
:10AFF80008F03338D31A4FEAD20EA3EB08030EF049
:10B00800113EA3EB0E0303EB231303F00F33A6FB50
:10B01800038E4FEADE1E12F00105CEEB0E2E18BF8E
:10B028000131A3EB0E0E18BFC9B2BEF1010F0ADD44
:10B03800BEF1020F40F02381002D00F0178112F4B9
:10B048002F7F00F01381002800F03981013902298F
:10B0580000F21581A34D8020F8F77AFB4FF06408C1
:10B068002B4605F5B17E4FF0000C9A88D98891429D
:10B07800B3F86210B3F8642028BFA3F804C0914263
:10B0880093F8732088BFA3F862C0013A632A93F843
:10B09800742088BF83F873800132D2B2092A88BF2E
:10B0A80083F874C003F16D00194600228E7A10F8F7
:10B0B800017F0132B74228BF80F800C0032A01F19E
:10B0C8000601F3D176337345CFD1874EB378042B7D
:10B0D80000F0278133B93388B3F5F07F84BF4FF48C
:10B0E800F0733380814EFFF735FA3368804A1A408F
:10B0F800002A00F06481D90700F13C815A0400F16C
:10B108001E811F0700F12281980100F12681990410
:10B1180000F12B811A0440F1D4800023E37384F8F2
:10B1280023301CF0E3FC002800F0AD80637E032B85
:10B1380000F0A9805A1E012A40F2BC8000232B830C
:10B14800A5F88E30A5F804311CF0D0FC002840F09A
:10B15800B080002385F84F3085F8C53085F83B313D
:10B16800644BDA79022A08BF01224FF0070008BFB2
:10B17800DA711CF039FA002840F009814FF4806038
:10B18800FEF7CEFA002800F00C815B4E344604F13D
:10B198007D057836617979B1207858B1574B02E04E
:10B1A80006339D4208D013F8052C8A42F8D11A7844
:10B1B800002AF5D01CF0BEF90634A642EAD1402098
:10B1C800F8F7C6FA4FF40070F8F7C2FA4FF40050D7
:10B1D800F8F7BEFA4FF48040F8F7BAFA4FF40030A7
:10B1E800F8F7B6FA4648474CF8F7B2FA4FF40010A9
:10B1F800F8F7AEFA4FF08060F8F7AAFAA388002BA8
:10B2080040F0BD80404A136813F07F4F1CBF0023F5
:10B218001360936823F4007323F002030BB1002337
:10B2280093601379013B042B84BF01231371374BBF
:10B23800B3F86E2002F00F01022903D8C2F30312FB
:10B24800012A03D94FF42062A3F86E20B3F87020C6
:10B2580002F00F01022903D8C2F30312012A03D90D
:10B2680040F60122A3F87020BDE8F081550606D506
:10B2780012F4057F03D0BCF1070F7FF6E4AE174840
:10B28800FDF7C9F9E6E60023AB816B82A5F88230A9
:10B29800A5F88830A5F8F830A5F8FE301CF026FC93
:10B2A80000283FF44BAF637E5A1E012A3FF646AF93
:10B2B80000E0637E023B022B3FF64BAF50E70120D4
:10B2C8008FE6E27B002A71D0002384F8233028E738
:10B2D800043A0020CC1F0308E4590020225900201A
:10B2E80081808080E8220020A84B0020904A00201E
:10B2F80009600002B43900203C34002041340020A9
:10B3080020001000441A0020681A0020581D002050
:10B3180001EBC3035B68002B7FF45CAE172313704B
:10B3280058E64FF48050F8F713FAF38AB3F57A7FAA
:10B3380037BF4FF47A72B378B378F282CAE62248FC
:10B34800F8F706FA33681F077FF5DEAE1F48F8F7EF
:10B35800FFF9336898017FF5DAAE46F20900F8F78D
:10B36800F7F9336899047FF5D5AE1948F8F7F0F97D
:10B378003368CFE61748F8F7EBF93368BEE620786C
:10B38800FFF7FAFD00287FF43DAFA0803AE70720D9
:10B398001CF0D0F84FF48060FEF7C2F900287FF463
:10B3A800F4AE4FF00060F8F7D3F9EEE642F201028E
:10B3B80013423FF4B6AE002384F82330B1E643F0DD
:10B3C8000073336097E600BF0920000201600002A5
:10B3D80009400002086000022DE9F04F8DB0FFF728
:10B3E800EBFDDFF894915B4FDFF8908118F006F9D8
:10B3F800594A5A4BB2F86421ADF80620A3EB090369
:10B4080000934FF0030A0026CDE90866CDE90A66E5
:10B41800009BCDF818900793D8F810301B0606D576
:10B428004F4BC8F8043003F18833C8F804300123BF
:10B438008DF82C303423C8F80C300222BDF80630C1
:10B44800ADF8083002A906A8F8F7E4F9022202A923
:10B458004FF6FF70F8F71DFD424BBB42834629D2D9
:10B468001C46658823888DF81560C5F30B05C3F362
:10B478000B00A91D1B0B0622ADF81010ADF8120029
:10B4880004A906A88DF81430F8F7C4F9584606221E
:10B4980004A9F8F7FEFC616883462A4606A8F8F76F
:10B4A800B9F9616858462A46F8F7F3FC1434BC42E7
:10B4B8008346D6D3022203A906A8ADF80C60F8F794
:10B4C800A9F9022203A95846F8F7E3FC40BAC34396
:10B4D800022204A906A8ADF81030F8F79BF90998DC
:10B4E80050BB0A989DF82C308BB9C0B1BAF1010A4B
:10B4F8008AD105201EF066F81B491C4B1C481D4AC2
:10B508000860DA6018F05AF80DB0BDE8F08FD8F886
:10B51800103043F08003C8F810300028E6D199F8BD
:10B528000030AC2BE5D199F80130BE2BE1D1F8F70A
:10B53800CAFC0028E6D1DCE708ABC0F10402002110
:10B54800184422F076FD089906A8F8F709F9CDE91C
:10B558000960C7E74C700308D4FC0208000004081F
:10B5680023016745EC6B0308FC9F002000ED00E019
:10B57800EFBEADDE0400FA0500F00308002002402B
:10B5880008B5FBF77DFAFFF727FFBDE80840FFF78E
:10B59800B9B8014B18601FE7904A00202DE9F84F11
:10B5A80018F02CF82B4B2C4A934250D22B4F03F116
:10B5B80014069B464FF00108294C258862197DB175
:10B5C800BA420DD2052D0BD936F8143C6188C3F365
:10B5D8000B0399420AD0144625886219002DEFD131
:10B5E80056F8101C5846FBF729FA0FE0637913F058
:10B5F800030AF0D156F8101C94F804905846FBF74B
:10B608001DFA36F8141CB9EB113F11D04FF00008A1
:10B61800114B0BF1140B9B4506F11406CCD3FFF725
:10B62800CBFCFFF76FF817F0C9FF4046BDE8F88F6D
:10B6380036F8123C56F8100CAA1FC3F30B039A42B3
:10B6480004F10601A8BF1A4622F0CFFCE0E74FF04C
:10B658000108E4E7EC6B03084C70030800000408D9
:10B6680002F003082DE9F04F85B0CDE902109B4D9B
:10B67800DFF878A2029B013B0293013300F02A8194
:10B688001DF018FE964C974FDFF864E2964E4FF483
:10B69800FA7301934FF01008DEF80430C3F308037F
:10B6A800002B40F0F680EFF31183002B40F0F1807F
:10B6B8002068AA6823689842FAD133689A42F7D872
:10B6C800D7F800C04FF47A7101FB0CF39B1AB3FB57
:10B6D800FCF301FB00304FF47A7C4FF00109DEF8EF
:10B6E8000430C3F30803002B40F0B580EFF3118357
:10B6F800002B40F0B0802368A96822689342FAD1F1
:10B7080032689142F7D83A680CFB02FBABEB0101B7
:10B71800B1FBF2F10CFB03131B1AB3F57A7FDED3EE
:10B72800019B013B0193B7D1039B6F4E581CC0B2DC
:10B738001DF02CFCDFF8B8E14FF47A730193DEF8C2
:10B748000430C3F308034FF01008002B44D1EFF383
:10B758001183002B40D12068AA6823689842FAD147
:10B7680033689A42F7D8D7F800C04FF47A7101FBD2
:10B778000CF39B1AB3FBFCF301FB00304FF47A7C0B
:10B788004FF00109DEF80430C3F30803002B44D15D
:10B79800EFF31183002B40D12368A96822689342F4
:10B7A800FAD132689142F7D83A680CFB02FBABEB4E
:10B7B8000101B1FBF2F10CFB03131B1AB3F57A7FFD
:10B7C800E0D3019B013B01933FF454AFDEF8043012
:10B7D800C3F30803002BBAD0EFF3118388F3128860
:10B7E800D5F808C02A68D20304D50122CAF8002077
:10B7F800D5F808C02068DAF80090DBB283F3118826
:10B8080039684FF47A72484402FB01F3A3EB0C0346
:10B81800B3FBF1F302FB0030B0E7EFF3118188F3DB
:10B828001288D5F808B02B68DB0344BFCAF800902B
:10B83800D5F808B02368DAF80020C9B281F3118876
:10B84800396813440CFB01F2A2EB0B02B2FBF1F2D4
:10B858000CFB0323B1E7EFF3118188F31288D5F8C5
:10B8680008B02B68DB0344BFCAF80090D5F808B0CD
:10B878002368DAF80020C9B281F3118839681344C3
:10B888000CFB01F2A2EB0B02B2FBF1F20CFB03235F
:10B8980042E7EFF3118388F31288D5F808C02A68C5
:10B8A800D20304D50122CAF80020D5F808C02068C0
:10B8B800DAF80090DBB283F3118839684FF47A72B2
:10B8C800484402FB01F3A3EB0C03B3FBF1F302FBC7
:10B8D800003000E705B0BDE8F08F00BF10E000E0E1
:10B8E800603D0020703D0020743D00206C3D00202C
:10B8F80000ED00E0224B5B68C3F3080330B4D3B912
:10B90800EFF31183BBB91F4A1F4D204813688468A1
:10B9180011688B42FAD129688C42F7D81C4A116801
:10B928004FF47A7202FB01F0001B30BCB0FBF1F05F
:10B9380002FB03007047EFF31182102383F3128890
:10B9480003F1E023D2B29C68196811F4803F1149D1
:10B958001EBF012008609C680A4B18680B6882F3B8
:10B9680011880B4A11684FF47A72034402FB01F004
:10B97800001B30BCB0FBF1F002FB0300704700BFB6
:10B9880000ED00E0603D0020743D002010E000E084
:10B99800703D00206C3D002008B50E4B1978012938
:10B9A80013D00DD3022902D10020F6F718FCFFF7B7
:10B9B800A1FF094B00F5F42000F59070186008BD50
:10B9C80000210846F6F74AFCF1E70020F6F746FCA6
:10B9D800EDE700BF60140020641400202DE9F84F43
:10B9E8008046274C274DDFF8A490274EFFF782FFAB
:10B9F800DFF89CE0DFF89CC04FF0100A4FF47A772C
:10BA0800DCF80430C3F30803CBB9EFF31183B3B9FF
:10BA18002368A96822689342FAD132689142F7D81C
:10BA2800DEF8002007FB02FBABEB0101B1FBF2F1F2
:10BA380007FB03131B1A4345E2D3BDE8F88FEFF366
:10BA480011818AF31288D5F808B02B68DB0304D576
:10BA58000123C9F80030D5F808B02368D9F80020C8
:10BA6800C9B281F31188DEF80010134407FB01F214
:10BA7800A2EB0B02B2FBF1F207FB0323DAE700BFEC
:10BA8800603D002010E000E0743D00206C3D002087
:10BA9800703D002000ED00E02DE9F04FDFF834C1E3
:10BAA800494CDFF834E1DFF83481484E8246484893
:10BAB8001AF1FF3AC0F08680DCF80430C3F30803BB
:10BAC800002B5ED1EFF31183002B5AD10568A268D1
:10BAD80003689D42FAD133689A42F7D8DEF80070BD
:10BAE8004FF47A7101FB07F39B1AB3FBF7F301FBE1
:10BAF8000535DCF80430C3F308034FF010094FF4A0
:10BB08007A77F3B9EFF31183DBB90368A1680268A8
:10BB18009342FAD132689142F7D8DEF8002007FB49
:10BB280002FBABEB0101B1FBF2F107FB03135B1B5B
:10BB3800B3F57A7FBCD2DCF80430C3F30803002BDA
:10BB4800E0D0EFF3118189F31288D4F808B02368A4
:10BB5800DB0304D50123C8F80030D4F808B0036823
:10BB6800D8F80020C9B281F31188DEF80010134418
:10BB780007FB01F2A2EB0B02B2FBF1F207FB032376
:10BB8800D5E7EFF31183102282F31288A1682268A7
:10BB9800D20303D50122C8F80020A168D0F800908C
:10BBA800D8F80050DBB283F31188DEF800704FF448
:10BBB8007A724D4402FB07F35B1AB3FBF7F302FBFF
:10BBC800053596E7BDE8F08F10E000E0743D0020F1
:10BBD800603D002000ED00E0703D00206C3D00203D
:10BBE80010B504462046F5F757FD00B110BD0A20F0
:10BBF800FFF752FFF6E730B4EFF31183102282F318
:10BC08001288084808490268084D094C0132026048
:10BC18008A682A6000222260DBB20A6883F31188EE
:10BC280030BC7047603D002010E000E0743D00200B
:10BC38006C3D00200E4B1B88014643B90D4B0E4A44
:10BC48001B7810680BB981F00101F6F7D9BA0B4BD4
:10BC58005A691AB11A6810B91060587470470848C0
:10BC68000849008891FBF0F1012011605874704771
:10BC78002C3F00202E3F0020303F0020343F002082
:10BC88004C3F002020A1070010B50020FFF7D2FF8D
:10BC9800074B084A00241C701470FFF77DFE064B02
:10BCA800C3F8A840A3F8AC40C3F8B04010BD00BF2B
:10BCB800601400205E2A00204011002098B31B4B1E
:10BCC8001B6813F4003327D101229042184908D089
:10BCD8000133192B03EB430226D011F8222090429E
:10BCE800F6D1144A30B4D2F8B04059003CB11248E9
:10BCF8006478CD1800EB8500407FA0420AD20C483A
:10BD08000B4400EB83030021C2F8B030A2F8AC105A
:10BD1800C2F8A81030BC7047084B1B78032B02D020
:10BD280001220023D1E7AFE7704700BF681A00205F
:10BD3800F0FC020840110020D4FC02087E250020F7
:10BD48002DE9F04706460B201BF026FEF0B9464CBD
:10BD5800D4F8B050C5B1D4F8A830B34214D8DFF83D
:10BD68002C8198F800304BB3B4F8AC706B68DB5D8D
:10BD7800B9467BB9002342F21072013702FB036611
:10BD8800A4F8AC70C4F8A860BDE8F0870A20FFF7F3
:10BD980095FFDCE70020FFF74DFF344A00231370BE
:10BDA80088F80030FFF7F8FD6B6813F80930FE2BB0
:10BDB8004ED10023A4F8AC30BDE8F0871AF0ECFAB5
:10BDC800D8B92B780A2B38D0022B16D1284A936879
:10BDD8009B0712D4274B28491B68F31A8B420CD9AE
:10BDE800264B1B684BB92648264906601279097804
:10BDF800FF2009F097F9D4F8B050B4F8AC706B682C
:10BE0800DB5DB946002BB5D02B78194A013B4FF0C2
:10BE1800010A12680AFA03F3134213D0134B0122E2
:10BE28001A70FFF7B9FD002FBED12B785A1F012ACF
:10BE380013D9182B11D0B946B6E70D4A936899055E
:10BE4800C8D5DAE75046FFF7F5FE88F800A0E5E721
:10BE5800FF2B90D1BDE8F04716E7FFF74BFD0A4BE3
:10BE68004FF0000918609FE740110020601400207F
:10BE7800681A002068140020804F12003C2A002015
:10BE8800402A002020590020E03300205E2A0020AC
:10BE980040004028094A30B4A8BF402000230225AA
:10BEA8001424D5540233D118834201F8014CF8D335
:10BEB800FF21D1540E2030BC00E700BF3C15002004
:10BEC80008B5FFF789FAFFF769FB0120BDE80840CC
:10BED800DEE7022838B504460FD8C0EB0013094A3C
:10BEE80009490A4D0C70C0EB830302EB4303184663
:10BEF8002B6019F00DFD1AF05BF9601CC0B2BDE8AB
:10BF08003840C5E7E8220020245C0020D822002021
:10BF18002DE9F047B0F908500D81EDB2382D96B0F3
:10BF28000C4600F014830646174645D9812D00F0CB
:10BF3800FA8000F28D80542D00F0648140F2DF8198
:10BF48006E2D00F0B582802D40F0DB819D4B1F786F
:10BF5800023717F0FF0700F090809B4EDFF87882D9
:10BF6800DFF894A2DFF8949237440A25013616E0E8
:10BF7800322D00F07383A5F13C00C0B2132840F2C3
:10BF8800A98300232268511C216015702268B742DA
:10BF980002F10101216013706FD016F8015B0A2DC0
:10BFA800E6D1B9F800300533A8FB0323DB08FF2BE3
:10BFB800A8BFFF23DBB2E5E7042D00F0EE8240F2D4
:10BFC8000982202D60D040F25582242D00F067822E
:10BFD800282D40F096810B68DFF824827B4E591C8F
:10BFE800022221601A70236806275A1C22601F70DB
:10BFF80023680A22591C21601A70236801255A19DE
:10C0080022601D70B8F800102046F7F764FCB8F8F5
:10C0180002102046F7F75FFC23685A1922601F7048
:10C0280023685022591921601A702368002259196F
:10C0380021601A7031882046F7F74DFC7188204638
:10C04800F7F749FC2B462846A38116B0BDE8F087D0
:10C05800A02D56D040F2D581B82D00F06782FE2D74
:10C0680040F04F815A4D05F1080635F9021B20466C
:10C0780089B2F7F730FCAE42F7D101252B462846A6
:10C08800A38116B0BDE8F087524D53496A882368EA
:10C098000532A1FB0202C2F3C702581C20601A70C5
:10C0A8002A8823680532A1FB0202C2F3C702581C82
:10C0B80020601A70AB8822680533A1FB0313C3F311
:10C0C800C703511C21601370A9892046F7F703FCA8
:10C0D80023686A7A591C21601A702368AA7A591C45
:10C0E80021601A7069882046F7F7F5FB29882046F1
:10C0F800F7F7F1FBA98820460125F7F7ECFB2B465B
:10C10800A1E7364B08461968F7F7CEFB344B2046B3
:10C118001968F7F7C9FB334B204619680125F7F76B
:10C12800C3FB2B468FE7274B1E78033616F0FF0616
:10C13800A3D02D4B2D4F1E4403F101094FF00A08DF
:10C1480020E0B8F1500F00F08C82B8F1320F00F007
:10C15800CC82A8F13C00C0B2132840F2E08200254E
:10C16800294623685A1C2260204683F80080F7F786
:10C17800B2FB29462046F7F7AEFB4E453FF47DAFAC
:10C1880019F8018BB8F10A0FDBD1194B19499D68D1
:10C198001A68087805EB85054FF6FF716D008D422A
:10C1A800A8BF0D469142A8BF114625EAE57521EAC8
:10C1B800E1712328ADB289B2D3D10548DB68838009
:10C1C800C280CEE7205900203CFE0208AC220020A5
:10C1D800B41C0020401D0020CDCCCCCCACF7FF1FF8
:10C1E800B0F7FF1FB4F7FF1F4CFE020854140020DD
:10C1F800CC130020B01C0020B0130020BC1300207A
:10C20800A42200200B68BD4ABD4F581C1121206094
:10C21800197023681278591C21601A70236897F8DE
:10C228006D20591C21601A70236897F86C20591CDE
:10C2380021601A70B7F868102046F7F74CFB23689E
:10C248000022591C21601A7023683422591C21606D
:10C258001A70B7F86A102046F7F73DFBBD1E07F1C4
:10C26800660635F8021F2046F7F735FBAE42F8D1CF
:10C2780022681421531C2360012500231170F96FD3
:10C28800226805FA03F0084203F1010314BF0121F3
:10C298000021501C142B20601170F0D12368022259
:10C2A800591C21601A70B7F86E102046F7F713FB77
:10C2B800B7F870102046F7F70EFBB7F87410204651
:10C2C800F7F709FB23680D22591C21601A70796F52
:10C2D8002046F7F7E9FA23685A1C22601D70236884
:10C2E8005A1C22601D7022680125531C23600021FE
:10C2F8002B4628461170A38116B0BDE8F087522D51
:10C30800F1D021462846FCF7C1F900287FF4B5AEE4
:10C31800742DD6E9008300F00E8240F2EC81772D6F
:10C3280000F08A81E62D40F0B181434500F0F682A5
:10C33800D4E9002CACEB0202029303930546571E86
:10C3480043460022974203F1010E06A902A81ADD0E
:10C35800C6F800E093F800E02368ADF810E0CDE9F6
:10C36800063CFFF7D5FD2268069BD4F804C09B1A4B
:10C37800013303F0FF03FF1AD6E900325CBF013531
:10C38800EDB29A42DDD1C6F80080CDF81CC027680E
:10C39800E5B14FF00008C14607F1010ACDF818A031
:10C3A80087F8009033685A1C32601B78ADF810305B
:10C3B800002206A902A8FFF7ABFD069B08F10108B9
:10C3C800A3EB0A033B704545069FE5D1012527608D
:10C3D8002B4638E6022D00F0278100F21481012D4A
:10C3E8008FD10B680022591C21601A7023685A1CCF
:10C3F80022601D7022682921531C23602B4611706E
:10C4080021E6822D7FF47DAF0B683E4A3E4D1178C0
:10C418003E4A3F4E581C2060197091892046F7F714
:10C428005AFA2B883B4922680533A1FB0313DB0822
:10C43800FF2B02F10101A8BFFF2321601370B1682F
:10C4480081F3100189B22046F7F745FA316801F304
:10C458000F0189B22046F7F73EFA23682E4A591C85
:10C46800127821601A70298820460125F7F733FAD7
:10C478002B4604E6052D7FF444AF0B2227492046BE
:10C48800F7F708FA082226492046F7F703FA0125A4
:10C49800072224492046F7F7FDF92B46D3E5224B1E
:10C4A80093F8B420002A00F0D680D3F8B81048E0FA
:10C4B800154D18492B882268154E0533A1FB031327
:10C4C800DB08FF2B02F10101A8BFFF2321601370D5
:10C4D800B16881F3100189B22046F7F7FCF916F02C
:10C4E8000BFD01462046F7F7F6F9316801F30F0115
:10C4F80089B22046F7F7EFF9B5E700BF9843002067
:10C50800581D00207F25002078250020401D002090
:10C5180068250020CDCCCCCC7E25002034510308E2
:10C52800405103084C51030840110020B74D0846FC
:10C538002968F7F7B9F923682A79591C21601A7014
:10C54800A96820460125F7F7AFF92B4697E50A6851
:10C55800AF4B0125511C2160157022680521501927
:10C568002060117022680A21501920601170226819
:10C578000021501920601170226819785019206024
:10C5880011702268597850192060117022689978C2
:10C59800531923602B46117055E52A469D492046BC
:10C5A800F7F778F900212046F7F795F923689A49B3
:10C5B8005A1C022622601E70236801255A1922601F
:10C5C8001D7023680C205A192260024618702046F4
:10C5D800F7F760F922680023511921601370226867
:10C5E8005119216006A819461370202221F021FD57
:10C5F800202206A92046F7F74DF92268531923602F
:10C608002B4616701FE50B6804215A1C226019700E
:10C6180023680022581C20601A70226801255319CB
:10C6280023602B4611700EE504227C492046012523
:10C63800F7F730F92B4606E543451BBF08F1010320
:10C648003360014698F80010754A204601250CF021
:10C6580057F92B46F7E4734B196872E7BAF80030BC
:10C66800A1E4714A9568116805EB85056D004FF6E0
:10C67800FF739D42A8BF1D469942A8BF194625EAE7
:10C68800E57521EAE171ADB289B26AE5F52D61D0AF
:10C69800392D00F0A58100F2D980212D00F06281AA
:10C6A800292D40F0BD8108F10103336098F800306E
:10C6B8000A2B01F02C81502B41F02F813046F7F7DF
:10C6C800D9F85A4F38803046F7F7D4F801257880E2
:10C6D8002B46B8E410F0A4FE00283FF452AC0378CF
:10C6E8000A2B3FF64EAC43885DE4D7E9001303EB11
:10C6F80083035D00BBE7442DC8D1434540F0048166
:10C708004B4B024618712368591C21601A70002F80
:10C718003FF4B3AC474B3B6001252B4693E410F044
:10C728007FFE00283FF41BAD03780A2B3FF617ADB8
:10C73800D0E90131DBE743451BBF08F10103336052
:10C74800014698F800103C4A204601250CF0D8F81C
:10C758002B4678E4434541F0B480354BFF2283F8FB
:10C76800BC204FF00009354D09F076F949462022E2
:10C77800334885F8009021F05CFC8DF818909DF8FE
:10C788001830072B01F24181DFF8BC802C4E4A4655
:10C798009DF8183003EB430308EBC3035B7CFBB144
:10C7A8009DF8183003EB430308EBC3035B69BBB187
:10C7B8009DF8183003EB430308EBC30320215B69A2
:10C7C80046F82230184623B1F4F77AFF2B7856F84A
:10C7D80023301846F5F70FFD2A780132D2B22A70B5
:10C7E8009DF818300133DBB28DF818309DF81830F9
:10C7F800072BCDD92368591C21601A70002F3FF4EC
:10C808003CAC104B3B6001252B461CE4681A002009
:10C81800A02200202B5C0020245103081C5103088F
:10C8280019F80008904A0020E4130020AC220020E8
:10C838004011002059860008D9FF00084D3000201B
:10C848001C300020390F0208E84A0020552D6AD014
:10C85800572D40F0E58008F10103336018F8377B65
:10C868000DF117020133336013F8011C02F8011FA0
:10C878004345F7D1DFF8A08198F80050002DFDD18D
:10C88800DFF8989101260421484688F80060F5F7FA
:10C8980073FED9F80800F5F7A9FC5B4B2946284632
:10C8A8001E70FBF737F939460920FBF733F906AE56
:10C8B80035460DF14E07A91BC9B20A20FBF72AF924
:10C8C80015F8011B0B20FBF725F90020F5F787FC6D
:10C8D800AF42F0D1A0210820FBF71CF90021A020CD
:10C8E800FBF718F910F02006F8D1D9F80800F5F789
:10C8F80082FC0125D9F804000221F5F763FE88F8C7
:10C9080000602B46FFF79FBB08F10103336098F8DE
:10C9180000203E4B012A1A717FF6F5AE4FF0FF3525
:10C928002B46FFF790BB08F10103336098F80070BD
:10C93800FF2F01F02780FE2F00F0F9873046F6F729
:10C9480099FFD6E90032D21A002A01F30580332F65
:10C95800E4D82F4B012523F8170010F0D2FF2B46FF
:10C96800FFF771BB424608F10103336012F8023B3E
:10C97800284F03EB83035B007B80326098F801301B
:10C9880003EB830308F103025B003B80326098F8F5
:10C99800023003EB83035B003046BB80F6F76AFF87
:10C9A8003268B8811346511C316013F8021B797242
:10C9B80033605278BA727268D31A052B7FF75DAB71
:10C9C8003046F6F757FF78803046F6F753FF388041
:10C9D8003046F6F74FFF0125B8802B46FFF733BBEB
:10C9E80008F10103336098F800300A2B00F07887CB
:10C9F8003046F6F74AFF3046F6F747FF3046F6F777
:10CA080044FFFFF73ABB00BF502700204011002029
:10CA1800581D0020401D00204F27002058430020AB
:10CA28000B3DA3EB0802EF2D3FF678AF01A151F8BB
:10CA380025F000BF7DD8000825C9000825C90008D1
:10CA480025C9000825C9000825C9000825C9000806
:10CA580025C9000825C9000825C9000825C90008F6
:10CA680025C9000825C9000825C9000825C90008E6
:10CA780025C9000825C9000825C9000825C90008D6
:10CA880025C9000825C9000825C9000825C90008C6
:10CA980025C90008F5D7000825C90008A7D8000847
:10CAA80025C900086FD6000825C9000825C900084F
:10CAB80025C9000857D7000825C9000891D60008DD
:10CAC80025C9000825C9000825C9000887D7000816
:10CAD80025C90008E5D0000825C900081DD30008AD
:10CAE80025C90008A3D2000825C9000825C90008DF
:10CAF80025C9000825C9000883C0000825C9000801
:10CB080049D2000825C9000825C9000829D200080B
:10CB180025C9000825C9000825C9000825C9000835
:10CB280025C9000825C9000825C9000825C9000825
:10CB380025C9000825C90008E5D1000825C900084D
:10CB480093D1000825C9000825C9000851D100085B
:10CB580025C9000825C9000825C9000825C90008F5
:10CB680025C9000825C9000825C900085BD50008A3
:10CB780025C90008EDD4000825C9000869D40008B3
:10CB880025C9000895D3000825C900082BD6000838
:10CB980025C90008E7D5000825C9000825C90008E7
:10CBA80025C9000825C9000825C9000825C90008A5
:10CBB80025C9000825C9000825C9000825C9000895
:10CBC80025C9000825C9000825C9000825C9000885
:10CBD80025C9000825C9000825C9000825C9000875
:10CBE80025C9000825C9000825C9000825C9000865
:10CBF80025C9000825C9000825C9000825C9000855
:10CC080025C9000825C9000825C9000825C9000844
:10CC180025C9000825C9000825C9000825C9000834
:10CC280025C9000825C9000825C9000825C9000824
:10CC380025C9000825C9000825C9000825C9000814
:10CC480025C9000825C9000825C9000825C9000804
:10CC580025C9000825C9000825C9000825C90008F4
:10CC680025C9000825C9000825C9000825C90008E4
:10CC780025C9000825C9000825C9000825C90008D4
:10CC880025C9000825C9000825C9000825C90008C4
:10CC980025C9000825C9000825C9000825C90008B4
:10CCA80025C9000825C9000825C9000825C90008A4
:10CCB80025C9000825C9000825C9000825C9000894
:10CCC80025C9000825C9000825C9000825C9000884
:10CCD80025C9000825C9000825C9000825C9000874
:10CCE80025C900083DD6000825C90008B3D00008AA
:10CCF80085D0000825C9000825C9000825C90008ED
:10CD080025C9000825C9000825C9000825C9000843
:10CD180025C9000825C9000825C9000825C9000833
:10CD280025C9000825C9000883C0000825C90008CE
:10CD38004BD0000825C900089DCF000883CF000804
:10CD480067CF000825C900084DCF000825C900088D
:10CD580021CF000825C9000883C0000825C900089C
:10CD680093CE000825C9000825C900087FCE000811
:10CD7800B9CE00086BCE000839CE000825C90008D6
:10CD880017CE000825C9000825C9000825C90008CC
:10CD980025C9000825C9000825C9000825C90008B3
:10CDA80025C9000825C9000825C9000825C90008A3
:10CDB80025C9000825C9000825C9000825C9000893
:10CDC80025C90008FDCD000825C9000825C90008A7
:10CDD80083C0000825C9000825C9000825C900081E
:10CDE800EFCE000825C9000825C9000825C9000894
:10CDF80079D200083046F6F73DFDBE4FB88130467F
:10CE0800F6F738FD012578812B46FFF71CB9304627
:10CE1800F6F730FDB84F78823046F6F72BFDB8822A
:10CE28003046F6F727FD0125F8822B46FFF70BB9A8
:10CE380008F101033360304698F80070F6F725FDD5
:10CE4800D6E900134A1C3260AC48097881709B1AF5
:10CE5800022B00F3FD87AA4B0125DF712B46FFF754
:10CE6800F2B8A84BA84918687622012521F0BDF828
:10CE78002B46FFF7E8B83046F6F7FCFCA34F38809E
:10CE88003046F6F7F7FC7880A2E5A14FDFF8B482C8
:10CE9800002506E0F6F7EEFC18F078FD0135A7EC62
:10CEA800010A98F800309D423046F3DBFFF7E5B8F9
:10CEB800424608F101033360964B12F8021B1970C1
:10CEC800326098F801205A7008F10302326098F82D
:10CED80002209A703046F6F7CDFC8C4B0125D8809D
:10CEE8002B46FFF7B0B83046F6F7ADFC054630469E
:10CEF800F6F7C0FC884E82B24FF47A71002330688E
:10CF0800C1FB0523121A854963F100030125C1E914
:10CF180030232B46FFF797B808F10103336098F8E0
:10CF28000000070600F19F877D4B1B78DE073FF561
:10CF3800A4A8032828BF00200125FEF7CAFF2B4616
:10CF4800FFF781B8764B1B78DD073FF596A80125DA
:10CF5800FEF716FBFEF722FB2B46FFF774B8704B63
:10CF68001B78D9073FF589A86E4A1378012543F045
:10CF7800040313702B46FFF766B8694B1B78D80774
:10CF88003FF57BA8684B4FF4C87201251A802B46E1
:10CF9800FFF759B8092A7FF7C1AC644F08F10103BC
:10CFA8003D6833602979EA7898F80030EB7091424F
:10CFB80008F1020208BF2B713260E979AA7998F862
:10CFC8000130AB71914208BFEB7105F1090205F11F
:10CFD8000C013368581C3060187802F8010B914234
:10CFE800F7D19A1C32605A78642AA8BF6422D91CE7
:10CFF8002A7331609A782A701A1D3260DB786B7058
:10D008003046F6F737FCD6E90083A3EB0802002A7E
:10D01800E88100F31A85A3EB0803012B0BDD4346D7
:10D0280008F101013A68316013F8021B117433608A
:10D0380098F80130537401251AF066FD2B46FFF766
:10D0480002B8304B1868034600F11E01424608F149
:10D058000105356012F8025B1D72326098F80120F4
:10D068005A7208F10302326098F802209A72063365
:10D07800994200F0D781D6F80080E7E708F101036C
:10D088002B4933600A7898F80030002A40F0C784AA
:10D0980004220A70274A9B001380FEF72BFC264BBC
:10D0A800012518602B46FEF7CEBF3046F6F7CBFBBE
:10D0B800D6E90083214FA3EB0802002A386000F369
:10D0C800BA84A3EB0803032B7EF7D7AF3046F6F7F5
:10D0D800BAFB0125B8602B46FEF7B5BF08F101037E
:10D0E8003360174B98F80020DA7301252B46FEF7BA
:10D0F800AABF00BF4C2A0020A84B0020403B0020BC
:10D10800B4300020D8220020E81B0308243900206E
:10D11800F8370020A0300020603D0020401100209A
:10D12800231E0020241E00205E140020DC36002070
:10D138007C2F0020A42F002084150020681A0020CE
:10D14800E459002020590020B84A1278012A3EF6F6
:10D1580094AF414608F101023260B54F11F8022B35
:10D16800BA7008F1030231609B1A98F80100326026
:10D17800012B98F8021040F373853046F6F77AFBD6
:10D18800012538802B46FEF75EBF08F101033360A6
:10D1980098F80070112F3FF6C1AB08F10203336015
:10D1A800A44D98F8013005F817303046F6F762FBC1
:10D1B80040F6CA039842A8BF184640F2EE2305EB92
:10D1C80047019842B8BF184601251923A0F2EE225C
:10D1D80092FBF3F22B464A70FEF735BF434608F13F
:10D1E8000102954D326013F8022B2A71336098F8CA
:10D1F80001306B713046F6F73DFB336828805A1CC6
:10D2080032601B78AB713046F6F734FB33686880C0
:10D218005A1C32601B78EB7101252B46FEF713BFB1
:10D22800864B03F1080208F10101316098F80010FB
:10D2380003F8011F9A423EF420AFD6F80080F2E7C7
:10D2480008F1010333607E4B98F800205A7030468D
:10D25800F6F71BFBD6E900329A423EF40EAF5A1C91
:10D268003260784A1B78137101252B46FEF7EBBE16
:10D27800754B1B78DA073FF551AB744B93F8B42024
:10D28800002A00F0DE85D3F8B800FEF782F9012500
:10D29800FEF784F92B46FEF7D6BE0723B2FBF3F35D
:10D2A800C3EBC305521B7FF439ABDFF8B0915FFACB
:10D2B80083F8154609F1080A27E0336899F902103E
:10D2C8005A1C326093F90020914200F0BE8599F90A
:10D2D8000A3093427FF422AB5746BA703046F6F7CD
:10D2E800C9FA336838801A46591C316012F8021B93
:10D2F800F97032605A783A71DA1C32609A78BA71E9
:10D308001A1D3260DB787B710135EBB29845D4D1B8
:10D31800FEF7B3BE08F10103336098F800001D283A
:10D328003FF6FCAA08F10203336098F801100329BC
:10D338003FF6F4AA464A474F0A2303FB00F3D018E6
:10D3480008F103054171356098F80210D15408F1CD
:10D358000403336098F80330437008F10503336021
:10D3680098F80430837008F10603336098F80530A4
:10D37800C37008F10703336098F80630037101257C
:10D388004FF0FF333B602B46FEF75DBE3046F6F7A5
:10D3980071FA3046F6F76EFA3046F6F76BFA304611
:10D3A800F6F773FA33682C4D1A46581C2968306012
:10D3B80012F8020B81F8460032605B7881F847303A
:10D3C8003046F6F762FA3046F6F75FFA3046F6F777
:10D3D8005CFA3046F6F759FA30462F68F6F74AFAFB
:10D3E800388730462F68F6F745FAD6E90083A3EB6D
:10D3F8000802012AF88600F31585A3EB0802032A20
:10D4080000F30185A3EB0802012A00F3F584A3EBDE
:10D4180008020D2A00F3B184A3EB0803062B00F3DE
:10D42800F483286818F00CF8FEF727BE482500207A
:10D438004C250020843A0020B4390020E35900200C
:10D44800A8300020281E0020231E002040110020A4
:10D45800A415002090010020D82200202259002085
:10D4680008F101033360D34DD34F98F80030FB80A7
:10D478003046D5F80080F6F7FDF9A8F802003046E6
:10D48800D5F80090F6F7F6F9D6E90083A3EB080281
:10D49800072AA9F8000000F35584A3EB0802032A21
:10D4A80000F34484A3EB0802002A00F33384A3EBBF
:10D4B8000803092B00F308847368A3EB0803082BFF
:10D4C80000F3E483FDF746F81DF026F9BB4B1B6813
:10D4D800002B00F0D0832868012516F0FDF92B46B3
:10D4E800FEF7B1BD434608F101023260B24F13F8AE
:10D4F800022B7A703360B24A98F80130137008F141
:10D5080003033360AF4D98F802302B7108F1040320
:10D51800336098F80330092BA8BF09233046AB7055
:10D52800F6F7A8F9D6E90083A3EB0802012A2880B8
:10D5380000F364834345424640F05183A2EB08025E
:10D54800072A00F32D830125FDF704F82B46FEF783
:10D558007ABD9D4B1D68002D00F020832B6828465E
:10D568005B68984707463046F6F784F93F2840F24B
:10D57800EB8241F26F73984203D8944B0022988053
:10D588001A70D6E90032D21A012A7EF776AD5A1CF3
:10D598003260DFF838821A7888F80220FF2F3EF4CC
:10D5A8006CAD9A1C16A9326000225F7801F8402DF4
:10D5B800284611F0FFFD9DF81830BB4203D03946CC
:10D5C800284611F0FAFDD6E900329A423EF455ADEC
:10D5D8005A1C32601B7888F80830FEF74EBD08F1F7
:10D5E80001029A42326018BF08F1020398F800104D
:10D5F8001ABF336098F801300023002900F09682A2
:10D608004FF40040FCF7B8F8714B1B78DB0701D5E5
:10D6180002F0B2FE6F4B002201251A702B46FEF76E
:10D6280012BD08F1010333606B4B98F800209A7023
:10D63800FFF7E1B9434608F10102326013F8025BD3
:10D64800336008F1030398F80100336098F802107A
:10D65800002D00F00882012D7EF40FAD08F0D6FBF6
:10D668002B46FEF7F0BC3046F6F704F95B4F3860FE
:10D678003046F6F7FFF878603046F6F7FBF80125F4
:10D68800B8602B46FEF7DFBC08F10103544D336048
:10D6980098F800302B723046F6F7ECF8E8823046FE
:10D6A800F6F7E8F868823046F6F7E4F83368A882B7
:10D6B8005A1C32601B786B7373689A1A032A00F33A
:10D6C8001082D6F800801A464346D11A052900F37D
:10D6D800F38100297EF7D1AC591C31601B78EB76B9
:10D6E800D6F80080A2EB0803052B29DD434608F194
:10D6F8000101316013F8021B6976336098F8013034
:10D7080085F8253008F10303336098F8023085F86E
:10D71800263008F10403336098F8033085F8273081
:10D7280008F10503336098F8043085F8293008F1CA
:10D738000603336098F8053085F82A30D6F800805B
:10D74800A2EB0803002B3FF759A9FEF796BC08F196
:10D7580001023260234998F8000008709B1A002BD8
:10D768007EF78BAC08F10203336098F80130003380
:10D7780018BF012301254B702B46FEF764BC08F146
:10D788000103336098F800301F2B3FF6C7A8052A1D
:10D798007FF4C4A83046F6F756F8D6E90032D21A14
:10D7A800002A7EF76AAC5A1C32600F4A1B78D37085
:10D7B800FEF763BCD8220020D0430020385900204F
:10D7C80098300020A84B0020602200205E25002011
:10D7D800231E0020F91400204C2A00205C1A002087
:10D7E800E4590020043A00205022002008F10102E8
:10D7F800326098F800500193132D3FF68FA808F176
:10D808000202326098F801000BF0B4F800283FF4E7
:10D8180085A8062202FB05F2D54D0178A95408F126
:10D8280003013160154498F802206A7008F1040277
:10D83800326098F80320AA70019B08F10502326053
:10D8480098F80410E9709A420ED008F10603336084
:10D8580098F805302B7108F10703336098F8060033
:10D868000BF088F803786B7101251AF09BF82B46AA
:10D87800FEF7E9BBBF490023102A28BF1022C1E9DF
:10D888000033C1E902330B7405E03068451C35608C
:10D898000078C85401339342F7D3FEF7EEBB304605
:10D8A800F5F7D1FFB44B93F8B420C3F8B800002AB9
:10D8B8007EF4E3AB012283F8B42015461346FEF745
:10D8C800C2BB08F101024346326013F8022BAA4991
:10D8D8003360FF2A81F8BC207EF405ADFEF741BF16
:10D8E80008F102033360A54B98F801201A7008F17B
:10D8F8000302326098F802205A7008F1040232607C
:10D9080098F803209A7001252B46FEF79CBB3046F9
:10D91800F5F7B0FF9A4FFEF7D5BE3046F5F7AAFFE8
:10D9280001253046F5F7A6FF2B46FEF78CBB08F11C
:10D938000203336098F80150022D3EF6EFAF3046EF
:10D94800F5F798FF8F4B03EB45034FF0FF35A3F82E
:10D958006E002B46FEF777BB5A1C32601B78002BF3
:10D968007EF4F5AF132F3EF6F2AF00285CD1854A5E
:10D978000125D36F05FA07F723EA0703D3672B4678
:10D98800FEF761BB08F1020333607F4B98F8012072
:10D998001A7008F1030333607A4F98F8023087F859
:10D9A8006D3008F10403336098F8033087F86C3061
:10D9B8003046F5F75FFFA7F868003046F5F75AFFDD
:10D9C8003046F5F757FFD6E90083A3EB0802012A92
:10D9D800A7F86A0005DD3046F5F74CFFD6E9008365
:10D9E8007867A3EB0802032A12DCA3EB0803002BD9
:10D9F8007EF743AB3046F5F748FFD6E900239B1A7C
:10DA0800002B3EF7FBAFFEF738BB4A46FEF7F2BEE7
:10DA18003046F5F718FFD6E900837867E5E7042A6A
:10DA28007EF42BABFFF736BB3846012510F01CFC03
:10DA38002B46FEF708BB08F10102326098F8002077
:10DA48003A71D6F80080FFF73CBB08F1010239684B
:10DA580032609A1A98F800000872002A09DCD6F891
:10DA68000080FFF7D8BA012517F0CEFC2B46FEF749
:10DA7800EABA08F10202326098F801204A71D6F831
:10DA88000080A3EB0802002A7FF7C5AA08F101016C
:10DA98003A68316098F800101171D6F80080A3EB4D
:10DAA8000802002A7FF7B7AA08F101013A68316035
:10DAB80098F80010D171D2E75A1C3260334F98F8A9
:10DAC80000303B703046F5F7BEFE32687860531C74
:10DAD800336012783A727268D11A00297FF700AE63
:10DAE800FAE53046F5F7C6FEE8833046F5F7C2FE9C
:10DAF800D6E90083A3EB0802032A28847FF7E3AD65
:10DB0800434608F10102326013F8022B2A7633608B
:10DB180098F80130AB763046F5F7ACFE0A22A0F54E
:10DB28007A7393FBF2F32B777368CAE5184919489F
:10DB38000A68003318BF012322F40042012503704C
:10DB48000A602B46FEF77FBAC208DFF84C80013224
:10DB580000F007030133D0B2014688F800001A46E6
:10DB6800284688F8013010F09DFEA8F8040008E562
:10DB78003C340020902B002040110020A0220020DF
:10DB8800A4220020581D002098430020B43400200F
:10DB9800B0290020F91400205E250020FF27E2E4C8
:10DBA800434608F10102326013F8022B3A713360E0
:10DBB80098F80130FB7008F10303336098F80230DD
:10DBC8003B703046F5F756FE78833046F5F752FE3F
:10DBD800336878825A1C32601B783B75B3E4304650
:10DBE800F5F753FED6E9003293423FF4ACAC591C2A
:10DBF80031601B78EB70D6F800809FE43046F5F76B
:10DC080039FED6E90083288294E4434608F10101ED
:10DC18002A68316013F8021B82F86E10336098F896
:10DC2800013082F86F3008F10303336098F802304E
:10DC380082F8703008F10403336098F8033082F8F2
:10DC4800713008F10503336098F8043082F87230B7
:10DC58003046F5F71AFE3046F5F717FEFFF7E1BB39
:10DC6800864B1A88012512FB00F22B4692FBF1F233
:10DC78003A80FEF7E8B982488249834A834B0360B9
:10DC880001250B6013602B46FEF7DDB908F1010290
:10DC98002B68326098F8002083F860203046F5F74A
:10DCA800E9FDB8833046F5F7E5FDF88330462F687F
:10DCB800F5F7E0FDA7F8620030462E68F5F7DAFDC3
:10DCC800A6F86400FFF7FEBB08F10103336098F87B
:10DCD8000030BB703046F5F7D8FD3046F5F7CAFD81
:10DCE800F8803046F5F7C6FD336838811A46591C66
:10DCF800316012F8021B797532605B78D5F80090B4
:10DD0800BB753046F5F7B6FDD6F80080A9F84C008B
:10DD1800FFF7D2BB08F101012A68316098F80010BA
:10DD280082F82610D6F80080FFF7C1BB3046F5F719
:10DD3800A1FDF8813046F5F79DFDD6E900833882CC
:10DD4800FFF7B0BB3046F5F795FD78813046F5F71B
:10DD580091FDB8813046D5F80080F5F78BFDA8F81D
:10DD680004003046D5F80080F5F784FD7368A8F8FC
:10DD78000600D6F80080FFF790BB08F101022B6877
:10DD8800326098F8002083F851203046F5F77DFD81
:10DD9800336829681A46581C306012F8020B81F85B
:10DDA800550032605B7881F853303046F5F76DFDE9
:10DDB80033682A68591C31601B7882F84F30304626
:10DDC800F5F763FD30462F68F5F754FDB881304606
:10DDD8002F68F5F74FFD788230462F68F5F74AFD32
:10DDE80033682A683883591C31601B7882F83030D0
:10DDF800D6E90083FFF710BB3046F5F73BFDD6E9BF
:10DE08000083FFF704BB30462F68F5F733FD7886AB
:10DE180030462F68F5F72EFD7368D6F80080B8866F
:10DE2800FFF7F0BA08F101022B68326098F8002079
:10DE380083F82D203046F5F728FDD6E90083FFF753
:10DE4800DCBAFDF7C9FAFFF722BA4F46FFF745BA21
:10DE58003046F5F71AFD33680D4A591C31601B78B6
:10DE6800D371FEF7CBBD00F07F00062828BF002045
:10DE7800012507F0F3FF2B46FEF7E5B882300020B6
:10DE8800CC3400203C350020243600206B050008E7
:10DE9800B430002010B5094C238823EA00009842CA
:10DEA800208009D0064B41F20241FF2219809A7066
:10DEB8000E20FDF703FF2388184610BD0826002012
:10DEC8003C15002010B5094C23881843984220803F
:10DED80009D0074B41F20241FF2219809A700E20A7
:10DEE800FDF7ECFE2388184610BD00BF0826002069
:10DEF8003C1500202DE9F047D54C2DED028BA36889
:10DF080020469847002800F0D180D24B1B78012288
:10DF1800042B84F8382000F0CD80B4F91A3006EECE
:10DF2800903AB4F91C3007EE103AB4F91E3007EEF7
:10DF3800903AF8EEE66AB8EEC77AF8EEE77AC4EDFA
:10DF48000B6A84ED0C7AC4ED0D7AC34B1B88002B49
:10DF580060D0C24B94ED0B2AD4ED0C2A94ED0D3A07
:10DF680093ED008AD3ED054A93ED090AD3ED0E3AF5
:10DF7800D3ED120A93ED174A93ED011A93ED065A61
:10DF8800D3ED0A1A93ED0F6AD3ED137A93ED187A4D
:10DF9800D3ED045AD3ED0D6AE8EE024AE0EE223AD8
:10DFA800A3EE204AA1EE025AA2EEA16AA3EE277AB6
:10DFB80093ED038AD3ED167A93ED020AD3ED0C0A9A
:10DFC80093ED0B1AD3ED151AC4ED0B4A65EEE45A1E
:10DFD800A8EE645A66EEE36AD3ED144A83ED055A57
:10DFE80067EEC47AE0EE025AA0EEE36AE2EE816AD6
:10DFF800A4EE617AE3EE247AC3ED065AC4ED0C3A36
:10E0080083ED0E6AC3ED0F6A83ED177AC3ED187AB4
:10E0180084ED0D4A924F94F822109248924E14F0D3
:10E02800E1FC3B88D6F8A050002B40F096808F4B3F
:10E038001B685B075BD4B5F9003094ED0C6A94ED6E
:10E048000D7A94ED0B5A8A4905EE903AB5F90230EB
:10E058000A6806EE903AB5F9043007EE903AF8EE01
:10E06800E55A844BF8EEE66AF8EEE77AD3ED003A23
:10E0780093ED014AD3ED024A75EE655A76EE666A6B
:10E0880077EE677AC4ED0B5A34EE266A73EEA55A1A
:10E0980034EEA77A0132C3ED005AC4ED0C6A83ED61
:10E0A800016AC4ED0D7A83ED027A0A60BDEC028B39
:10E0B800BDE8F087B4F91A00B4F91C10B4F91E20B1
:10E0C8006D4B07EE900AF8EEE76A07EE901AB8EE85
:10E0D800E77A07EE902AF8EEE77AC4ED0B6A188023
:10E0E80059809A8084ED0C7AC4ED0D7A2DE7634F40
:10E0F8003B88322B00F0CC80002B40F01881604820
:10E108000378002B97D05F4FD6F8E83087FB03ECF5
:10E11800DB17D6E93821C3EB2C13B4F818C0A3EBEE
:10E128000C03AB8087FB02C387FB01C7C917C1EB90
:10E138002711D217544F6980C2EB231200230370B2
:10E148002A807B81BB81FDF747F9FDF727FA01207B
:10E15800FDF79EFED6F8A0506DE7B3F5C87F18BF4F
:10E16800D6ED327AD4ED0B6A0CBF9FED487AB8EE43
:10E17800E77ADFED467A0023C4ED0B7A2B803B88E3
:10E18800B7F8008037EE267AB3F5C87F18BFD6ED0A
:10E19800337ABDEEC77A18BFF8EEE77A17EE102A81
:10E1A80086ED327A94ED0C7A77EE877A0021FDEECF
:10E1B800E77A0020B8F5C87F216317EE903A6880A7
:10E1C800C6ED337A00F0AA80D6ED347A94ED0D7A54
:10E1D8006163F8EEE77AB8F1010F77EE877AA880E5
:10E1E800FDEEE77A17EE901AC6ED347A2BD1DFF8F8
:10E1F80094C0B4F818E0C8318CFB01A9C832C83300
:10E20800C917C1EBE9118CFB02A98CFB03ACDB1726
:10E21800C3EBEC13D217DFF870C06B80A1EB0E01D3
:10E22800C2EBE912A9802A80ACF80A00ACF80C000D
:10E23800FDF7D2F8FDF7B2F94046FDF729FEB7F829
:10E248000080D6F8A05008F1FF38A7F80080EEE665
:10E25800842A0020B01C00207C310020803100205E
:10E268005E140020B02A002040110020904A0020AF
:10E278008439002088390020B41C0020941500201F
:10E28800911500201F85EB514C2A0020000000004A
:10E29800384B2A68D3F80A30C6F8DC309FED367A56
:10E2A800B5F90430C6F8D420A6F8D830DFED327AB4
:10E2B800D4ED0B6AC4ED0B7A00232B803B8837EE34
:10E2C800267A322B18BFD6ED397A3B88BDEEC77A4D
:10E2D80018BFF8EEE77A86ED387A94ED0C7A77EE87
:10E2E800877A0021FDEEE77A0022322B2163C6ED02
:10E2F800397A6A8034D0D6ED3A7A94ED0D7A616332
:10E30800F8EEE77A012B77EE877AAA80FDEEE77AB6
:10E31800C6ED3A7A10D0013B3B80F0E6D4ED0D7A99
:10E328006163FDEEE77AA880C6ED347A8BE7D6ED17
:10E33800387AB8EEE77AB9E71048114902700B202D
:10E348000B70FDF7BBFCD6F8D4302B60094AB6F940
:10E35800D800D6F8DC10A8803B88C2F80A10DAE7A3
:10E36800D4ED0D7A6163FDEEE77AAA80C6ED3A7ABC
:10E37800D1E700BF4C2A00200000000096150020BD
:10E38800901500202DE9F04FAA4BAB4D1A7829784B
:10E39800D20785B0034654D5A84CA94E012979D097
:10E3A800C0F09280022943D0E27B62B3A28952B3C3
:10E3B800A448007838B3A4489FEDA46AD0ED026A57
:10E3C80007EE902AF8EEE66AB8EE677AF8EEE77A92
:10E3D80077EE666A66EE866A86EEA77AFDEEC77AFB
:10E3E80017EE902A002AC0F2E880642A00F37881A8
:10E3F800002A00F0E280D2B2207C90422CBF01209B
:10E408000020307000E03078257A632D05D8904ED2
:10E418000229327864D0002A76D18E4AA37B8142C1
:10E4280038BF01461170002B44D105B0BDE8F08F0C
:10E4380089488A4A008812889042B5D901212970F2
:10E44800B2E7854F7D4C3888CA1E012A77D97A8869
:10E45800821A002AB8BF5242142A05DCE288824296
:10E468005AD82688864257D3754E7D4A1278022A92
:10E4780094D178883A88734F121A002AB8BF52424A
:10E48800142A78483F788780CCBF002201220129CE
:10E49800C28085D1714A70481288677C0088D21B77
:10E4A80090422EDD704A12888242BFF47DAF00216F
:10E4B800297079E701297AD00229B6D1072005B059
:10E4C800BDE8F04FFDF7FABB674A63481288677CDE
:10E4D8000088D21B90423FF767AF0121297063E79C
:10E4E80092B9012773603770C5F164055F4B02FB71
:10E4F80005F283FB0253D217A2EBA3526432727067
:10E508008BE7022129704FE772689A1A584B9A4292
:10E51800C8BF757081DCE7E7B0EB420F484EA4DC5A
:10E52800DFF820E1DFF840C14C48002203213170B8
:10E5380029708EF80020ACF80020028095E7E28868
:10E5480082422DD8268886422AD37A88821A002ABF
:10E55800B8BF5242142A87DC394E227D4FF0000999
:10E5680086F8009085F8009052B336484946027004
:10E57800B4F804C03C48B4F80280DFF8E0E092B296
:10E588001CFB02FCA0F800C018FB02F23048AEF8F1
:10E5980000204FF0640C002280F801C0426064E75C
:10E5A800B0EB420FD1DC03293FF45EAF4FE7082000
:10E5B80005B0BDE8F04FFDF781BB0220307023E7BE
:10E5C8002C4A21881268B0FBF1F10131082992F92F
:10E5D8007400DFF87080A8BF0821CAB2884288F8A2
:10E5E800002000917ED000287CD02348DFF890E0FE
:10E5F80090F800B00BF1010CAEFB0C10410801EBD8
:10E608004100ACEB0001594501918C466AD01B4989
:10E618004FF0760A0AFB0C19009999F9749049454C
:10E62800604653D0CDF808A0CDF800E04FF0FF3A8F
:10E6380003932BE0231E0020A0130020401D002080
:10E64800C81300207F250020682500200000C8424C
:10E65800A81300207E25002078250020A413002080
:10E66800B01C0020B41C0020A21300206BCA5F6BF2
:10E678007F969800D8220020245C0020E822002001
:10E68800ABAAAAAA9EF9749089452DD0009B0CF1DB
:10E69800010EA3FB0E3C4FEA5C0C029B0CEB4C0CEE
:10E6A800AEEB0C0C9E46124BBAF1000F0EFB0C3E63
:10E6B80003DAB9F1000F08BF8246DC456046E1D1B4
:10E6C800039BCDF804A0514600290BDB9DF80400FC
:10E6D8000093FDF7FEFB98F800202978009B47E798
:10E6E800642289E6002143E70190039B0146EBE79A
:10E6F800E82200201D4B70B59C68636DA26BDD6934
:10E70800CAB1E36B33B12B0700D470BD636D082227
:10E718001A6270BD2A06F6D5D4E909028242616DF3
:10E7280011D0501CA669A062B25C26690A85B04265
:10E73800E9D3A362E7E7A906E3D5E26A42B1988C78
:10E74800216B9047DDE70B6823F080030B60DAE765
:10E75800E1699B8C6069DBB24E1CE6614354E16958
:10E76800E368994228BFE261CBE700BF2C1A00207A
:10E778002DE9F04FB94B1B78242B8DB000F0B981EF
:10E78800B74B1D78002D57D1B64BB74C93F800B056
:10E79800DFF80493DFF804A30BF0010B04F52578E8
:10E7A80054F80B0C40B1F2F780FF0646002840F001
:10E7B8000D8114F8033C3BB9DC34444505F10105EF
:10E7C800EED10DB0BDE8F08FDAF8002054F8071C40
:10E7D800521A632AF0D9012B00F04083022BEBD1A7
:10E7E800A24BA349DA7889F805020032A148C9F892
:10E7F800EC0018BF01229A4854F80B3C0A7001211A
:10E808009D4A0170C9F8F030C9F8F831C9F80032EA
:10E818009A48C9F8FC21402389F80432F4F792FF9A
:10E828004FF48050FAF7A8FF9548F4F70BFF89F8E2
:10E83800486289F84962BFE7DFF85C92D9F8EC00D2
:10E848000028BED0F4F7B3FEDFF834A209F1F808C7
:10E85800D9F8F000F2F729FF0028B2D0D9F8F00073
:10E86800F2F71DFF09280346D9F8F4601DD03F28A8
:10E878001BD0002E6FD1042800F0A6820C2800F0CF
:10E888009E807F28E4D0A0F12002D2B25E2ADFD891
:10E89800202BDDD009EB06021846013682F8F83045
:10E8A800C9F8F460F4F7C6FED2E7002E65D1754BBF
:10E8B800354603F59877002D46D00833BB42FAD188
:10E8C800DFF8DCB12868DBF80020845D935D9C42AA
:10E8D800304402EB060140F0BF82741E44443246C5
:10E8E80013B9FD2A40F2F88004F8013F0132C9F853
:10E8F800F42010F8013F11F8017F9F42F0D00AB1CF
:10E90800AB4513D06048F4F79DFEAB4508D355F8E6
:10E91800080BF4F797FE0920F4F78CFE5D45F6D94D
:10E928005046F4F78FFED9F8F420002696428FD28D
:10E93800741E444414F8010FF4F77CFED9F8F4303F
:10E9480001369E42F6D383E703F10802BA421D4618
:10E95800B6D01346AFE70C2831D00A2B64D00D2B64
:10E9680062D07F2B00F0FB81FF2E3FF671AFA3F141
:10E978002002D2B25E2A8DD96AE7424C4FF0000BD2
:10E9880004F598775D4602E00834BC420DD0324663
:10E9980021684046F5F742F90028F5D1A346002D35
:10E9A800F2D125460834BC42F1D1002D8AD1BBF101
:10E9B800000F3FF44DAF3448F4F744FEA7E733485F
:10E9C800F4F740FE5046F4F73DFE41E7304BDAF8E5
:10E9D800002044F8072CDC27002607FB0537A4F1A4
:10E9E8000B0304F8036C009354F80B0CF2F75DFE6C
:10E9F80000283FF4E1AE54F80B0CF2F750FE14F87F
:10EA0800021C4B1E02460B2B00F29781DFE813F025
:10EA1800800178016C01450133011901ED00A9005D
:10EA28009C00C70083007B00F4F778FE2321194877
:10EA38001FF016FB002800F07D81A0EB0802C9F842
:10EA4800F420D2B3531E09EB030191F8F8102029E2
:10EA580040F03582023A42442AE000BFB01C002050
:10EA68004D270020231E0020BB400020245C0020EE
:10EA7800101800203C13002097010008905103084B
:10EA88005C5103085CFE02085451030864510308F2
:10EA9800B04000203812002040110020603D0020C6
:10EAA80084FF020812F80119202940F06881034602
:10EAB800581E002BF6D1C9F8F4304FF480720021AB
:10EAC80040461FF0B6FAC24B1B78002B3FF479AED4
:10EAD8005046F4F7B7FDBBE6511C09EB01004A4468
:10EAE800202482F8F840C9F8F4100A4680F8F83073
:10EAF80006E7B84BB84A1B6800215B1A18BF012308
:10EB0800538011803CE694F8CE30934200F09E800A
:10EB180004F8026C68E7114694F8CE000192F5F704
:10EB2800ABF9D4F8C530019A84F8CE00F91801334E
:10EB3800C4F8C530CA72D4F8C92093427FF454AFE0
:10EB48000C2304F8023C4FE794F8CD3094F8CE102B
:10EB58005340914284F8CD30DAD1062304F8023CC0
:10EB680042E7114694F8CE000192F5F785F9D4F8FA
:10EB7800C53094F8CD10019A84F8CE00F8185140A9
:10EB88000133C4F8C53084F8CD10C272D4F8C92056
:10EB980093427FF429AF092304F8023C24E7D4F810
:10EBA800C530F9180133C4F8C530CA7294F8CE00DC
:10EBB80001931146F5F760F9019B84F8CE00052B07
:10EBC8007FF412AFB4F80330B4F801102278C4F817
:10EBD800C560C4F8C930A4F8C11084F8C320002B5C
:10EBE800AED00B2304F8023CFEE6D4F8C530F91881
:10EBF8000133C4F8C530CA7294F8CDC094F8CE0079
:10EC0800019382EA0C0C114684F8CDC0F5F734F96B
:10EC1800019B84F8CE00072B7FF4E6AEB4F80530EC
:10EC2800B4F80310A278C4F8C560C4F8C930A4F8D1
:10EC3800C11084F8C320002BADD0082304F8023C8F
:10EC4800D2E694F8CD3093427FF462AF0D2304F8F6
:10EC5800023C14F8017C002F00F0C880012F00F05E
:10EC68000F81002304F8023CDC34444505F101051A
:10EC78007FF496ADA5E5D4F8C530F9180133C4F88A
:10EC8800C530CA7294F8CD00D4F8C91042408B42FE
:10EC980084F8CD207FF4A8AE5FE7D4F8C530F91822
:10ECA8000133C4F8C530CA7294F8CD10022B82EA39
:10ECB800010284F8CD207FF497AE2378C02B3FF66D
:10ECC80027AF6278FF2A00F0FC80C4F8C930A4F8A6
:10ECD800C12084F8C360C4F8C560002B3FF43DAF81
:10ECE800052304F8023C7FE60A233C2A04F8023C88
:10ECF8000BD03E2A7FF40CAF012304F8013C73E6E5
:10ED080004233C2A04F8023CF3D104F8016C6BE6B6
:10ED18004D2AC4F8C56084F8CD6084F8CE6049D027
:10ED2800582A7FF4F5AE0322022304F8022C84F853
:10ED3800C43059E6D9F8F42083E6242A40D0BBF140
:10ED4800000F02D00D2984D04EE6232A13D0234B7E
:10ED58009B7C934204BF012304F8033CF2E7013E85
:10ED680009EB060300221E48C9F8F46083F8F8206E
:10ED7800F4F768FC6CE5022304F8033CE2E7C9F801
:10ED8800F4304B44174C002283F8F82004F59877A8
:10ED980003E00834BC4200F09E8021684046F4F746
:10EDA80092FF0028F5D0BC4280F0958063689847B0
:10EDB800002380E6022384F8C46004F8023C13E6CA
:10EDC800012304F8023C0FE60748F4F773FCF8E463
:10EDD8004D2700207C3B0020B41C00202259002035
:10EDE8008C5103085CFE0208381200203C4BB4F832
:10EDF800C1E0ADF82C700FCB0DF1300C04AE86E8F5
:10EE08000F00D4F8C9104CF8247D601894F8C3306A
:10EE1800099001276246314608A80894ADF828E011
:10EE28008DF82A308DF82E70FDF772F8E8B9039E38
:10EE3800002304F8023C002E3FF4BEAC54F80B0C3F
:10EE4800FCF7CEFEDC3454F8E70CB047444505F136
:10EE580001057FF4A5ACB4E4324650E5214A224BC3
:10EE680022491160224ADA60A6E4049A214B0592ED
:10EE78003146009894F8C420049309F033FCD6E78F
:10EE8800D4F8C930B4F8C1200894234409936E2AF1
:10EE98004FF00003ADF82E30CDF82A30ADF8282019
:10EEA8007FF4DFAE08A8F4F7F0FC08A8F4F7E2FC5A
:10EEB80008A8F4F7DFFC08A8F4F7DCFCD1E6134651
:10EEC8005FE7052B7FF624AE0122072384F8C420D0
:10EED80004F8023C88E50848F5F79AF968E700BFA6
:10EEE8008CFF0208FC9F002000ED00E0EFBEADDEC5
:10EEF8000400FA05345C002070510308174B9FED9D
:10EF0800185A1B681844BFEE007A437A06EE103A86
:10EF1800C378A0EE007A07EE903A8379B8EE466A95
:10EF280005EE903A60EE850AF7EE006AF2EE044AC2
:10EF3800B0EE664A20EE240AA6EE204A27EE057AAD
:10EF4800F8EEE55AF8EEE77AE5EE876A67EE807A3A
:10EF580024EE270A20EE260A704700BFDC36002080
:10EF68000AD7233C2C4B1B68184483799BB107EEC6
:10EF7800903ADFED2A6AF8EEE77A20EEA07A67EE9B
:10EF8800A67A27EE207AF7EE006AD7EE877A77EE30
:10EF9800A67A20EE270AC378DFED206A07EE903ABA
:10EFA800F8EEE77AB0EE007A67EEA67AF4EEC77A62
:10EFB800F1EE10FA05DD37EEC77ADFED196AE7EEF4
:10EFC800267A437A9FED177A20EE070A20EE270A61
:10EFD80003B3DFED127A9FED147A06EE903A60EEF5
:10EFE800A77AF8EEE60A60EEA70AF4EEC70AF1EE91
:10EFF80010FA04DDDFED0D7A20EE270A7047F5EEF2
:10F00800C00AF1EE10FA05D4F7EE007A77EEE00ABE
:10F0180080EE200A704700BFDC3600200AD7233C68
:10F02800D7A3684100004843A4707D3F0000C84250
:10F03800F0B45D4E5D4832785D4B5E4DDC6B2D78EB
:10F048000132A0FB0270000900EB8000A2EB8000F7
:10F058001A683070914201EB04005C6811D293F891
:10F068004520002A4ED000F58030B0FBF5F08442F0
:10F078000BD2041B4FF4803292FBF5F2A21A9A606D
:10F088000AE0B0FBF5F0844244D34FF4803292FB9F
:10F09800F5F2121B02449A6040F68C240025A24225
:10F0A800C3E9001083F8455017D993F8402093F925
:10F0B80042108A4256B241D0002093F9411083F899
:10F0C80043008A4247D00121002283F8426083F836
:10F0D800441083F84020F0BC704793F8441000298E
:10F0E800F9D0A2F2EF2040F2DA5188421AD893F808
:10F0F80040100B2916D803EB81000131C26083F858
:10F108004010E8E7B0FBF5F08442BED2041BA21A17
:10F118009A60C1E793F84520002AAAD1041BA21AD5
:10F128009A60B9E7244A002102F1300083F84410BC
:10F1380042F8041F8242FBD1F0BC7047111F082916
:10F14800BAD893F84310182926D8013183F8431008
:10F1580093F94110B5E793F844100029B3D0FAB1F8
:10F168001649154C0FFA82FC084601EB4C0754F877
:10F17800045F20F8025BB842F9D10B2A07DC10487B
:10F1880001EB4C02002122F8021B9042FBD10D49F1
:10F198000A7801320A7096E783F84160314690E7B1
:10F1A80094460649EBE700BF90130020CDCCCCCCA9
:10F1B8009C4A0020F00F0020A44A00204C2F002079
:10F1C800642F00203C2F002030B40E4D0E4B2A78BF
:10F1D8000E4C0132A3FB02031B09E06B03EB830314
:10F1E800A2EB83034FF6FF72914200F101002B70EE
:10F1F800084408BF0123E06308BF84F8453030BCE9
:10F20800704700BF90130020CDCCCCCC9C4A002086
:10F21800002800F01B81B24B1A7CF0B4002A40F0A1
:10F2280097801968002201280A6043D093F82810B3
:10F23800002941D19969002202280A603AD093F83E
:10F24800401000295ED1196B002203280A6031D0D2
:10F2580093F85810002940F0A080996C00220428E7
:10F268000A6027D093F87010002940F0F080196EDA
:10F27800002205280A601DD093F88810002940F064
:10F288000C81996F002206280A6013D093F8A01009
:10F29800002940F02D81D3F89010002207280A6039
:10F2A80008D093F8B810002940F0A380D3F8A8300C
:10F2B80000221A60F0BC7047D9698A4D8C0AAC42AA
:10F2C80000F0518140F23781874A944200F05B8117
:10F2D8004B32944240F033810322EFF311845025DE
:10F2E80085F31288814E4F6A4D6902EB820206EB64
:10F2F800C202013745F001055762E4B24D6184F35B
:10F30800118897E7596B774D8C0AAC4200F02D8134
:10F3180040F21781744A944200F03D814B32944286
:10F3280040F013810322EFF31184502585F31288EE
:10F338006E4E4F6A4D6902EB820206EBC20201373C
:10F3480045F001055762E4B24D6184F311887AE70C
:10F358005A68644C910AA14200F0F98070D9624C55
:10F36800A14200F0F8804B34A14240F0F280032122
:10F37800EFF31184502585F312885C4E576A55695E
:10F3880001EB810106EBC101013745F001054F6230
:10F39800E4B2556184F3118843E7D96C514D8C0A66
:10F3A800AC4200F0018140F2D8804F4A944200F00C
:10F3B800F9804B32944240F0D4800322EFF3118459
:10F3C800502585F31288494E4F6A4D6902EB820237
:10F3D80006EBC202013745F001055762E4B24D6100
:10F3E80084F31188996C002204280A607FF43AAFEC
:10F3F80060E7D3F8AC103B4C880AA04200F0E380E9
:10F4080040F2B780384A904200F0DB804B3290429D
:10F4180040F0B3800322EFF31180502484F3128864
:10F42800324D4E6A4C6902EB820205EBC205013689
:10F4380044F001046E62C2B24C6182F3118835E770
:10F44800B1F5801F40F08580002191E77047596E23
:10F45800244D8C0AAC4200F0AE8040F29680224ADD
:10F46800944200F084804B32944240F09280032210
:10F47800EFF31184502585F312881C4E4F6A4D69AD
:10F4880002EB820206EBC202013745F00105576222
:10F49800E4B24D6184F31188E9E6D96F114D8C0A05
:10F4A800AC4200F08A8078D90F4A944267D04B3238
:10F4B800944275D10322EFF31184502585F3128805
:10F4C8000A4E4F6A4D6902EB820206EBC20201370F
:10F4D80045F001055762E4B24D6184F31188D0E626
:10F4E800E84A002001001000020010009C3B0020A8
:10F4F800D3F89410354D8C0AAC4260D056D9344AB2
:10F5080094423ED04B32944253D10322EFF31184FC
:10F51800502585F312882F4E4F6A4D6902EB8202FF
:10F5280006EBC202013745F001055762E4B24D61AE
:10F5380084F31188AFE6B4F5801F3FF4CEAEFE2207
:10F54800CBE6B4F5801F3FF4EEAEFE22EBE60121D8
:10F558000EE7FE210CE702210AE7B4F5801F3FF40D
:10F568002DAFFE222AE70122B7E60122DBE60222BE
:10F578007EE7B0F5801F3FF44EAFFE224BE7022234
:10F5880099E70222C2E70222A7E6B4F5801F3FF4FA
:10F598006FAFFE226CE70222C5E6B4F5801F8AD061
:10F5A800FE2288E7022209E7012207E7B4F5801F57
:10F5B800ACD0FE22AAE701225AE701227BE701220A
:10F5C800A4E7022227E7012225E700BF0100100077
:10F5D800020010009C3B0020704700BF70B4150B60
:10F5E800C2F30324C2F3031305EB45054E00183597
:10F5F80004EB440403EB4303056018340D0118338E
:10F6080002F00F0240F8214002EB420240F8263097
:10F6180044190E440023183240F82620435106208E
:10F6280044F8213070BC704712F4004F2DE9F04FB8
:10F6380014BF4FF00E0A4FF0070A12F4804F4FEA3A
:10F64800410614BF4FF00E094FF0070912F4005F8E
:10F6580014BF4FF00E084FF007088D1912F4805FA1
:10F6680001EB050414BF4FF00E0E4FF0070E12F415
:10F67800006F01EB040314BF4FF00E0C4FF0070CA2
:10F6880012F4806F14BF0E27072701EB030B12F447
:10F69800007FC0F800A040F8219018BF4FF00E0A74
:10F6A80040F8268008BF4FF0070A01EB0B0612F45A
:10F6B800807F40F825E018BF4FF00E0801EB060EDA
:10F6C80008BF4FF0070812F0800F40F824C040F838
:10F6D800237014BF0E24072401EB0E0312F0400F11
:10F6E80001EB030514BF4FF00E0C4FF0070C12F09E
:10F6F800200F40F82BA018BF0E2740F8268008BF1F
:10F70800072740F82E4012F0100F01EB050440F8CF
:10F7180023C014BF0E2607260B1912F0080F40F855
:10F72800257001EB030514BF0E27072712F0040FFD
:10F7380040F8246040F8237018BF0E2601EB05033B
:10F7480008BF072612F0020F40F825604FEA81141F
:10F7580001EB030514BF0E26072612F0010F40F82F
:10F76800236000EB040214BF0E23072340F8253062
:10F7780000230351122042F82130BDE8F08F00BF6A
:10F78800704700BF024B1A889B78028083707047CD
:10F798003000030870B4104A104BB2F90060B2F997
:10F7A80002501C780E4940F6E44202FB00F2120BAC
:10F7B80042F2107303FB02F393FBF6F32B4481FB35
:10F7C8000310232C4FEAE373C3EBA00002D1054BCF
:10F7D8001A80588070BC7047A4220020B01C0020FA
:10F7E80067666666B41C0020084B596869B110B496
:10F7F800DC680020642202FB04F25860B2FBF1F2DC
:10F80800D8601A815DF8044B704770479013002048
:10F8180003680A7A591C01601A70704770B4354938
:10F82800354B364E487A364D364C042232701A74AF
:10F8380064225A7601284FF000025A829A821A7678
:10F84800DA612A70226027D0022811D08C7A2E48DB
:10F858000022012C026083F83820C0E901222FD051
:10F86800022C03D129495A65C1E9012270BC7047AD
:10F87800487D9FED277ADFED276A1A6207EE900A26
:10F88800F8EEE77AB0EE476AA7EEA66A5A62C7EEC4
:10F89800067AC3ED0A7AD9E7487D9FED1D7ADFED38
:10F8A8001D6ADA6207EE900AF8EEE77AB0EE476A68
:10F8B800A7EEA66A1A63C7EE067AC3ED0D7AC5E706
:10F8C800897D9FED137ADFED136ADA6307EE901AEC
:10F8D800F8EEE77AB0EE476AA7EEA66A0E4900206E
:10F8E800C7EE067A4A60C1E90222D864C3ED147AE9
:10F8F800BCE700BF401D0020901300207E2500209B
:10F908007F2500207825002068250020E4130020AA
:10F918000AD7A33C3661823CCC1300204A4A4B4BA1
:10F92800126851024A49F0B5096858BF03F58013B7
:10F93800D70058BF43F480738E074649097844BFFF
:10F9480043F4057343F0020383B001F0EF0043F082
:10F958004004082800946FD00E296DD03E49009BC2
:10F968000978D50354BF43F4006343F4C053D40467
:10F9780054BF43F4900343F4D00309B143F0006348
:10F98800900648BF43F48063510748BF43F40053CF
:10F99800520554BF43F4804343F4404302AE43F05E
:10F9A80047432E4C46F8083D2D4F40230193251D13
:10F9B80014F8010BFF2814D000212A4A0B4603E053
:10F9C8000133282B0DD0117A884202F10C02F7D1AD
:10F9D80003EB430307EB83031979A1F12003032BFE
:10F9E8002ED9AC42E4D1019B43F08003019300245B
:10F9F80002E00134282C18D021463046E5B2F7F74A
:10FA080010F80028F5D0174B002203F5EA7101E041
:10FA180013F80C2F9542ECD08B42F9D12146304691
:10FA28000134F6F7DFFF282CE6D196E803000E4BE9
:10FA380083E8030003B0F0BD43F0600300938DE753
:10FA48003046F6F7DFFFCCE7904A002001000010AF
:10FA5800482A0020043A0020C24B0020A04300207E
:10FA68003000030834000308F0130020F8B50446FA
:10FA78001EF060FA3449642303FB04131D7B05B9A7
:10FA8800F8BD324B93F868C093F86920944580B26A
:10FA98001FD04FEA820E0EEB020703EB8707551CB7
:10FAA800FE6E05F00305002E3ED097F87460002E18
:10FAB8003AD197F87560002E36D0724403EB820372
:10FAC800234493F8760020B1642303FB0413012236
:10FAD8001A76642606FB04151D4B2A7E1F7828819A
:10FAE80042EA400293B21A1282EA13125A4002F012
:10FAF8000F0242EA0312174B0020287692B21B68C5
:10FB0800AFB906FB04101C300121984769696C895C
:10FB1800B1F830212B692243A1F8302158601A68C6
:10FB280042F001021A60F8BD6545C6D1D1E769689F
:10FB38006869497901F0FC010C31084404219847AF
:10FB48006B6980001881F8BDD44B00209013002009
:10FB5800D04B0020C84B002038B500EB4000084DC2
:10FB6800C4002B1993ED027AD3ED037AE7EE007AFD
:10FB7800B0EE670A1EF0DEF92B59186038BD00BFD9
:10FB8800E84A002010B5F1F753FF044630B11122BE
:10FB980000238271C3712021F1F792FD0A20FBF73F
:10FBA8001DFF2046F2F774FB034B002814BF022206
:10FBB80001221A7010BD00BF1A30002070B405462B
:10FBC80000F19C06074C0FCC2860696003CC2488A0
:10FBD800AA60EB602C83286169611A35B542F1D1BE
:10FBE80070BC7047140203082DE9F7430120F9F7A8
:10FBF80097FD294E294F05460024002D39D0022CA7
:10FC080037D8DC236343F25812B10134E4B2F4E785
:10FC1800EB7895F9020057F82330019203210091FF
:10FC280001211AF0DDF98146C8B12B88DC2504FBD7
:10FC3800056013F40F7805FB04F54FF0D8024FF078
:10FC4800000100F1040018BF03F001081EF0F1F9EB
:10FC58007319013446F8059083F8DA80E4B2104944
:10FC6800104891F8BC208C46D3B2012B04D98CF8EB
:10FC7800BC3003B0BDE8F08302F1010E00EBC20511
:10FC880030F832200133D207DBB202D581F8BC301C
:10FC9800B3E77246E8E700BFB0400020B81D03088C
:10FCA80090130020225900206B4B1B78002B39D071
:10FCB80070B56A4B6A4D9B7AD5F8C040C5F8C0004C
:10FCC800013B041B032B00F28180DFE803F04402B0
:10FCD800302A17F0BFFE634B63491A784B8802F04D
:10FCE8000102002878D06148EB65D0ED037A002A3C
:10FCF80040F0868003FB04F007EE900ADFED5C6AB3
:10FD08005C4AB8EEE77AD5ED167AE7EE267AC2E9CC
:10FD18000033BDEEE77AC5ED167A85ED157A82EDEA
:10FD2800027A70BD534AC2E9003393607047524B60
:10FD38001B681B01F5D5FF200DF072FB18B1037885
:10FD48000A2B6BD9002003464A4AC5E93103C2E9A8
:10FD58000033906070BD494A494BD27933F812603C
:10FD6800B6B23046FFF716FD07EE906AA864B8EE03
:10FD7800670A4448F0F7E8FBBCEEC00A10EE103AF8
:10FD880098B2FFF707FDA96CD5ED107ADFED386A58
:10FD9800384B3D4A686401FB04F407EE104AB8EE9C
:10FDA800C77A1860E7EE267A107859602328BDEEE6
:10FDB800E77AC5ED107A17EE102A83ED027A85ED01
:10FDC8000F7AAED1314B9980DA8070BD294B002271
:10FDD800C3E900229A6070BD274E3668F60682D5C0
:10FDE800EB65002A86D0B1F90010294A00FB01F022
:10FDF80082FB0012C017C0EBA2100344EB6579E741
:10FE0800FDEEE77A234E17EE900AA0F57A7000FB14
:10FE180000F2A6FB026200EB1210E4E71E4A1F4B39
:10FE280051881A68D0ED027ADFED1D6A1D4C4368CF
:10FE380002FB01F207EE102AF8EEE77AB8EE477AED
:10FE4800A4FB0121E7EE267A03EBD103FDEEE77A66
:10FE580017EE900A78E700BF7F250020401D00209C
:10FE680090130020231E0020AC22002030320020F6
:10FE78002FE33E3168250020904A0020A83E00204C
:10FE8800D03E0020DC130020B01C0020B41C002051
:10FE9800D34D62101F85EB51182A0020603D0020C9
:10FEA8007D219534CDCCCCCCF8B53E4B5B7A012B7B
:10FEB80030D0022B0ED03C4B00221A603B4B1B78F3
:10FEC800022B00D0F8BD384A394B51881288198066
:10FED8005A80F8BD374B1B681B01EFD5FF200DF08A
:10FEE8009FFA00285AD003780A2B51D99FED320A7D
:10FEF8000023324C04F124006384F0F725FBBCEEA8
:10FF0800C00A10EE103A9BB22384274A618C5180B4
:10FF18001380D3E72A4A2B4B9278284C33F81210D7
:10FF2800294F8DB207EE905A04F13000B8EE670AF7
:10FF3800F0F70AFBBCEEC00A3978DFF890C07E788B
:10FF4800194810EE103A40F6E44202FB01F29BB267
:10FF580002FB05F102FB03F3ACFB0323ACFB01122C
:10FF680044F6FB71BD7801EBD30301EBD201C6EB7C
:10FF78000632B3FBF2F3B1FBF2F2B3FBF5F3B2FBDB
:10FF8800F5F29BB292B2A385E2850380428095E7A1
:10FF9800438807EE903AB8EE670AAAE7074C238C25
:10FFA800B3E700BF401D002078250020B01C0020CA
:10FFB800B41C0020904A002000000000901300208C
:10FFC800A83E0020D03E0020A0220020CDCCCCCCE2
:10FFD80070B54E68054630461DF04CF9314604466A
:10FFE800024628681EF001F82A68131901333B21DC
:08FFF8002B60115570BD00BF24
:020000040801F1
:100000002DE9F843954D2C68E00500F1CD80944A28
:10001000944B92F80080944F00221A70B8F1000FB0
:1000200000F0B28006219148F6F7FFFC002800F0AE
:10003000A68044F010048E4A8E4B16682C6016F48D
:100040008056B3F906905FD18B4B9B8A4B456EDC93
:1000500044F04004894B2C601B78190706D41B21FF
:100060008248F6F7E2FC002800F0C08024F080040B
:100070003B89642BB7F8CE308CBF44F4806424F401
:1000800080641BB17E4B1B689A0704D47D4BD3F868
:10009000AC30002B4ED044F400647B4B2C6003F159
:1000A000780102E006338B4216D01A781C2AF9D167
:1000B0009878DA78904202D35A79002AF2D01C213B
:1000C0006A48F6F7B2FC20B1704B1B785B0740F131
:1000D000948044F400742C601F216448F6F7A5FC5A
:1000E00058BBB8F1000F2ED0002C46D1002387F862
:1000F000D030FBF703FCD7F8D430C01A002841DB1E
:10010000BDE8F843FBF74CBC15215848F6F78DFCC9
:10011000002899D15E4B1A7B002A95D15649DA887E
:100120004B8A991A494593DA13444B4590DD24F0E4
:1001300040048FE724F40064AFE744F480342C607B
:10014000B8F1000F19D1534B1B78002B3AD19846C8
:10015000002E41D100214548F6F767FC002856D013
:10016000002CC3D0B8F1000F07D1002E49D020B920
:1001700024F480142C60002CB8D00223B7E724F0BC
:10018000100458E7BDE8F883434A97F8CC30167856
:100190007BBB7EB341463548F6F747FC00284AD181
:1001A00024F008042C6025E03C4A3D4B91791A6804
:1001B0004FF47A7303FB01F393429CBF24F48074E1
:1001C0002C6024E724F4801828F40068B8FA88F832
:1001D0004FEA5818002EBDD015212448F6F725FC0B
:1001E00018BB2B4B1B7B53B30646B3E744F080048C
:1001F0003EE766BB87F8CC6014E724F400742C60FB
:100200006AE70028B4D044F480142C60B5E724F0E9
:100210002004014615482C60F6F707FC3CB1B8F104
:10022000000FA4D1002EA2D1EBE7002692E7002810
:100230007FF45CAF9CE744F008042C60DAE724F418
:10024000801626F04006B6FA86F6760982E7414621
:100250000648F6F7EAFB0028CCD1A1E7B029002038
:10026000440F0020221E0020901300205C3000204C
:10027000904A0020D4290020E4590020241E0020A8
:10028000482A0020084400203C340020231E00207F
:1002900024390020A8300020482F0020245C0020B2
:1002A000603D0020314A324B10B5B2F906401B6860
:1002B000B4F5FA6FA8BF4FF4FA64B4F57A7FB8BF0B
:1002C0004FF47A74DB0410D42A4B9B8A6420E41A1E
:1002D00000FB04F0C3F5FA6390FBF3F06428A8BFB9
:1002E000642020EAE07040B210BD15212248F6F7E4
:1002F0009CFBB8B9214B187B0028E5D11D49DA8851
:100300004B8A9918A14225DB9B1AA342ECDD1C1BEA
:100310006FF06300A3F57A7300FB04F090FBF3F039
:1003200040B210BD134A154B908A1A7B241A6423DD
:10033000C0F5FA6003FB04F494FBF0F49C42A8BF00
:100340001C4624EAE474E0B212B1404240B210BD4F
:1003500060B210BDE01A841AC3F5FA6364209B1AD8
:1003600000FB04F090FBF3F040B210BDD429002054
:10037000904A0020E45900205C30002024390020FD
:100380006F4A1378D90700D470472DE9F04123F064
:1003900001036C4C1370FBF7B1FA6B4D2378C5F871
:1003A000D8001BBB694B1B78012B1FD0684B9A7878
:1003B0001ABB684B1B88002B4BD1674A674B1178DF
:1003C000186881F00101F1F71FFF654E33782BB1FA
:1003D00023781BB1634B1B68DA0443D5624B1B685F
:1003E00000229B0622702FD5BDE8F0815F4B0122D1
:1003F0001A70574B9A78002ADBD01B79022BD8D081
:100400005B4E33780B2B18D801229A4040F603013B
:1004100012EA0107CDD112F4C06F0ED0093B012BB7
:100420000BD845200FF0D8F9FF200FF0D5F951482F
:100430000FF0BEF938460FF0CFF94F4A4F4B126814
:100440005A600B233370B4E70420BDE8F041FBF79A
:1004500039BC4B4B5A69002AB7D0196800220A6090
:100460005A74B2E7474B1F78FBF748FA3378002BF2
:10047000B4D095F8686095F86930721C02F00302F8
:100480009A42ABD04FEA860808EB060105EB8101E2
:1004900000F51C50103085F868200A234FF47A725A
:1004A000C8660A6781F87530002F46D01421364897
:1004B00011FB063318443A461DF0BFFD334A138939
:1004C000012FB3FA83F34FEA53132ED0B2F86C1016
:1004D000002918BF0023022F27D0B2F8D01000291E
:1004E00018BF0023032F20D0B2F83411002918BF01
:1004F0000023042F19D0B2F89811002918BF002347
:10050000052F12D0B2F8FC11002918BF0023062FC6
:100510000BD0B2F86012002918BF0023072F04D0B7
:10052000B2F8C422002A18BF002383F00103464416
:1005300005EB860585F8743050E73B46F7E700BFCA
:10054000231E0020221E002090130020442A002099
:100550004C2500202C3F00202E3F0020303F002063
:10056000C24B0020904A0020B0290020672A0020BA
:10057000482500204C540308603D002088300020AE
:10058000343F002020590020FC130020D44B0020D1
:100590002DE9F04FDFF80893B04AD9F8DC10B04CE1
:1005A0001368C9F8DC002DED0E8BA0EB010B99B0A0
:1005B000257806905B441360002D53D0DFF8E4A249
:1005C000A84E9AF8005033788BBBA74AD9ED395A18
:1005D000D2ED017AA54BC9ED397A77EEA57A05EE11
:1005E00090BAD2ED023AD9ED3A4A92ED034A99ED2A
:1005F0003B5A93ED006A93ED027AD3ED016AC9ED9F
:100600003A3AFAEEEF5A73EEA44A34EE055AA5EEE2
:10061000A76AF0EE477AE5EEA46AE5EE257A83ED67
:10062000006AC3ED016A89ED3B4AC3ED027A052DEC
:1006300000F0EC808E4AD9F8F0301178B3FBF1F27B
:1006400001FB12320133C9F8F030002A00F0B58006
:100650009AF80030012B00F0CC8019B0BDEC0E8B65
:10066000BDE8F08F834C63682046984704900028CB
:1006700000F0D380D4F8AC6084F85C50002E41F0D8
:10068000E580B4F9503094ED085AD4ED095A94ED50
:100690000A6A94F85A1006EE903AB4F9523007EE0E
:1006A000103AB4F9543007EE903AF8EEE66AB8EE34
:1006B000C77AF8EEE77A76EEC56A37EE657A77EEB6
:1006C000C67A04F12C00C4ED0B6A84ED0C7AC4EDFB
:1006D0000D7A12F08BF9684B1D78002D01F0C8855A
:1006E000DFF8C0A1654A9AF800500B92B0462B463D
:1006F00004F12C0704F5CA761546B7EC018AD4ED4F
:10070000077A142B28EE278A02F03882062B08D1AC
:10071000B0EE480A07931DF011FC594B23F818005E
:10072000079B2A68910004D594F88426424503F07B
:100730001082B0EE480AD4F8903130469847D4F889
:10074000003206F170009847D4F8B030A6F1E0000E
:100750009847D4F82031A6F1700098472B689A008A
:10076000B0EE408A18D594F88436434503F0FF81F3
:10077000D7EDCC7AD4F8703277EE887AB0EE480AAA
:10078000C7EDCC7A06F1E4009847D4F8743206F548
:10079000A8709847B0EE408A9AF80030032B02F018
:1007A000F68108F10108B8F1030F87ED028A06F11E
:1007B0002406A2D11D4601F08FBD324B1B78002BC1
:1007C00072D0314B3149B3F906208B8A08919A4295
:1007D00000F346812E4B1B780E2B00F04181082B35
:1007E00000F03E812B4A2C490A92002393608B60D3
:1007F0005EE0D9F8E020224BD169B9F808201980D1
:100800005A8019B0BDEC0E8BBDE8F08FFBF776F87F
:10081000069A1B4B801A18800CE7DFF888A0D4F8E2
:10082000AC309AF80050002B00F03B820D4E1B4B71
:100830001B78002B3FF4C7AE162D01F02C82152D2E
:1008400041F0918294ED0E0A0D4F1DF077FB94ED6F
:100850000F0A38801DF072FB7880B4E674390020EE
:10086000B0300020BC370020F84300207839002049
:100870009830002008440020AC300020904A00202E
:10088000B41C0020440F0020D4290020E45900208B
:10089000043A00203032002030370020AD300020F4
:1008A00090130020B01C0020994B0893994B0A9399
:1008B00099F8F420002A40F0DA80974B0B93974B7D
:1008C0000C93089E96F82510012940F0418199F873
:1008D0002431934C002B40F0F081002096F82A50F0
:1008E00089F82411C4F89C004FF6FF7196F8260091
:1008F0002370C4F89830C4F8A030C4F8A410A4F849
:100900009400002D01F0408596F82710A4F8961069
:10091000002843F0E882002942F0CD87814F012171
:100920003D7889F82511002A40F0CC8105EA010BB9
:10093000AE1045FA01F14FEAE508089B93F829202B
:10094000BBF1000F41F06E85C90703F101835B46DF
:10095000F10740F11C8299ED4C7A002B42F07B812B
:100960000A9B18F0010F83ED027A04D099ED4D7ABD
:100970000A9B83ED037A99F8F420002A40F036822E
:10098000002D40F04A879AF80060052E01F099800A
:1009900000240C9B0699186813F0A4FD9AF8003007
:1009A000052B01F08780DFF8A4B19BF8007017F0E9
:1009B000010700F097825C4B1B78DE0600F1928203
:1009C0005A4B5B78002B00F08D8299F86831584CB7
:1009D000002B40F088822378002B40F0848299F825
:1009E0006931002B40F07F820B9B1B68DD0604F110
:1009F0008481504BDFED507A93ED097AB0EEC77ADF
:100A0000B4EEE77AF1EE10FA83F2D18793ED047A2F
:100A1000B0EEC77AB4EEE77AF1EE10FA83F2C78748
:100A200093ED0E7AB0EEC77AB4EEE77AF1EE10FAF3
:100A300083F2BD870023C9F86C319AF80030212B6E
:100A400040F05982D9F86C313C4A9BF80070003371
:100A500018BF01235380012313801F4000F0E5BE1F
:100A600099F8F4202B4B0A93002A3FF426AF344B1D
:100A70001B78002B3FF421AF324DB9F8F6302749EF
:100A8000254C08680C91A5FB03539B09642595FB35
:100A9000F3F50A9B2168D3ED037AD9F8F8300B946B
:100AA000BDEEE77A142D448EA8BF142517EE106A08
:100AB000CF0409EB430103F101034CBF640824B2E6
:100AC000A1F8FC609D4290F83010C9F8F830DCBF06
:100AD0000023C9F8F83001297FF4F3AE09EB430392
:100AE000B3F9FC3007EE103AB8EEC77A77EEC77A62
:100AF000FDEEE77A17EE903A1BB2002BB8BF5B42CF
:100B0000A34203F3CA84104B4FF07E511960D8E61C
:100B1000E459002030320020904A0020D8220020E2
:100B20003C590020105A0020241E0020983000203C
:100B3000221E0020F431002000001644B41C0020C6
:100B4000E9360020D34D621094070020231E0020B8
:100B5000357E002D00F03C81022D02F0BE86032D73
:100B600041F09784B37EC3EB431103EB8103DB00B9
:100B70009BB2002A01F0FD86002B01F0FA86CD4AD7
:100B8000CD4F1268B3FBF2F30FFA83FB07EE90BA76
:100B90003C78A9F83CB1B8EEE77AF7EE006A14F0B9
:100BA0000108C6EE877A0AD00A9BD9ED546A93ED04
:100BB000007A37EE667A27EE277A89ED507A66104A
:100BC000F2070AD50A9BD9ED556A93ED017A37EE03
:100BD000667A27EE277A89ED517AA510EB070AD5B8
:100BE0000A9BD9ED566A93ED027A37EE667A27EEC4
:100BF000277A89ED527AE410E0070AD50A9BD9EDED
:100C0000576A93ED037A37EE667A67EE277AC9ED75
:100C1000537A9AF80030072B03F0E483BBF1000FFE
:100C200040F3E4803C7804F001086610A510E4105D
:100C3000B8F1000F0AD099ED547AD9ED507A0A9B99
:100C400077EE877AC9ED547AC3ED007AF1070AD5B9
:100C500099ED557AD9ED517A0A9B77EE877AC9EDED
:100C6000557AC3ED017AEA070AD599ED567AD9ED9E
:100C7000527A0A9B77EE877AC9ED567AC3ED027AEB
:100C8000E3070AD5D9ED577A99ED537A0A9B77EEA7
:100C9000877AC9ED577AC3ED037A99F8F4200425D1
:100CA00098E0864BA26B5A60E16B226C844E99608F
:100CB000DA6094F854333370B9E57F4F23783D7888
:100CC000002A7ED099F8252115F0010B03D00A994E
:100CD0000968C9F828116910CE0703D50A98406839
:100CE000C9F82C01AE10F00703D50A988068C9F83E
:100CF00030014FEAE50818F0010F03D00A98C068E8
:100D0000C9F83401002A41F0C883002B3FF415AE26
:100D10009AF80030292B01F0AA83089B93F8292028
:100D2000BBF1000F01F0938399ED4A7AD4ED016A8B
:100D3000D4ED027A002A03F0CB80D4ED065A94ED6C
:100D4000073AD4ED033A94ED086A94ED044AD4EDE1
:100D5000094A94ED055A0A9B84ED067A65EEA77A56
:100D6000C4ED075AE7EE267A84ED096AE3EE237AAA
:100D7000E6EE447AE4EEC57AC4ED087AC3ED007A73
:100D8000CF0701F13887F30701F16387012318F0DA
:100D9000010F3FF4F0AD99ED4D7A002B3FF4E8AD33
:100DA000D4ED1C6AD4ED1D7A002A43F0A18037EE01
:100DB000667A0A9BE7EE276AC4ED1C6AC3ED036AF4
:100DC000D9E505F0010B6910AE104FEAE5089CE784
:100DD000A9F83C519AF80030072B7FF4CEAD394B7F
:100DE000B9F83C119980002A3FF4CAAD0223079359
:100DF000354A364BDFF8E480354F364DDFF8E0B04A
:100E00009FED358A049300241646B6EC010A2B6840
:100E100020EE080A2046F0EEC00AA8EC010AE7EC32
:100E2000010A9847DBF80030049A03EB440302EB15
:100E300084005B8A07EE903AF8EEE77AB1EE677AC3
:100E4000B4EEC70AF1EE10FA08D4B4EEE70AF1EEF8
:100E500010FA8CBFB0EE677AB0EE407A9AF80030A4
:100E600080ED007A082B06D1BDEEC00A154A10EEBF
:100E7000101A22F81410079A01349442C5DD072B8A
:100E80001E4608D1049BD3ED007A0E4BFDEEE77AA7
:100E900017EE902ADA80089BDC7E002C40F09585C6
:100EA00099F8F430002B3FF470AD002389F8F4304A
:100EB0006BE500BF38590020105A0020F84300208D
:100EC000BC370020B41C0020303200203037002016
:100ED00064370020243A00206F12033B543700206F
:100EE000DC360020DA4C9AF800300022212BC9F8B9
:100EF0006C2100F09884012B00F0C885052B00F0D0
:100F000029879BF800700023049307F001070C9BCE
:100F10001A680B9B92F846801B680A9AD80492EDD7
:100F2000038A40F13A84089B5D8A0FB9A9F874518D
:100F30001521C848F5F779FD20B9C74B1A7B002A5F
:100F400001F01B82089B9B8AA3F57A7303EBD37392
:100F5000C3F34F03EA1A1D4492B2ADB207EE902AD2
:100F6000F8EEE77AA2F57A73C5F5FA6107EE103A62
:100F700006EE901AF4EEC87AF1EE10FAB8EEC77ADF
:100F8000F8EEE66A99F9763103DA2178002901F062
:100F9000C281B24AB249D2ED006AB24A91ED006A0A
:100FA0001278C9ED5E6A89ED5F6A002A00F0DB8580
:100FB00076EE665A0133C9ED605AC9ED616A01F0F7
:100FC0001486069BC9F88831002277EEC87ABCEEF9
:100FD000C88AFF2318EE101AC9ED637AA9F87411B4
:100FE00089F87631A04B9A4240F2A78687EE878A2D
:100FF00023789E4D2C78F7EE007AB4EEE78AF1EE76
:1010000010FA88BFB0EE678AB5EEC08A9FED987A75
:10101000F1EE10FAB8BFB0EE478A89ED638A002B73
:1010200040F0DD83934B0C9A93F800C01068BCF13C
:10103000010F40F0058490F866108F4E8F4B012908
:1010400008BF1E46038D8E495A4207EE902A91ED45
:10105000046AF8EEE77A07EE103AB4EEE76AF1EECA
:1010600010FAB8EE477A00F1EE83B4EEC76AF1EEFB
:1010700010FA88BFB0EE476AD1ED096ADFED815AF8
:10108000F4EEE67AF1EE10FA26EE256A08DCB4EE0C
:10109000E67AF1EE10FA8CBFF0EE667AF0EE477A5F
:1010A000438D91ED0E7ADFED775A5A4206EE902A83
:1010B000F8EEE66A67EEA57AB4EEE67AF1EE10FA9B
:1010C0000AD406EE903AF8EE666AF4EEC76AF1EEDC
:1010D00010FA88BFF0EE476A6B4B9FED6A7A5B7837
:1010E00066EE876A0BB9F1EE666AB8F1000F40F060
:1010F0004085F7EE005A654B1B68197CC1B15B7CDB
:10110000632B13D807EE103A9FED615AB8EEC77AF9
:10111000012927EE057A02F0A087022906D1B4EE54
:10112000C78AF1EE10FA88BFB0EE478A89ED638A6C
:10113000584B1B78002B40F07C83BCF1010F41F031
:10114000E0809FED4B8A4FF0010889ED638A002C07
:1011500002F0CA83D6ED028AD6ED014A96ED035A13
:101160009FED437A67EEA88AE6EE248AE6EE858A4A
:1011700065EEA88AF4EEC78AF1EE10FA8CBFB0EEE5
:10118000479AB0EE689ACDED108AD8BFF0EE478A44
:10119000012C00F0FF8096ED067AD6ED054A96ED1B
:1011A000075A27EE877AA6EE247AA6EE857A25EEF0
:1011B000877AB4EEE87AF1EE10FA00F3B584B4EE73
:1011C000C79AF1EE10FA88BFB0EE479A022C8DED67
:1011D000117A00F0DF8096ED0A7AD6ED094A96ED95
:1011E0000B5A27EE877AA6EE247AA6EE857A25EEAC
:1011F000877AB4EEE87AF1EE10FA00F35185B4EE96
:10120000C79AF1EE10FA88BFB0EE479A032C8DED25
:10121000127A00F0BF8096ED0E7AD6ED0D4A96ED6B
:101220000F5A27EE877AA6EE247AA6EE857A25EE67
:10123000877AB4EEE87AF1EE10FA01F35E80B4EE4C
:10124000C79AF1EE10FA88BFB0EE479A24E000BFCB
:10125000221E00205C30002024390020302600208F
:1012600020390020C24B00208FD0030020590020DD
:1012700000000000442A00201C3800209C38002078
:10128000F43100206F12833A043A0020DC3600204B
:101290000AD7233C0A260020042C8DED137A79D03E
:1012A00096ED127AD6ED114A96ED135A27EE877A0B
:1012B000A6EE247AA6EE857A25EE877AB4EEE87A51
:1012C000F1EE10FA01F3F984B4EEC79AF1EE10FAD8
:1012D00088BFB0EE479A052C8DED147A5AD096ED62
:1012E000167AD6ED154A96ED175A27EE877AA6EEAE
:1012F000247AA6EE857A25EE877AB4EEE87AF1EEC6
:1013000010FA02F3CC82B4EEC79AF1EE10FA88BF5D
:10131000B0EE479A062C8DED157A3BD096ED1A7AF1
:10132000D6ED194A96ED1B5A27EE877AA6EE247A57
:10133000A6EE857A25EE877AB4EEE87AF1EE10FA19
:1013400002F3C782B4EEC79AF1EE10FA88BFB0EE8E
:10135000479A072C8DED167A1CD0D6ED1E4A96EDD5
:101360001D5A96ED1F7A67EEA47AE6EE057AE6EE50
:10137000877A65EEA77AF4EEE78AF1EE10FA02F1C9
:101380000484B4EEE79AF1EE10FA88BFB0EE679AE3
:10139000CDED177A78EEC99AE14B1B787BB9E14B1A
:1013A000E14AD3ED007AD3ED016A38EE677AE6EED2
:1013B000877A38EE677AC3ED007A82ED007AD9F841
:1013C0009431069941F28732CB1A934200F302849A
:1013D000D64BDFEDD76A93ED007AB4EEE67AF1EE04
:1013E00010FA20DDD34BD3ED007A93ED015A78EE5D
:1013F000675AB7EE006AE5EE257A78EE675AC3EDD4
:10140000007AA7EE258AB4EEC68AF1EE10FA88BFFC
:10141000B0EE468AB4EEE68AF1EE10FAB8BFB0EE4E
:10142000668A89ED638AB7EE007AC34AC34B82EDC0
:10143000008AF4EEC79AF1EE10FAC3ED009A40F379
:101440007783FCB3C7EE297A012C9DED107A27EE45
:10145000277A8DED107A35D09DED117A27EE277A17
:10146000022C8DED117A2DD09DED127A27EE277A80
:10147000032C8DED127A25D09DED137A27EE277A75
:10148000042C8DED137A1DD09DED147A27EE277A6A
:10149000052C8DED147A15D09DED157A27EE277A5F
:1014A000062C8DED157A0DD09DED167A27EE277A54
:1014B000072C8DED167A05D09DED177A67EE277A09
:1014C000CDED177AB8F1000F03D0B6EE008A89EDA2
:1014D000638A0B9B1B68DA0602D5002F40F06987F0
:1014E000002C00F01781964A964B92ED005A99ED28
:1014F0005E7ADA78D9ED5F5A99F9763199ED606ABA
:10150000D9ED617ABDEEC55A06EE903A15EE100A95
:101510008D4BBDEEC75AFDEEE55A1B78F8EEE66A34
:1015200015EE101A15EE90CA002A41F02E8296EDA3
:10153000007ADDED105A28EE077AA6EEA57AF0EED5
:10154000675AE6EE075ABDEEE57A17EE103A994271
:1015500000F31A846345A8BF634607EE103AB8EE5D
:10156000C77A7A4A012C82ED007A00F0CD8096EDA0
:10157000047ADDED115A28EE077AA6EEA57AF0EE90
:10158000675AE6EE075ABDEEE57A17EE103A994231
:1015900040F3BA8607EE101AB8EEC77A022C82ED35
:1015A000017A00F0B18096ED087ADDED125A28EE4E
:1015B000077AA6EEA57AF0EE675AE6EE075ABDEE78
:1015C000E57A17EE103A994201F37B836345A8BF91
:1015D000634607EE103AB8EEC77A032C82ED027A22
:1015E00000F0928096ED0C7ADDED135A28EE077A22
:1015F000A6EEA57AF0EE675AE6EE075ABDEEE57A5A
:1016000017EE103A994202F360816345A8BF634622
:1016100007EE103AB8EEC77A042C82ED037A73D045
:1016200096ED107ADDED145A28EE077AA6EEA57A2B
:10163000F0EE675AE6EE075ABDEEE57A17EE103A7D
:10164000994202F359816345A8BF634607EE103AF9
:10165000B8EEC77A052C82ED047A55D096ED147A4F
:10166000DDED155A28EE077AA6EEA57AF0EE675A58
:10167000E6EE075ABDEEE57A17EE103A994202F30C
:1016800088826345A8BF634607EE103AB8EEC77A72
:10169000062C82ED057A37D096ED187ADDED165AD4
:1016A00028EE077AA6EEA57AF0EE675AE6EE075A1C
:1016B000BDEEE57A17EE103A994202F34E84634587
:1016C000A8BF634607EE103AB8EEC77A072C82ED42
:1016D000067A19D096ED1C7ADDED175A28EE078AA6
:1016E000A6EEA58AE6EE087AFDEEE77A17EE903AC6
:1016F000994203DC9C456146A8BF194607EE901A43
:10170000F8EEE77AC2ED077A27B9A20010490F4830
:101710001CF06FFC0F4B1B7813B3002C6ED11BE039
:10172000E8360020D0360020EC360020E8370020D4
:1017300000000000283600204C320020F83600203F
:10174000F4370020A4250020C24B002034260020BE
:10175000F837002098580020DC4B20461B6898473B
:101760009AF80030052B00F07D81D94A1478002CBE
:101770007EF470AFD74DAA78002A40F09F829AF885
:101780000030052B7EF466AFFAF7B8F8D24A9AF823
:101790000030001BD080FEF75DBFD04BD04A93EDE8
:1017A000007AD04BDFEDD06A93ED006AD2ED007A7B
:1017B000CE4B89ED5E7A38EE668AF8EEE77A76EE01
:1017C000476A89ED617A93ED007AC9ED606A012379
:1017D00077EE887A89ED5F6A89F8763106E4002F22
:1017E00040F00083002C00F07187A200C049C1487E
:1017F0001CF0FFFBC04B1B78002BB1D0BD4FDFF8B6
:1018000020830026F0B2D8F80030B7EC010A9847E0
:101810002C780136A642F5DB9EE7022DA8BF0225F3
:101820000795FFF7E5BAAC4B1A6000230493FFF766
:101830006EBBBCF1010F3FF484AC4FF0010886E4AD
:10184000AE4EFFF7FFBBB0EE676A15E4AC4BAD4A96
:10185000B3F81AC01068DFF8CCA29F4F19789AF835
:10186000008042F2107505FB0CF5B5FBF0F5B4F9FC
:101870005000B7F906C0AE4207EE900A02F081832D
:1018800094ED197AD4F880E0F8EEE77A0EF10100D1
:1018900037EE277A0128C4F8800084ED197A02F027
:1018A000BE86D4ED1C5AD4ED1E6A07EE100A37EE40
:1018B000E56AB8EEC75A012E86EE057A37EE257A2C
:1018C00077EEC77A84ED1D7AE7EE866A84ED1C7A9E
:1018D000F0EE667AC4ED1F6AC4ED1E6A00F09386CE
:1018E000B4F9520094ED1A7A07EE900AD4F89400F5
:1018F000F8EEE77A00F1010E37EE277ABEF1010F1C
:10190000C4F894E084ED1A7A02F06C86D4ED215A82
:10191000D4ED236A07EE10EA37EEE56AB8EEC75A4F
:10192000012E86EE057A37EE257A77EEC77A84EDBA
:10193000227AE7EE866A84ED217AF0EE667AC4EDCB
:10194000246AC4ED236A00F0F985B4F9540094EDDB
:101950001B7A07EE900AD4F8A800F8EEE77A00F1B7
:10196000010E37EE277ABEF1010FC4F8A8E084ED2E
:101970001B7A00F01386D4ED265AD4ED286A07EEC0
:1019800010EA37EEE56AB8EEC75A012E86EE057A00
:1019900037EE257A77EEC77A84ED277AE6EE276A66
:1019A00084ED267AF0EE667AC4ED296AC4ED286AE1
:1019B00000F06686A7F806C0D4F8AC309AF800505C
:1019C000013BC4F8AC30FEF72EBF16214E48F5F7A8
:1019D0002CF800283FF464AA4C4B1B885F063FF5A7
:1019E0005FAA99F86031A34242F02885484B99EDEF
:1019F000590A93ED008A049B9FED466A93ED027AA3
:101A0000D3ED005ADFED446A60EE477A25EE800A96
:101A1000E5EE887AA7EE080AF4EEC67AF1EE10FA3F
:101A200088BFF0EE467AF4EEE67AF1EE10FAB4EE04
:101A3000C60AB4BFB0EE667AB0EE677AF1EE10FA7D
:101A40008CBFF0EE467AF0EE407AF4EEE67AF1EEF4
:101A500010FAB8BFF0EE667A83ED007AC3ED027A31
:101A6000FFF71EBAF9F74AFF9AF8003004991A4AAC
:101A7000401A052B908040F01781F9F73FFF144B77
:101A80001B780446002B7FF47AAE73E6F9F736FF35
:101A9000224AD9F8703112680F499BF800700490FF
:101AA000C31A9A1AC9F87001CA808B8007F001071F
:101AB000FFF72DBAF9F722FF074B001B5880FEF7FE
:101AC00072BFF9F71BFF0446FEF763BFCC4B002043
:101AD0004D2700204C250020B41C0020302600207B
:101AE000B03900205426002000007A443439002008
:101AF000F837002034260020985800201C38002099
:101B0000D0430020F84300205C300020082600204D
:101B10008801002000C0F94400C0F9C438590020F1
:101B2000C44B0020B01C0020F0EE478AFFF74EBBEC
:101B3000B8F1000F00F09184B1EE499AB4EEC89A62
:101B4000F1EE10FA0ADCB7EE009A39EE689AB4EEBC
:101B5000C89AF1EE10FA88BFB0EE489AB0EE498A02
:101B600089ED639AB5E476EEC65AF0EE466AFFF761
:101B700021BA874B597A00293FF4BBAA85490978D5
:101B800000293FF4B6AA1B889FED834A07EE103A5E
:101B9000824BF8EE475A1B8807EE101A05EE103AF2
:101BA000B8EEC77AB8EE455A25EE877AF7EE004AC6
:101BB000C7EE055AF4EEC45AF1EE10FA88BFF0EE03
:101BC000445AF4EEE45AF1EE10FAB8BFF0EE645A5B
:101BD000FFF791BA9FED720A28EE000A1CF0AEF9E9
:101BE000704B07905B6898423FF4F2AB6E4BDFEDB1
:101BF0006F7A1B780A9307EE100AB8EEC7AA2AEE8E
